S01B00004170706C69636174696F6E5F706362313032372E7372656337
S113A000F0FE002081AC000083AF000083AF0000AD
S113A01083AF000083AF000083AF000000000000A6
S113A0200000000000000000000000008FA80100F4
S113A03083AF00000000000005A9010083AF000009
S113A04083AF000083AF000083AF000083AF000044
S113A05083AF000083AF000083AF000083AF000034
S113A06083AF000083AF000083AF000083AF000024
S113A07083AF000083AF000083AF000083AF000014
S113A400FFFFFFFFFFFFFFFFFFFFFFFFFEFFFFFF59
S113A4100000000000000000000000000000000038
S113A4205630312D30322E303531373000000000B7
S113A4300000000000000000000000000000000018
S113A4400000000000000000000000000000000008
S113A45000000000000000000000000000000000F8
S113A46000000000000000000000000000000000E8
S113A47000000000000000000000000000000000D8
S113A48000000000000000000000000000000000C8
S113A49000000000000000000000000000000000B8
S113A4A04175672020312032303134000000000033
S113A4B00000000000000000000000000000000098
S113A4C00000000000000000000000000000000088
S113A4D00000000000000000000000000000000078
S113A4E00000000000000000000000000000000068
S113A4F00000000000000000000000000000000058
S113A5000000000000000000000000000000000047
S113A5100000000000000000000000000000000037
S113A52031313A34353A3434000000000000000080
S113A5300000000000000000000000000000000017
S113A5400000000000000000000000000000000007
S113A55000000000000000000000000000000000F7
S113A56000000000000000000000000000000000E7
S113A57000000000000000000000000000000000D7
S113A58000000000000000000000000000000000C7
S113A59000000000000000000000000000000000B7
S113A5A000000000000000000000000000000000A7
S113A5B00000000000000000000000000000000097
S113A5C00000000000000000000000000000000087
S113A5D00000000000000000000000000000000077
S113A5E00000000000000000000000000000000067
S113A5F00000000000000000000000000000000057
S113A6000000000000000000000000000000000046
S113A6100000000000000000000000000000000036
S113A6204DF8044D40F61011C1F6FF711EC980E8C3
S113A6301E0010BC704700BFAFF30080AFF3008072
S113A6402DE9F0038946904698E81E0040F620174D
S113A650C1F6FF7724EA020503EA020635432944DA
S113A660066831443E68314402EB716123EA010516
S113A67002EA010635432C44466834447E68344477
S113A68001EB345422EA040501EA040635432B4461
S113A69086683344BE68334404EBF33321EA03058C
S113A6A004EA030635432A44C6683244FE68324449
S113A6B003EBB22224EA020503EA020635432944E5
S113A6C0066931443E69314402EB716123EA0105B4
S113A6D002EA010635432C44466934447E69344415
S113A6E001EB345422EA040501EA040635432B4401
S113A6F086693344BE69334404EBF33321EA03052A
S113A70004EA030635432A44C6693244FE693244E6
S113A71003EBB22224EA020503EA02063543294484
S113A720066A31443E6A314402EB716123EA010551
S113A73002EA010635432C44466A34447E6A3444B2
S113A74001EB345422EA040501EA040635432B44A0
S113A750866A3344BE6A334404EBF33321EA0305C7
S113A76004EA030635432A44C66A3244FE6A324484
S113A77003EBB22224EA020503EA02063543294424
S113A780066B31443E6B314402EB716123EA0105EF
S113A79002EA010635432C44466B34447E6B344450
S113A7A001EB345422EA040501EA040635432B4440
S113A7B0866B3344BE6B334404EBF33321EA030565
S113A7C004EA030635432A44C66B3244FE6B324422
S113A7D003EBB22223EA040502EA040635432944C2
S113A7E0466831443E6C314402EBF16122EA0305D0
S113A7F001EA030635432C44866934447E6C3444B0
S113A80001EBF45421EA020504EA020635432B4421
S113A810C66A3344BE6C334404EBB34324EA0105F3
S113A82003EA010635432A4406683244FE6C324486
S113A83003EB323223EA040502EA040635432944D1
S113A840466931443E6D314402EBF16122EA03056D
S113A85001EA030635432C44866A34447E6D34444D
S113A86001EBF45421EA020504EA020635432B44C1
S113A870C66B3344BE6D334404EBB34324EA010591
S113A88003EA010635432A4406693244FE6D324424
S113A89003EB323223EA040502EA04063543294471
S113A8A0466A31443E6E314402EBF16122EA03050B
S113A8B001EA030635432C44866B34447E6E3444EB
S113A8C001EBF45421EA020504EA020635432B4461
S113A8D0C6683344BE6E334404EBB34324EA010533
S113A8E003EA010635432A44066A3244FE6E3244C2
S113A8F003EB323223EA040502EA04063543294411
S113A900466B31443E6F314402EBF16122EA0305A8
S113A91001EA030635432C44866834447E6F34448C
S113A92001EBF45421EA020504EA020635432B4400
S113A930C6693344BE6F334404EBB34324EA0105D0
S113A94003EA010635432A44066B3244FE6F32445F
S113A95003EB323282EA03056540294446693144F7
S113A960D7F88060314402EB317181EA02055D4021
S113A9702C44066A3444D7F88460344401EB74549C
S113A98084EA010555402B44C66A3344D7F88860ED
S113A990334404EB334383EA04054D402A44866B75
S113A9A03244D7F88C60324403EB722282EA030506
S113A9B06540294446683144D7F89060314402EB3D
S113A9C0317181EA02055D402C4406693444D7F8AC
S113A9D09460344401EB745484EA010555402B44DB
S113A9E0C6693344D7F89860334404EB334383EAAD
S113A9F004054D402A44866A3244D7F89C603244A8
S113AA0003EB722282EA030565402944466B314414
S113AA10D7F8A060314402EB317181EA02055D4050
S113AA202C4406683444D7F8A460344401EB7454CD
S113AA3084EA010555402B44C6683344D7F8A8601E
S113AA40334404EB334383EA04054D402A448669C6
S113AA503244D7F8AC60324403EB722282EA030535
S113AA6065402944466A3144D7F8B060314402EB6A
S113AA70317181EA02055D402C44066B3444D7F8F9
S113AA80B460344401EB745484EA010555402B440A
S113AA90C66B3344D7F8B860334404EB334383EADA
S113AAA004054D402A4486683244D7F8BC603244D9
S113AAB003EB722262EA04055D40294406683144CE
S113AAC0D7F8C060314402EBB16161EA0305554037
S113AAD02C44C6693444D7F8C460344401EBB454FC
S113AAE064EA02054D402B44866B3344D7F8C860B2
S113AAF0334404EB734363EA010565402A44466921
S113AB003244D7F8CC60324403EBF22262EA040503
S113AB105D402944066B3144D7F8D060314402EBE0
S113AB20B16161EA030555402C44C6683444D7F842
S113AB30D460344401EBB45464EA02054D402B4420
S113AB40866A3344D7F8D860334404EB734363EA2A
S113AB50010565402A4446683244D7F8DC60324433
S113AB6003EBF22262EA04055D402944066A31449B
S113AB70D7F8E060314402EBB16161EA0305554066
S113AB802C44C66B3444D7F8E460344401EBB45429
S113AB9064EA02054D402B4486693344D7F8E860E3
S113ABA0334404EB734363EA010565402A44466B6E
S113ABB03244D7F8EC60324403EBF22262EA040533
S113ABC05D40294406693144D7F8F060314402EB12
S113ABD0B16161EA030555402C44C66A3444D7F890
S113ABE0F460344401EBB45464EA02054D402B4450
S113ABF086683344D7F8F860334404EB734363EA5C
S113AC00010565402A44466A3244D7F8FC60324460
S113AC1003EBF222D8F800502944D8F804502A440F
S113AC20D8F808502B44D8F80C502C4488E81E005F
S113AC3000F14000B9F101097FF40CADBDE8F00367
S113AC40704700BFAFF30080AFF30080AFF3008024
S113AC502DE9F04140F61018C1F6FF7898E8F000AD
S113AC6082E8F000FFF7ECFCBDE8F081AFF3008070
S113AC700A464FF00101E3E4AFF30080AFF3008034
S113AC800F481049104A4FF0080333B140F8042B21
S113AC9041F8042BA3F10103F7E7EFF3088080F3F5
S113ACA00988EFF3148040F0020080F3148800F068
S113ACB00DB880F308887047000000000000000011
S113ACC080E100E080E200E0FFFFFFFFC046C046F5
S113ACD0C046C04600F000F800F00BF8002801D090
S113ACE000F00CF80020C046C04600F01BF800F04D
S113ACF021F880B500F054F8012002BD10B50749D1
S113AD0079441831064C7C44163404E00A68081D62
S113AD10511888470146A142F8D110BD280301000B
S113AD208803010080B5024800F066F8002002BDE7
S113AD3014B0010000F020B9012080F3138870479B
S113AD40002080F31388704780B5FFF7F5FF26488D
S113AD504CF22051C1814DF62811C181D1210180CD
S113AD604FF47A71C18000218180C18215E080B5E1
S113AD70FFF7E2FF1D484AF2026101804BF2804175
S113AD800AE080B5FFF7D8FF17484CF22051C18183
S113AD904DF62811C181D0210180BDE80140CFE7E3
S113ADA010B5134C2069C0F3033040B91148016851
S113ADB021F019010160416821F01901416000F09E
S113ADC05BFA00F073FB00F015FE4FF08840206042
S113ADD0FFF7B2FF4AF20261044801804BF280415E
S113ADE00180BDE81040ABE7002005400C20054081
S113ADF01480044004F00140F0B5064683B0706846
S113AE00584D0F30040924012C604FF451710FF296
S113AE10601020600FF25C102060204600F006FEF7
S113AE2004F5D2703146302200F08CFEC4F8A841FB
S113AE30D4F8AC0100090001C4F8AC0100F0BEFE76
S113AE4000F02AFF10B100F039FFFEE7D4F8B0613A
S113AE50D4F8CC719FB9D82E3CBFD820C4F8B00127
S113AE60D4F8B00100F11006304600F037FF0700B7
S113AE7002D100F023FFFEE7022100F039FF314642
S113AE80384600F0F6FFF019401E00090001E063A7
S113AE90D82000F023FF060002D100F00FFFFEE7E8
S113AEA0012100F025FF06F1D7000009000104F19B
S113AEB05001A0F164024A61086106F10F00000923
S113AEC0000188614869686001F016F810B100F06B
S113AED0F5FEFEE7012104F5EA7001F041F80121D5
S113AEE004F5A47001F03CF801F068F810B100F02A
S113AEF0E5FEFEE7D4E9BE010A3041F10001C4E9F0
S113AF00BE0101230020019000900022E069C16885
S113AF1004F5357000F0F2FE10B900F0CFFEFEE744
S113AF2000F0B0FFD4F8B45102E000F0ABFF2035DC
S113AF30286888B1287DC007F9D5002001900090C9
S113AF400023E069AA69C168284600F0D7FE0028FA
S113AF50EBD100F0B3FEFEE70FF082FC002003B05B
S113AF60F0BD0000200AFF1F80B500F0A7FEFEE739
S113AF7000000803C0AF01000746384601F0CAF8D4
S113AF80FBE7FEE770B40022010003D0012808BFEC
S113AF90012200E00422DFF860341C7814F0C004BD
S113AFA00ED0402C07D0802C0CD15C7964064CBFA9
S113AFB00324022407E05C78640804F0010402E03E
S113AFC0042400E000240FF2504504EB84045519D6
S113AFD0645D042C00F2EB80DFE804F00344569D2A
S113AFE0D00000B3012840F0E28047251D702525DC
S113AFF05D70DFF80864DD7805F01F05DD7000255D
S113B0003570DFF8FC532E68760876002E60002534
S113B0101D715D719D79ED06FCD59D7905F00C05DA
S113B020042DFAD1C3E044251D7025255D70DFF899
S113B030CC63DD7805F01F05DD7000253570DFF881
S113B040C0532E68760876002E6001251D710025F8
S113B0505D719D79ED06FCD59D7905F00C05042DF7
S113B060FAD1A4E0012840F0A28047251D702725CD
S113B0705D700025DFF8846335709D79ED06FCD59D
S113B0809D79ED07FCD592E018B3012840F08F803C
S113B0900025DFF868633570DFF864532E6876089E
S113B0A076002E6025255D709B251D70DD7805F0EA
S113B0B01F05DD7000251D715D719D79AD07FCD5FF
S113B0C09D79ED06FCD49D7905F00C05082DFAD187
S113B0D06DE00025DFF824633570DFF824532E6813
S113B0E0760876002E6025255D7098251D70DD7824
S113B0F005F01F05DD7001251D7100255D719D7929
S113B100AD07FCD59D79ED06FCD49D7905F00C05C1
S113B110082DFAD14BE0C8B1012848D10025DFF849
S113B120DC623570DFF8D8522E68760876002E601F
S113B1309B251D7025255D7002251D7140255D71BF
S113B1409D7905F00C05082DFAD130E00025DFF8D3
S113B150AC623570DFF8A8522E68760876002E604F
S113B16098251D7025255D7001251D7140255D7193
S113B1709D7905F00C05082DFAD118E0B8B9002521
S113B1809E4E35709E4D2E68760876002E601825EA
S113B1901D7025255D7001251D7140255D719D790A
S113B1A005F00C050C2DFAD19D796D06FCD5A24253
S113B1B07FF409AF70BC704770B50446032801D30F
S113B1C0022070BD18B1022837D01BD350E0884844
S113B1D08B4D007802280DD18A4E307800F0DF00C4
S113B1E03070894828640020FFF7CCFE307840F0A6
S113B1F02000307085482864686C20F00D0040F011
S113B20002002BE07A487E4D007802280DD17D4E55
S113B210307800F0DF0030707B4828640020FFF7AE
S113B220B1FE307840F02000307079482864686CB2
S113B23020F00D0040F0020010E0724E704D3078A6
S113B24000F0DF003070704828640120FFF79AFE98
S113B2504FF440302864686C000900016864286871
S113B26040F4803028606B48016841F4002101609B
S113B2705F480470002070BD80B5FFF765FD0121B3
S113B2805D4891F8FE13FF290AD0817040F2FE3226
S113B290C178127801F0E00102F01F021143C1707D
S113B2A057495A4A0A644A6C22F00D0242F00202DB
S113B2B04A640A6842F480320A60564A136843F4C6
S113B2C00023136000234D4A13700B685B085B0076
S113B2D00B602523437098230370C37803F01F0386
S113B2E0C370012303710023437183799B07FCD549
S113B2F08379DB06FCD4837903F00C03082BFAD1A1
S113B300002313700B685B085B000B6098230370C9
S113B310252343700123037140234371837903F090
S113B3200C03082BFAD1002313700A685208520048
S113B3300A60182202702522427001220271402202
S113B3404271827902F00C020C2AFAD182795206F7
S113B350FCD5427942F020024271486B40F40070FF
S113B360486301BD10B50446FFF726FF38B9002134
S113B370204600F0DBFEC82100F01AFE002010BDBC
S113B38000BF1B4800787047032838BF1E2908D225
S113B39000EB80020FF29C0000EBC20050F8210089
S113B3A07047002070471248007801281AD11148CC
S113B3B01E2181700A21C170802101700178090663
S113B3C0FCD4017889060BD41F2181708021C170BF
S113B3D0C021017001780906FCD40078800603D5E9
S113B3E01B207047012070470020704700000000B8
S113B3F04D1EFF1F08400640004006400050064016
S113B400048004400540064000003301000013019D
S113B410000077770070044000010202020001007E
S113B42000000000020303020202030403030303F7
S113B4300400000000D8B805006CDC02006CDC02DB
S113B44000366E01006CDC0200D8B8050000000074
S113B4500000000000800000093D0000001BB70050
S113B460001BB700001BB700001BB700006CDC0218
S113B47000D8B805000000000000000000800000B3
S113B480093D000080841E0080841E0080841E000C
S113B49020A10700000000000000000080841E00BE
S113B4A0000000000080000000400000DFF83414B9
S113B4B0112008707047DFF830144FF48070086072
S113B4C00020DFF828140860DFF82404016841F044
S113B4D0400101607047DFF81C04016841F48051A9
S113B4E001600022DFF81004042142700270C2706F
S113B4F0827042710271C27182710830491EF4D1A6
S113B500DFF8F80360210170012141708270017835
S113B51041F0800101707047DFF8E4134FF480704C
S113B52008600020DFF8DC130860DFF8DC03016842
S113B53041F0800101607047DFF8D0134FF4807050
S113B54008600120DFF8C8130860DFF8C803016849
S113B55041F4000101607047DFF8BC13012808685A
S113B56000F4E0602AD1B0F5407F35D04FF440704C
S113B5700860DFF8A803016841F080710160DFF81A
S113B580A003416F490603D5416D41F004014165B3
S113B590416DE44A41F0010141650021016014213B
S113B5A041610821016040F202211160416D4907A7
S113B5B012D5416F41F0400141677047B0F5807F7B
S113B5C00AD04FF4807008600120D7490860D7483A
S113B5D0016841F0100101607047CF48006800F431
S113B5E0E060B0F5407F01D1012070470020704732
S113B5F0CF484FF4807101614161C1618161C160D3
S113B6008160416001600021CA4801614161C161FA
S113B6108161C160816041600160C748016841F493
S113B62080510160016841F400510160016841F4F6
S113B63000410160016841F480410160016841F406
S113B64000610160016841F480610160016841F4B6
S113B65000710160016841F4807101607047B7496D
S113B66041F23420088070470005A349000D08808A
S113B6707047B3490A78497800204B0648BF012037
S113B6800B0648BF40F00200530748BF40F00400D7
S113B6908B0648BF40F008008B0748BF40F01000FD
S113B6A04B0748BF40F02000930748BF40F04000DC
S113B6B001F0010102F00102114318BF40F08000C3
S113B6C07047A0484FF48071016041608160C1609F
S113B6D00161416181617F219B48416000210160DA
S113B6E0016941F07F01016170479749C24302F04B
S113B6F07F024A6000F07F00086070479348854AE3
S113B70040F203110160136823F480331360416035
S113B710136823F4003313608160136823F48023D7
S113B7201360C160136823F400231360016113687C
S113B73023F4801313604161136823F4001313602E
S113B74081614FF4FE01106820F48000106080488D
S113B75001601F2181600121016070477D480068FC
S113B760C0F3034080F00F0070477A480068000D72
S113B77002E078480068400D00F0010080F001000C
S113B780704774480068800DF6E7734A73494FF4B4
S113B790807010600B6823F020030B604B6943F04A
S113B7A020034B61D0610B6823F480530B604B6919
S113B7B043F480534B6110620B6823F400530B6015
S113B7C04B6943F400534B6150620B6823F480438C
S113B7D00B604B6943F480434B6190620B6823F424
S113B7E000430B604B6943F400434B61D0620B6828
S113B7F023F480330B604B6943F480334B61106353
S113B8000A6822F400320A604A6942F400324A614A
S113B810534A10600B6C23F008030B644B6D43F028
S113B82008034B6590610A6C22F400720A644A6D45
S113B83042F400724A654B494B4A10600B6823F08E
S113B84080030B604B6943F080034B6150620B68CB
S113B85023F480330B604B6943F480334B61906273
S113B8600A6822F400320A604A6942F400324A61EA
S113B8703E4A10600B6C23F010030B644B6D43F0D5
S113B88010034B6550600B6C23F020030B644B6D6D
S113B89043F020034B6590600A6C22F040020A6476
S113B8A04A6D42F040024A653149324A10600B68E1
S113B8B023F080730B604B6943F080734B615060DD
S113B8C00B6823F000730B604B6943F000734B610A
S113B8D09060086820F080600860486940F08060EB
S113B8E04861704700D0074018D004401820FE4338
S113B8F014F10F402C80044000C00C4021C00C40C7
S113B9001CC004401C18FE43D4F00F405CA004404B
S113B9105C08FE4354F00F40109004403C80044007
S113B92000800340948003401000FE4314F00F4055
S113B93020B004402010FE4394F00F400E20054038
S113B94000E0074000B0044084F00F4040A00440F1
S113B950C0A0044050F00F401490044000F00F4089
S113B9600CA0044080F00F401CB0044010C0044000
S113B97000F10F4060D0044003281CD1C80704D54F
S113B98023484FF4507242600260880703D50022B6
S113B9901F4842600260480704D51E48026842F40A
S113B9A000520260080704D51A48016821F40051C6
S113B9B00160002070470FE001600020704758B913
S113B9C016484FF4007141608160C1600160124803
S113B9D0016841F48051EFE74FF0FF3070471048A1
S113B9E0016841F4A0210160016B41F480210163ED
S113B9F0002070470B48016841F47851DCE70328C4
S113BA0003D109494FF440700860002070470000DA
S113BA1010D00440348004403C80044000C0044002
S113BA20048004403880044048B00440024604299D
S113BA306ED3C30704D5002002F8010B491E10463B
S113BA40820703D5002220F8022B891E8A0922D0FE
S113BA50002340F8043B40F8043B40F8043B40F822
S113BA60043B40F8043B40F8043B40F8043B40F8F6
S113BA70043B40F8043B40F8043B40F8043B40F8E6
S113BA80043B40F8043B40F8043B40F8043B40F8D6
S113BA90043B521EDCD18A0802F00F02521E0E2A09
S113BAA036D8DFE802F0322F2C292623201D1A175E
S113BAB014110E0B0800002240F8042B002240F859
S113BAC0042B002240F8042B002240F8042B00220F
S113BAD040F8042B002240F8042B002240F8042BE9
S113BAE0002240F8042B002240F8042B002240F8E6
S113BAF0042B002240F8042B002240F8042B0022DF
S113BB0040F8042B002240F8042B002240F8042BB8
S113BB108A0744BF002220F8022BC90744BF002132
S113BB200170704762B38B0708D0521E11F8013BB5
S113BB3000F8013B00F024808B07F6D1830740F026
S113BB40208000BF103A07D330B4B1E83810103A5F
S113BB50A0E83810F9D230BC530724BFB1E808106C
S113BB60A0E8081044BF51F8043B40F8043BD20756
S113BB7024BF31F8022B20F8022B44BF0B7803704A
S113BB807047083A07D3B1E80810083A40F8043B74
S113BB9040F804CBF7D25307E4E750F8041B61B133
S113BBA050F8042BD30744BFA9F101039A180023CA
S113BBB042F8043B091FFAD1EFE7704738B52F4824
S113BBC0046843F6F83020824FF4D5706082082070
S113BBD02060012060600220E0810F206081A0814C
S113BBE0D4F8B40110B90120FFF7BEF90120C4F85C
S113BBF0F402C4F8180100F061F904F15000E061A6
S113BC004FF6FF75E18A6183E18A8184D4F8A41137
S113BC1045EA0141C1600321816004F59E70002161
S113BC2000F086FA002104F5BE7000F081FAD4F821
S113BC30B411002005E0CA68904238BF1046203194
S113BC406D1E0A68002A18BF002DF4D104F5357161
S113BC50C4F81401401C0A4A0A60E0228A600FF208
S113BC6028020A61074A4A60C860002104F58E7000
S113BC7000F05EFA0120C4F8280131BD200AFF1F3C
S113BC8003000080A98E01005F6D71785F69646CA8
S113BC90655F7461736B000080B50748026802F544
S113BCA05170C2F8140300F13001D2F8AC21521AD9
S113BCB000F044FA002002BD200AFF1F0648006875
S113BCC0C169496D11B9C18A81F31188C069416D97
S113BCD0491C4165704700BF200AFF1F03490968DA
S113BCE0D1F814230023503100F05ABA200AFF1F60
S113BCF010B120F8021C0120704700002DE9F44F18
S113BD0005466C48D0F8008084B08946D8F8140100
S113BD10E9681C46884205D208F53570854218BF8B
S113BD200E202DD1DDF838B0BBF1000F13D00F9FDA
S113BD30B7F5C87F98BF022022D900235A4602A92A
S113BD40384600F005FB06460298A7EB000AACB1A2
S113BD50AAF1200A12E0A868D92838BFD8200F30E9
S113BD6000094FEA001A002C14BF0AF120005046C3
S113BD700023002202A900F0EBFA064626B90A20A5
S113BD8000F03AFB002071E00320B06037690FB97E
S113BD90029887196CB1B5E80E5038462037A0E8F0
S113BDA00E500ECD0EC0A0F12005286840F00040D2
S113BDB028604FEA9A013846491C3F4A01E040F89E
S113BDC0042B491EFBD1E868D8F82010000140423A
S113BDD04018F0613062BBF1000F8189B184696958
S113BDE018BF41F02001B1622B46049901915246DB
S113BDF0808900903946304600F016FBB0B3B56632
S113BE0028687066E86938B1D6E92823002110183B
S113BE105941C6E9280107E008F53E71B1E80C1064
S113BE2006F1A000A0E80C1008F52670C16D0229E7
S113BE3003D1B16A41F00401B162BBF1000FD8F83B
S113BE40981271674168B1678068F067C6F86090BE
S113BE500BD13146304600F00FFB002C14BFA7F184
S113BE6020003846314600F007FB304605B0BDE8F7
S113BE70F08F8908491C104A01E040F8042B491E40
S113BE80FBD170470B490968C269D1F824C05368D3
S113BE90944538BF4A620221816043601968016099
S113BEA0186050600021C0F8AC10C0F8B010C0F8A1
S113BEB0B4107047200AFF1F6B61747380B5254866
S113BEC0006800F5D2714A69082A28BF072201D206
S113BED00AB901224A61510101F0E001C182C02284
S113BEE06A211D4800F0CCFA1C494FF0FF3008606D
S113BEF048608860C86001BD70B5164804680020B9
S113BF002062D4F81401861C300100F0D7FA050031
S113BF1001D1042070BD0521FFF7EAFEB6B1D4F8C3
S113BF20B8018119491E2D60761E6D60EE810729C6
S113BF303DBF8219520102F0E002C022AA81491ECB
S113BF40226AAA6025621035002EECD1206A606254
S113BF50002070BD200AFF1F00E400E080E100E043
S113BF6038B5044610480568A16104F108000021B1
S113BF7000F0DEF8FFF7A2FED5F83C1105F59E703F
S113BF8000E00968814206D0A142FAD100F0A0FA8B
S113BF904FF4826032BD214600F0AEFA034860617E
S113BFA000F096FA002032BD200AFF1F6D73776CF3
S113BFB0B0FBF1F04B49401E0860704710B542F2E7
S113BFC0620000F0B5FA4FF00051002000F0BEFA14
S113BFD0FA21002000F0C8FA002865D1424800F098
S113BFE0CDFA0F2000F0D4FA00220FF2C1010F2085
S113BFF000F0D6FAF8B100F097F83C4C002100F0BC
S113C00095F8C821B0FBF1F0401E60600720206065
S113C0103748016841F080510160416841F0804136
S113C02041600120FFF79EF928B9FFF7BCF910B968
S113C030FFF798F908B1262010BD2E4804682E4851
S113C040C4F89401C82000F0F1FAD4F8940100F087
S113C050F5FA00210FF2590000F0F8FA00F000FBA5
S113C06000F008FB00BB254C0FF29800214600F0BD
S113C07076FB21460FF2940002F081F802F0DAF91F
S113C080FFF719FAFFF727FAFFF746FAFFF754FA12
S113C0900120FFF761FAFFF7ABFAFFF712FBFFF796
S113C0A02DFBFFF772FB002010BD000002F0DAB98F
S113C0B00C49DFF84CC00A684B68DCF800C0120277
S113C0C0120A1B020020521C1B0A5FEA4C1C03D5F7
S113C0D0486803021B0A104603B91346D11A4018D4
S113C0E07047000014E000E00000FF1F10E000E0D3
S113C0F01CED00E0200AFF1F00530700E4AF01001D
S113C10004ED00E0737069303A00000069737069EF
S113C110303A000080B5C046C046024A11001820DB
S113C120ABBEFBE726000200FFF72AB9FFF72CB9E4
S113C13000604060002202814181704770B504466E
S113C14015480568501800090001206101F10F002D
S113C15000090001E060E0622169091A0160002120
S113C160816044606061A061E0612062FFF7A6FD28
S113C17005F54276D5F8080318B900213046FFF7D3
S113C180D7FF2146304600F0B7F900F0A1F9034883
S113C190A060204670BD0000200AFF1F70656D6C12
S113C1A02DE9F843154604468846A86867490027E0
S113C1B09946884201D0382054E004F10C0010283C
S113C1C038BF10200F3000090401FFF777FD6E69B6
S113C1D001E03746B668002E41D0AE6100F078F930
S113C1E0FFF76CFDAE696869864208BF3746306860
S113C1F0A042EED3011B102907D3A01901604560AA
S113C200B1688160B060346001E00446B068696977
S113C2108E420CBF6861B8606869A8616869E861AA
S113C22068692862E8686862E868A862D8F80C005F
S113C2303081002070817560E86AB04238BFEE62D8
S113C24000F046F9B9F1000F05D0A4F10C0106F194
S113C2500C00FFF7EBFB06F10C00BDE8F28300F0E5
S113C26037F9042000F0C8F80020BDE8F2832DE976
S113C270FC471F4604468846B86834490025914661
S113C280884201D038205CE004F10C00102838BF4B
S113C29010200F3000090601FFF710FD786906EB46
S113C2A00801A1F10C0AA8F10C0401E0054680681C
S113C2B0002843D0B86100F00BF9FFF7FFFCB86920
S113C2C07969884208BF0546016800F1100294426A
S113C2D024BF0A185245E9D3221A891B891A02601D
S113C2E0102906D332191160576081689160826009
S113C2F001E08E198268AA602660A2607969B9613A
S113C3007969F96179693962F9687962F968B962B8
S113C310D9F80C102181002161816760F96A81429A
S113C32038BFF86200F0D4F80A9820B1A6F10C01E5
S113C3304046FFF77BFB4046BDE8F68700F0C8F8AF
S113C340042000F059F80020BDE8F68770656D6C94
S113C350F8B5054627480768B7F8240114464FF690
S113C360FE72904213DAB820086024B1B821204646
S113C370FFF75CFB15E000F0A1F8040007D02846A5
S113C38000F0DCF8206120B9204602F0F5F8002026
S113C390F2BD24212046FFF7ABFC20692521FFF7DD
S113C3A0A7FC07F592756E68D7F8A401A968B6B220
S113C3B046EA0040E06007F58E7700290CBF394655
S113C3C06C3104F16C02384602F042F92046014611
S113C3D0761CC86EA0F16C021046B6B206B90126EE
S113C3E0BA4203D0D26892B2B242F0D0A9606E6071
S113C3F02046F2BD200AFF1F0A490A68138B002B4E
S113C40019BF516BC968D169C96D002818BF0029CB
S113C41005D1002B19BF526BD060D269D065084694
S113C420704700BF200AFF1F38B55218521E120968
S113C4300F311201090902610901A2F16405816148
S113C44045611C4664212846FFF7F0FA0020286065
S113C45004986860074828640598E862606840F0BA
S113C460010068644FF08070A8646FF00200A86255
S113C470012032BDD98E0100C96820F8041C704720
S113C48062F30F2262F31F4200B500BF1300964609
S113C4909446103928BFA0E80C50FAD85FEA417CD2
S113C4A028BF0CC048BF40F8042BC90728BF20F898
S113C4B0022B48BF00F8012B00BD000003490968A6
S113C4C0D1F81423C9690123FFF76ABE200AFF1FAC
S113C4D008480068C1694A6D52B1521E4A6507D1C5
S113C4E0018B00291ABF406B8068408B80F3118850
S113C4F0704700BF200AFF1F38B504460D46FFF7FA
S113C500DDFB2089618929B1884203D3FFF7E0FF6D
S113C510002032BD616809682960401C62681560AA
S113C52062686A604D602081FFF7D2FF012032BD4E
S113C5300149096808817047200AFF1F09490968F1
S113C540D1F81423C9690023FFF72ABE80B5054A30
S113C550126800230093D2F81433D269FFF787FEE0
S113C56002BD0000200AFF1F10B502F08FF804007E
S113C57008BF02F0CBF8204610BD0000034A116842
S113C58010600846704701480068704708ED00E0F5
S113C59002490968C1F88801704700BF200AFF1FDB
S113C5A02DE9F04104461F480768B86B0D469046D4
S113C5B008B9182006E0F86A844224BF386BA04208
S113C5C005D21420FFF718FF0020BDE8F081FFF723
S113C5D075FBF86AB96B201AC00851F8206003E0B3
S113C5E03068A04214D03669002EF9D11420FFF728
S113C5F075FB06462321FFF77BFBF86AB96B0A4FEC
S113C600201AC00851F82020326141F8206000E06F
S113C610776834607560C6F80C80FFF759FF3846B8
S113C620BDE8F081200AFF1F718E010002490968EC
S113C630C1F89001704700BF200AFF1F0249096832
S113C640C1F89801704700BF200AFF1F034A12680F
S113C650C2F89C01C2F8A011704700BF200AFF1F56
S113C6600348016849084900FFE70160002070475A
S113C67000D0004003480068012100F51C70FFF75A
S113C6806FBC00BF200AFF1F2DE9F04F00220126D6
S113C69000234FF0FF3994460FF6F01E00240FF6E6
S113C6A0FC180127DEF800A0D8F800B007FB00F55D
S113C6B00BFB0AFAB5FBFAF54D1B48BF6D424D451D
S113C6C003D2A946624623463E467F1C032FE9D384
S113C6D0641C08F10408102CE3D30CF1010C0EF1D6
S113C6E0040EBCF1040FD9D30FF6F01E140404F4A5
S113C6F0403403F00F052C43751EED076D4245EAE7
S113C70004064FF0FF3989004FF0000C0024DEF8D6
S113C71000504D43A5402D1A48BF6D424D4502D2ED
S113C720A94662462346641C102CF0D30CF1010C7C
S113C7300EF1040EBCF1040FE8D3180300F47040AA
S113C7409105304301F440010843190101F0F0015F
S113C7500843910401F440210843BDE8F08F00B57B
S113C76083B00FF2A5730FF2A11202910FF201210F
S113C77001910FF6090100910FF2090101F0E0FFA8
S113C78003B000BDF8B506460C463068C0B202F0EE
S113C7907DF805004FD04FF4907002F097F8070031
S113C7A001D10420F2BD40F20341FFF7A1FA276052
S113C7B03D60381D31463022FFF7C4F90020F86788
S113C7C0002107F17C00002241608160C1600161A9
S113C7D041618161C161016241624A498162002112
S113C7E0C1627168C1F30541416400218164C1647F
S113C7F0C166016501674165416781658167C165FE
S113C800C1670166C7F8FC10416607F1FC014A6084
S113C81082668A60CA600A614A618A61CA610A6280
S113C8203068FFF7CCF810F1010F07D1206801F050
S113C830A3FE002020604AF20570F2BD286820F4AF
S113C8408040286043F6014028604FF06050E86063
S113C850F1683069FFF718FFE9680843E860706918
S113C86028B102282DD024D303282ED035E0E8683F
S113C87020F08060E860E86820F00070E8602868D4
S113C88040F080702860286840F47F002860B06819
S113C89001282AD128684000400828600020286325
S113C8A06FF00070E86228684008400028600020AB
S113C8B0F2BDE86820F08060E860E86840F000704D
S113C8C0DCE7E86840F08060D4E7E86840F0806026
S113C8D0E860E86840F00070D0E7206801F04CFEA2
S113C8E0002020604AF20170F2BD18B9286840F0B7
S113C8F00040D2E7206801F03FFE002020604AF2A9
S113C9000270F2BDFFFF00802DE9F04104460D00E6
S113C91014BF002C4AF2067028D02868016841F040
S113C92001010160006800281BD5002605F1C80735
S113C9304FF001083B6818000CD0D5F8C400F04053
S113C940C00707D508FA06F03A6A0004012100F48A
S113C9507C109847761C3F1D082EEBD30020C5F8A9
S113C960C400A06901F008FE0020A061BDE8F081C8
S113C9702DE9F04F054683B000242E68C81E00F050
S113C9800D8140F6FE57C01B3BD0401E51D0401EC7
S113C99068D0401E79D0401E00F04682401E00F050
S113C9A04782401E00F0A080401E00F0A780401E79
S113C9B000F0BB80401E00F0C280401E00F0558194
S113C9C0401E4BD0C01E00F0D280401E00F0D98023
S113C9D0401E00F02581401E00F02981401E00F019
S113C9E04981401E00F04E81401E00F05281401EDD
S113C9F000F07281401E00F0D180401E00F01482CD
S113CA0014E2002A00F06981F06869690FF27C651C
S113CA100FF28866C0F3014355F8233000F00F0588
S113CA2056F825506B43C00F23FA00F0B1FBF0F029
S113CA3026E1002A00F05181106810B94AF203740B
S113CA40F6E1306840F001003060F068116800F0F1
S113CA50FE476869FFF718FE384305E1306840F087
S113CA60010005E1002A00F03881F0684001F06817
S113CA7004D5800154BF0220032001E100F00070BE
S113CA80401E8041C043C00FFAE0002A00F0258117
S113CA90306840F001003060106828B102280FD0DF
S113CAA00AD3032814D01CE0F06820F08060F06002
S113CAB0F06820F0007012E0F06820F080600AE076
S113CAC0F06840F08060F060F06820F0007006E0EC
S113CAD0F06840F08060F060F06840F00070F06052
S113CAE0C3E04AF20174C0E0002A00F0F680306826
S113CAF000F00040401E8041C00FC1E0002A00F059
S113CB00EC80306840F0010030601068012803D1E7
S113CB1030684000400803E020B9306840F000402D
S113CB203060A2E04AF202749FE0002A00F0D5804F
S113CB30F068C00154BF01204FF40040A0E0002A77
S113CB4000F0CB80306800280ED51068B0F5004F97
S113CB5003D1F06840F0807004E0012804D1F0684B
S113CB6020F08070F06063E14AF2047460E1002A0E
S113CB7000F0B38005F58470B0E8EA10A2E8EA108A
S113CB8056E1C5F80801C5F80C01C5F81001C5F84F
S113CB901401C5F81801C5F81C0149E1D5F88C0049
S113CBA00028FBD1D5F8A0000028FBD1D5F8A800B7
S113CBB00028FBD1980304D540F61760814240F069
S113CBC037813068002840F13381002705F1C80916
S113CBD04FF00108D9F8003018000DD0D5F8C40082
S113CBE0F840C00708D508FA07F0D9F82020000457
S113CBF0012100F47C1098477F1C09F10409082FD7
S113CC00E8D3C5F8C440306840F0010030603068B3
S113CC10400040083060306840F00040306024E05C
S113CC20002A5AD0F068C0F3C360401C28E0002AF0
S113CC3053D030680028306840F001003060F0685C
S113CC400AD520F0F040F060F0681168491EC9066A
S113CC5001F0F041084307E040014009F060F0684A
S113CC601168491E40EAC160F06030684008400025
S113CC703060DDE08AB3D5F8C000000400F47C1015
S113CC801060D5E04AB31068C0F30540C5F8C00091
S113CC90CEE012B3002705F1C800012606FA07F317
S113CCA0116801EA034111F47C1F03D0516801604B
S113CCB091680162791C136806FA01F503EA0543D9
S113CCC013F47C1F03D053684360936843624F1C82
S113CCD00830082FE2D3ABE012B94AF20774A7E098
S113CCE0D5F8C000000400F47C1040F0004002902D
S113CCF05768106891680191002800F099800090AD
S113CD004FF00108D5F8C000D5F8C410D5F800904C
S113CD1091EA000F2AD0D9F80000002826D5A246AF
S113CD2005F1C80BD5F8C400D5F8C010414021FA6C
S113CD300AF1C9070FD5DBF8003019000BD020FA2F
S113CD400AF000F0010108FA0AF0DBF820200004E0
S113CD5000F47C1098470AF1010A0BF1040BBAF1B4
S113CD60080FDFD3D5F8C000C5F8C4003878D9F867
S113CD700C10C1F3C361082924BF797841EA00206B
S113CD80D9F82C108901FBD502990843C9F834005D
S113CD90D9F82C008003FBD5D9F83800D9F82C1029
S113CDA041F40031C9F82C10D9F82C1009030AD524
S113CDB0D9F82C1041F40021C9F82C10D5F8101121
S113CDC0491CC5F81011D9F82C1009010AD5D9F855
S113CDD02C1041F00061C9F82C10D5F81C11491C25
S113CDE0C5F81C1180B2F168C1F3C361082906D3E8
S113CDF0019A521C0192010A02F8011D7F1C01993B
S113CE00491C01917F1C01F8010DD5F80C01401C4F
S113CE10C5F80C01D5F81401401CC5F8140100989C
S113CE20401E009004D06DE72C2401E040F6092454
S113CE30204627E12DE9F04780460D46D8F80070DA
S113CE409946002A3DD0D8F8C000D8F8C41091EA19
S113CE50000F27D03868002824D5B9F1000F21D05D
S113CE60002408F1C8064FF0010AD8F8C400D8F825
S113CE70C0104140E140C9070CD53368190009D0FE
S113CE80E04000F001010AFA04F0326A000400F400
S113CE907C109847641C361D082CE6D3D8F8C000D3
S113CEA0C8F8C4002878F968C1F3C361082924BF0D
S113CEB0697841EA0020F96A8901FCD540EA090051
S113CEC07863F86A8003FCD5B86BF96A41F40031E1
S113CED0F962F96A090308D5F96A41F40021F96293
S113CEE0D8F81011491CC8F81011F96A090108D5BD
S113CEF0F96A41F00061F962D8F81C11491CC8F8BC
S113CF001C1180B2BDE8F0872DE9F8438769006AF7
S113CF103C6888469146002600F4803529E0206864
S113CF2000F000402843421ED7F8C000924100049C
S113CF3000F47C10D24340F00043D20F41463846FF
S113CF40FFF778FF25B1D7F81411491CC7F814115D
S113CF50D7F80C11491CC7F80C11E168C1F3C3617F
S113CF60082903D3010A08F8011B761C08F8010BF1
S113CF70761C4E45D3D33046BDE8F2832DE9F44FF9
S113CF8082B08569286800900C464FF000094FF084
S113CF90010A72E0D5F8C0002E68010401F47C1186
S113CFA041F00048D5F8C41091EA000F25D030684C
S113CFB0002822D5002705F1C80BD5F8C400D5F800
S113CFC0C0104140F940C9070ED5DBF80030190004
S113CFD00AD0F84000F001010AFA07F0DBF820203B
S113CFE0000400F47C1098477F1C0BF1040B082FFD
S113CFF0E3D3D5F8C000C5F8C4002078F168C1F3C4
S113D000C361082924BF617841EA0020F16A8901DB
S113D010FCD540EA08007063F06A8003FCD5B06B6D
S113D020F06A40F40030F062F06A000308D5F06A58
S113D03040F40020F062D5F81001401CC5F810013E
S113D040F06A000108D5F06A40F00060F062D5F89B
S113D0501C01401CC5F81C010098C068C0F3C360E3
S113D060082824BF641C09F10109D5F81401401CE7
S113D070641CC5F8140109F101090298814589D39A
S113D0804FEA090003B0BDE8F08F00000200000081
S113D090030000000500000007000000020000007B
S113D0A0040000000600000008000000100000005A
S113D0B0200000004000000080000000000100008B
S113D0C0000200000004000000080000001000003E
S113D0D0002000000040000000800000010000006B
S113D0E0030000000500000007000000C169D1F83A
S113D0F0A810890703D4006AC06800B1406870476B
S113D100C169D1F8A820920700D57047F0B5006A2C
S113D110C068002300281CBF4268002A4BD08268E4
S113D1201218127CCE2A41D143686BB14268521E58
S113D13042608268531C12188360127C83680468FE
S113D140A34204BF0023836043686BB14268521E4C
S113D15042608268531C12188360127C83680468DE
S113D160A34204BF00238360446813466CB1426841
S113D170521E42608268541C12188460127C8468B7
S113D1800568AC4204BF0024846013EB02230DD075
S113D1901A1DB2F5807F09D8D1F8A82042F0020206
S113D1A0C1F8A8200222C1F8AC2004E0002310B189
S113D1B043608360C360D1F8A82092076CD51A1D20
S113D1C0D1F894405208DD0748BF521CDDB245F443
S113D1D04A4544F8045B03F47F4544F8045B0025A6
S113D1E0A3B3476877B14668761E46608668771CA5
S113D1F036188760367C8768D0F800C0674504BF5E
S113D20000278760F6B237026D1C9D4219D2D0F810
S113D21004C0BCF1000F13D04668761E46608668D1
S113D22006F1010C3618C0F808C0367CD0F808C0E6
S113D230D0F800E0F44504BF4FF0000CC0F808C07B
S113D24037436D1C44F8047B9D42CAD3C86ADFF897
S113D250785B4401631940F20226DE8004269E6056
S113D260D1F89460665104249C800024DC600C682E
S113D27034341C6100249C829C615404640CDC8260
S113D280DC8308249C8312B1DFF8402B1070D1F8A2
S113D2901401401CC1F81401F0BDF0B40A46002486
S113D2A00025C6694FF0FF31042A04D14FF480747D
S113D2B04FF4007505E0052A04BF4FF480644FF471
S113D2C00065006B0027C30748BF0127830702D509
S113D2D07F1C022F04D200F0010090F001001FE037
S113D2E0D6F8BC00002819BF0020274601202F468D
S113D2F0D6F8A8303B4210D0042A06D106EB8002AF
S113D300D2F8AC20052A0ED107E0052A02BF06EBAD
S113D3108002D2F8AC20052A05D0D6F8BC0000283B
S113D3200CBF27462F46D6F8A8203A4205D0D6F897
S113D330A810B943C6F8A8100146F0BC08467047C7
S113D3402DE9F24F054682B0E869019000F17C07AF
S113D3500026F86A10F0030F40F05081029900246F
S113D3604FF0FF3AB046B146B346042913D12846DC
S113D370FFF793FF824610F1010F00F0C180C7F858
S113D38040A0C7F838A04FF02009F86A40F0010027
S113D390F8620420AAE0052911D12846FFF77DFF91
S113D3A0824610F1010F00F0AB80C7F840A0C7F827
S113D3B038A0F86A40F00100F862052096E00329DD
S113D3C01BD1D7F840A078680198C06F4FF00809C6
S113D3D04FF0010B052808D3B0F1040805D0B0F5CF
S113D3E0807F98BF4FF0100900D9B046F86A40F02A
S113D3F00100F862C7F838A082E0022940F080807A
S113D400284600F066FA02280BD295F8300000F0A6
S113D410010080F0010005EB8001096AC968B1B11F
S113D42012E0E869D0F8B800401E8041C00F05EB57
S113D4308001096AC96851B1496839B980F00100AD
S113D44005EB8001096AC968496801B182464FF059
S113D450010B1AF1010F1FBF05EB8A00006AC468B3
S113D460002C4DD0A0680019007CCE2844D16168FE
S113D47061B16068401E6060A068411C0019A16031
S113D480007CA1682268914208BFA660616861B10E
S113D4906068401E6060A068411C0019A160007CA7
S113D4A0A1682268914208BFA6606268014662B121
S113D4B06068401E6060A068421C0019A260007C85
S113D4C0A26823689A4208BFA66011EB002813D013
S113D4D008F10400B0F5807F0ED8C7F83CA0C7F867
S113D4E038A0F86A40F00200F8620220019901EBCA
S113D4F08A01C1F8AC0003E0B046204600F082F88F
S113D500F86A10F0030F79D0012000FA0AF108F14B
S113D5100402B86953085FEAC87248BF5B1C029AE8
S113D520022A0CBF42460022090401F47C1141EA9C
S113D5300B71D6B20E4346F0004646F44A4640F814
S113D540046B02F47F4249EA020646EA0102B8F19A
S113D550000F18BF42F0004240F8042B4FF0000ABD
S113D5604FF6FF723BD003E045F0004540F8045B02
S113D5706CB3029E022E2AD166686EB165686D1E78
S113D5806560A5686E1C2D19A6602D7CA6682768A9
S113D590BE4204BF0026A660EDB22E020AF1010AC3
S113D5A0C24511D2676877B165686D1E6560A5686C
S113D5B06F1C2D19A7602D7CA768D4F800C067459F
S113D5C004BF0027A7602E430AF1010A02E01646B1
S113D5D00AF1020A46EA0105C245C5D305600320E3
S113D5E0009004220198042100F07DF90198D0F8FC
S113D5F014010199401CC1F814010126304603B0FE
S113D600BDE8F08F18B1002141608160C1607047AE
S113D6102DE9F84304464FF00408D4F81C90D9F8D7
S113D6208000002568B94FF40070FEF757FBC9F875
S113D630800030B1D9F8800040F20141FEF758FB78
S113D640012509F18007786960B94FF40070FEF78D
S113D65045FB786130B1786940F20241FEF748FB3E
S113D66045F00205D9F8800000281CBF786900281D
S113D67045D0606B04EB8000006A00283FD1102085
S113D68001F024F9616B04EB81010862606B04EB27
S113D6908000066A9EB340F2FF313046FEF728FB55
S113D6A0A0698069306045F004051030FEF716FB70
S113D6B0B060A069C06970601030FEF70FFBF060C5
S113D6C0B06800281CBFF168002918D040F201415D
S113D6D0FEF70EFBF06840F20241FEF709FBB0686A
S113D6E031680160002141608160C160F068716847
S113D6F00160002141608160C160884638E0E8072C
S113D70006D5D9F8800000F037FF0020C9F8800062
S113D710A80704D5786900F02FFF00207861680716
S113D72026D5606B04EB8000006A806838B100F095
S113D73023FF606B04EB80000021006A8160606B52
S113D74004EB8000006AC06838B100F015FF606B1C
S113D75004EB80000021006AC160606B04EB800070
S113D760006A00F009FF606B04EB80000021016295
S113D7704046BDE8F28338B5C169D1F8802013680A
S113D7801D0A4FF0FF34CA2D15D1526802F47F44AC
S113D790DBB21C43CB6873B1D2B2130608D4930630
S113D7A002D5FFF7ADFC06E0D00601D4100702D580
S113D7B00020C1F8A800204632BDF0B4C469E26F6D
S113D7C0D4F8BC5000EB85000023006A8068002870
S113D7D078D044680568AC4202D2036844681B1BD5
S113D7E0002A74D0141D9C4271D2C3684468056831
S113D7F0AC420ED2C468651CC5602418002525748B
S113D800C4680568AC4204BF0024C4604468641C56
S113D810446044680568AC420DD2C468651C241891
S113D820C5602274C4680568AC4204BF0024C460A7
S113D8304468641C446044680568AC420ED2C46801
S113D840651CC5602418150A2574C4680568AC42B3
S113D85004BF0024C4604468641C446000240D6850
S113D860466807682D0ABE420DD2C668771C361872
S113D870C7603574C5680668B54204BF0025C56035
S113D88045686D1C4560641C94423FBF0D68466842
S113D8900768BE420DD2C668771C3618C760357457
S113D8A0C5680668B54204BF0025C56045686D1C9F
S113D8B04560641C091D9442D1D31818CE2101740B
S113D8C0F0BC7047D4F81001401CC4F81001F0BC3F
S113D8D07047006B0021C20748BF0121800748BF81
S113D8E0491C08467047F0B5059DEC072FD5466ADC
S113D8F0DFF8D4444FEA461C0CEB040740F2022E36
S113D900A7F806E04FF0040EC7F808E0D0F800E0EE
S113D9100EF1380E4CF804E00024BC80FC600029B1
S113D92014BFD0F8804000F190043C61B9825C04DB
S113D9300021B961640CFC82FC83C16800290CBF1E
S113D9400A210821B98313B1DFF880140E70A907E6
S113D9501ED540F20227C16ADFF86C444E01351926
S113D960EF800427AF60D0F894703751AA805C042C
S113D9700022EA60640C006834302861AA82AA613B
S113D980EC82EC830820A88313B1DFF84004017013
S113D990F0BD2DE9F8430446A669206B4FF000085A
S113D9A040B90A4604F11C013046FEF7EBFE00289C
S113D9B040F08480E5692F68206B90B9306800A935
S113D9C000F06DFF5FEA000807D1E06900F0D4FDC4
S113D9D00020E0611420BDE8F283F86840F0F040D4
S113D9E0F8602046FFF714FE10B10420BDE8F2836E
S113D9F0206B00283AD1F868DFF87419084040F425
S113DA00802040F0B0003861E86820BB0027B8F1FE
S113DA10010F15DB05F134060FF28579009850F8F3
S113DA20270000F05DFFB0612246009850F82700FF
S113DA304946FEF7B5FD7F1C46F8040B4745EDDB70
S113DA40686A0FF688130FF2997153F82000224682
S113DA50FEF7A6FD0AE0002000F042FFA867224678
S113DA600FF659110020FEF79BFD6867E86820BB9C
S113DA70D4F834800FF694110FF6A01051F8281042
S113DA8050F8280051F8202022F4702242F4302269
S113DA9041F8202005EB88050FF6881050F828700F
S113DAA0384600F01DFFE86622460FF6801050F855
S113DAB028103846FEF774FD68660020BDE8F2833E
S113DAC02DE9F04182B004460D0014BF002C4AF247
S113DAD0067000F08380A06A00283CD1206B0028E7
S113DAE039D028680168016841F001010160002211
S113DAF000210163686ADFF87C184254E86A4254E2
S113DB00E868F8B9686A0FF6C40313F82000042122
S113DB1000F012FF686800A900F0C1FE06464FF04D
S113DB200008012E17DB05F13407BA6957F8041B06
S113DB30009850F82800FEF733FD08F10108B045BD
S113DB40F3DB08E00421002000F0F6FEAA6F696F01
S113DB500020FEF725FD666B002E0CBF012002207D
S113DB60216B21EA00002063E86878B90FF6B4005D
S113DB7050F8267000220421384600F0DDFE05EB43
S113DB808600C26E416E3846FEF70AFDE06900F079
S113DB90F3FC0020E061D5F8800000F0EDFC0020EB
S113DBA0C5F88000D5F8940000F0E6FC0020C5F824
S113DBB0940004EB8604206A806800F0DDFC216A8E
S113DBC000208860206AC06800F0D6FC216A00202A
S113DBD0C860206A00F0D0FC00202062BDE8F68115
S113DBE0F8B506000C4618BF002C02D14AF20770A3
S113DBF0F2BD306B744D00285DD12068DFF87827C2
S113DC00016841F0010101600427016B11430163C4
S113DC1000220168490849000160DFF860070168D3
S113DC2041F002010160606ADFF854170870636A0A
S113DC30DFF840071A54E26A0A700021E26A1154BC
S113DC40616A4B015A1940F20221D180976027681A
S113DC5038375F5100239380D36004F1900313613C
S113DC60002393829361D382D383E368002B0CBF98
S113DC700A2308239383E26A53015A19D1800421A9
S113DC809160D4F89410595100219180D160216899
S113DC9034311161002191829161D182D1830821B3
S113DCA09183616AA26A42F080020A54E16A226B9B
S113DCB042F080020A54FEF701F8706B00280CBF92
S113DCC001200220316B08433063FEF701FCE06859
S113DCD0002850D1606800A900F0E1FD0546002746
S113DCE0012D09DB009810F827000122042100F01F
S113DCF023FE7F1CAF42F5DB606A0FF2D06313F89A
S113DD0020000122042100F017FE706B0FF214733F
S113DD1053F820000122042100F00EFEFDF7CEFF8F
S113DD20716B0FF2F0600FF2F46350F82100026996
S113DD3053F82130F069DA40D20719D4002907BF1B
S113DD404FF480714FF480624FF400714FF400621D
S113DD50D0F8A8300A4323EA0202C0F8A820D0F879
S113DD60A8201143C0F8A81030460421FFF7E8FAB0
S113DD70FEF7AEFB25E001220421002000F0DCFDCB
S113DD80606A4201511940F20223CB8004238B6064
S113DD9023683833535100228A80CA60D4F8802023
S113DDA00A6104228A8200228A614022CA82CA83CA
S113DDB0E268002A0CBF0A2208228A83DFF8C01511
S113DDC048700020F2BD0000009000401B8000401D
S113DDD0F8B50E46416B00EB81001446006A856875
S113DDE00027002C1EBF002D686800286FD0A8688B
S113DDF04019007CCE2863D1FDF760FF686868B1E4
S113DE006868401E6860A868411C4019A960077CC6
S113DE10A8682968884204BF0020A860686868B1BF
S113DE206868401E6860A868411C4019A960077CA6
S113DE30A8682968884204BF0020A8606968384639
S113DE4069B16968491E6960A9684A1C4919AA60D0
S113DE500F7CA9682A68914204BF0021A96000EBE5
S113DE600727BC4216D387B33846696871B169681D
S113DE70491E6960A9684A1C4919AA60097C317065
S113DE80A9682A68914204BF0021A960761C401E3B
S113DE90EBD11AE08FB1686868B16868401E6860A9
S113DEA0A868411C4019A960007CA86829688842B8
S113DEB004BF0020A8607F1EEDD14FF0FF3704E0BF
S113DEC0FDF7FCFE2846FFF79DFBFEF701FB3846F5
S113DED0F2BD2DE9F04104460D46616B04EB81016E
S113DEE00020096ACF6816464FF0FF38002F74D01F
S113DEF079683A68914202D238687968401A002EEB
S113DF006BD0311D814268D2D7F80C80FDF7D6FE64
S113DF107868396888420ED2F868411CF960C019E3
S113DF2000210174F8683968884204BF0020F86051
S113DF307868401C78607868396888420DD2F8683F
S113DF40411CC019F9600674F8683968884204BF36
S113DF500020F8607868401C7860786839688842E6
S113DF600ED2F868411CF960C01931120174F868C6
S113DF703968884204BF0020F8607868401C7860E3
S113DF80304629787A683B689A420DD2FA68531C65
S113DF90D219FB601174F9683A68914204BF0021F8
S113DFA0F9607968491C79606D1C401EE9D108EB61
S113DFB00701CE200874FEF78BFAB046FDF77EFE0B
S113DFC0E069C06820B902212046FFF7B9F902E0F0
S113DFD02046FFF78BF8FEF77BFA4046BDE8F08158
S113DFE0F8B505460F46E869FEF7C2FC40F609217C
S113DFF00446884240F0C180E869066800244FF472
S113E00062603F1A06D07F1E00F0A0807F1E00F0E1
S113E010A580B1E0FDF752FE3068D749D94A40F0F7
S113E0200100306040F20223306840F44060306008
S113E0304FF0040E306B08433063306840084000F2
S113E0403060CF4804700470E9694E6A4FEA461C98
S113E0500CEB0207FB80C7F808E0D1F800E00EF1F2
S113E060380E4CF802E0BC80FC60D1F880C0C7F8E0
S113E07010C04FF0040CA7F814C0BC614FF0400C62
S113E080A7F816C0A7F81EC0D1F80CC0BCF1000F49
S113E0900CBF4FF00A0C4FF0080CA7F81CC04670D8
S113E0A0CE6A4FEA461C0CEB0207FB800423BB60DC
S113E0B0D1F894304CF802300422BA80FC6009682C
S113E0C034313961BC82BC614021F982F983082171
S113E0D0B9834670E8690068016841F00101016094
S113E0E0016841F440610160016849084900016028
S113E0F00120E969C1F8B440E969C1F8BC40E969A3
S113E100C1F8B840E969C1F8AC00E969C1F8B000E8
S113E110E969C1F8A840286A38B18068FFF772FA43
S113E120286A10B1C068FFF76DFA686A58B1806850
S113E130FFF768FA686A00281CBFC068002802D08C
S113E14044608460C460E869C06812E0FDF7B6FD0D
S113E150686B05EB8000006A806806E0FDF7AEFDA1
S113E160686B05EB8000006AC06810B1446084608D
S113E170C460FEF7ADF900E00C462046F2BD00B5E0
S113E18085B0814B814A0391814902918149019172
S113E19081490091814900F007FC05B000BD0000F1
S113E1A0C0690168CA6AD0F808315B1CC0F808313C
S113E1B0130108D5CB6A43F00063CB62D0F81C315D
S113E1C05B1CC0F81C31120308D5CA6A42F4002251
S113E1D0CA62D0F81011491CC0F810117047000031
S113E1E02DE9F04180466E49D8F81C50686A0870E1
S113E1F005F1A807D5F8A80080088000C5F8A80094
S113E2000126386E401C3866F86805EB8000D0F8AB
S113E210AC00042808BF05262ED0F86805EB800062
S113E220D0F8AC00052810D105F124044046FFF7CE
S113E230A2FAA065A06D10F1010F02D10020A06523
S113E24001E0A06DC0B1032616E0F86805EB80007C
S113E250D0F8AC00032808D105F12400C16D404674
S113E260FFF7ABFA786E401C7866D5F8A80010F476
S113E270407F14BF04260226F86805EB8000C0F82E
S113E280AC60F86805EB8000D0F8AC104046FFF7AE
S113E29057F850B9052E0BD0D5F8A80010F4406FEC
S113E2A004D005214046FFF74BF860B9042E0AD08C
S113E2B0D5F8A80010F4407F05D04046BDE8F041F1
S113E2C00421FFF73DB8BDE8F08118B4354A116860
S113E2D0C90721D5C169344B1B68146844F0010493
S113E2E0146001F1A802146E641C1466DA07D1F8F4
S113E2F0A8200BD422F4A062C1F8A820D1F8A82049
S113E30042F48072C1F8A820042104E042F480623F
S113E310C1F8A82005214DE011BC704718B4234A68
S113E3201168C90721D5C169214B1B68146844F0E1
S113E3300104146001F1A802146E641C1466DA0767
S113E340D1F8A8200BD422F42062C1F8A820D1F877
S113E350A82042F40072C1F8A820042104E042F489
S113E3600062C1F8A820052124E011BC7047000018
S113E3700FFFF3FF0010024000000B0B3C80044031
S113E3801A80004000900040C1DA0000E1DB000088
S113E390E1DF0000D3DE0000D1DD000093D90000EE
S113E3A01F800040A0C00440D0F00F40A0D0044023
S113E3B010F10F4014BCFEF7C3BF0000C069D0F8D1
S113E3C00811491CC0F80811704700001000000033
S113E3D011000000120000001300000014000000EF
S113E3E015000000160000001700000018000000CF
S113E3F0190000001A0000001B0000001C000000AF
S113E4001D0000001E0000001F00000000C00440AA
S113E41000D00440C0F00F4000F10F4000000000A5
S113E420000000006A0000006B000000CBE2000066
S113E4301DE3000010B50A480468D4F8C40168B1AB
S113E440D4F8C81100F01CFCC4F8980204F5267036
S113E450D4F898124160D4F89812816010BD00BFBE
S113E460200AFF1F2DE9F84342480568D5E9590100
S113E470401C41F10001C5E95901FDF71FFCD5F825
S113E4809C11080004D0D5F8A0018847C5F86C0198
S113E49005F5B27000F03AFCB5F88461AEB3D5F876
S113E4A07C01761C1BE0B5F88421521EA5F884215A
S113E4B0426811604A60816821F4807181604A0574
S113E4C00AD521F480618160016CC26B0A605160DD
S113E4D0816B0A89521E0A81FDF7D4FC2046761E00
S113E4E013D0D0E91123D5E9598901680C464B456D
S113E4F0D9D301D84245D6D3D5E95923D0E91189D6
S113E5004B45D0D828BF4245CDD2E869816A4A0735
S113E51020D5D0E92B23521C43F10003C0E92B235F
S113E520C90417D4D0E92823D0E92B67BB420BD305
S113E53001D8B24208D3D0E92B23D0E92867BB42E3
S113E54008D301D8B24205D3416802680A60516019
S113E550FDF798FCFDF7BCFFD5F80403010018BFD4
S113E5608047D5F83C0301001CBFBDE8F2430047D7
S113E570BDE8F183200AFF1F38B53349096820B983
S113E5800120FDF739FF012032BD304AA0F10C040F
S113E5906568A868904204D03820FDF72DFF382024
S113E5A032BDC9692089C96889B288421CBF4FF647
S113E5B0FF71884204D00320FDF71EFF032032BD03
S113E5C0FDF77CFB686905E0E961FDF781FFFDF774
S113E5D075FBE869696909B18C420BD20846216868
S113E5E00A19824203D10268511821608068A06030
S113E5F06C611CE081688C4201D30029E4D10A4695
S113E60021680B19934206D1126851182160816860
S113E6108968A16000E0A26001680A18A24205D1DD
S113E620226851180160A168816000E08460686913
S113E630A8616869E8612862E8686862E868A862B5
S113E640FDF746FF002032BD200AFF1F70656D6C88
S113E65070B504460D00164608BF2546FDF72EFB8F
S113E660608930B12189814203D3FDF731FF002055
S113E67070BD286830602E60756046602089401C3B
S113E6802081FDF725FF012070BD00002DE9F8432E
S113E69004460D46A54238BF0C202ED31848066800
S113E6A01848C6F808011848B062281B401CC00866
S113E6B000F101084746B80000F008F95FEA0009D4
S113E6C008BF042019D00321FDF712FB06F128002E
S113E6D0C0F8109044608560A6F840730320A6F843
S113E6E04203B8F1000F07D009EB8700001F002197
S113E6F040F804197F1EFBD10020BDE8F28300BF5F
S113E700200AFF1F67A90100718E010009480068F3
S113E710C06B80F308880848084A3C2140F8042B61
S113E72040F8042B40F8042B40F8042B491EF5D183
S113E730704700BF200AFF1F4000FF1F67A90100A8
S113E7402DE9F041804684B00D4616461F4624202C
S113E75000F0BCF8040008BF04201FD04FF480610F
S113E760FDF7C6FA25606660A7600A980FF2C50334
S113E7700FF295020FF25501E0600B9820610C989E
S113E780606103940FF21D0002900FF2B900019032
S113E7900FF2A9000090404600F0D0FA04B0BDE8A2
S113E7A0F081000010B50446606AC16959B9426835
S113E7B0110002D0816940699047606AFFF7DCFE6E
S113E7C00020606210BD40F60A2010BDF8B5044672
S113E7D00D462068476A1646FDF770FAF86918B1C5
S113E7E0FDF776FE2C20F2BD0120F861FDF770FEE6
S113E7F03E62A66078693B682A4607F1180198478B
S113E80008B10021F961F2BD38B50068456A0024F9
S113E810FDF754FAE869401EE86106D16A68100001
S113E82003D0A969284690470446FDF751FE2046C7
S113E83032BD00000068406A836818470068406A77
S113E840C368184770B5034600201C68646AB1F1B8
S113E85009050ED040F60466AD1B02D06D1E03D030
S113E8600DE0216A116070BD116821621168996020
S113E87070BD1021116050604C21916070BD2569FC
S113E8802B0002D0236AA069A84770BD032804D2D4
S113E8900FF2200151F82000704700207047032830
S113E8A006D20FF21C0202EB8000086001207047C0
S113E8B00020704700C0024000D0024000C00A405F
S113E8C02A0000002B0000002C0000000349096806
S113E8D0D1F8142301235031FDF762BC200AFF1F35
S113E8E038B5044613480568A86B18B91820FDF715
S113E8F083FD1DE0E86A844224BF286BA04203D252
S113E9001420FDF779FD13E0FDF7D8F9E86AA96B47
S113E910201AC00851F8205000E02D69002D1CBFBA
S113E9202868A042F9D1FDF7D3FD0DB1E86832BDE6
S113E930002032BD200AFF1FF0B4A0F11003FB2811
S113E9402AD217489C0800EB840403F00305ED0069
S113E950D4F80063FF274901AF4001F0E001BE4352
S113E960A9403143C4F800134AB1FB2B11D2012151
S113E97003F01F0291405A0940F8221009E0FB2BD2
S113E98007D2012003F01F018840064A590942F8C2
S113E99021000020F0BC7047F0BC0C207047000040
S113E9A000E100E080E100E02DE9F041804684B020
S113E9B00E4617461C464FF4AC70FFF787FF050060
S113E9C008BF042021D040F2FF31FDF791F92E60F9
S113E9D06C60AF600A980FF285130FF221120FF2E8
S113E9E05901E8600B9828610C9868610D98A8613A
S113E9F003950FF21D0002900FF2F91001900FF22F
S113EA00A5100090404600F099F904B0BDE8F081EB
S113EA1038B50446656AA86A58B96A68100002D015
S113EA20E969A86990472846FFF7A6FD00206062BF
S113EA3032BD40F60A2032BDF8B5054617462868AF
S113EA40446A0E46002000220B783A2B1CBF11F8B2
S113EA50013F3A2B04D0491C921C0A2AF4DB0EE035
S113EA6011F8012F42F02002632A02BF4A7842F0D3
S113EA702002732A03D18978312908BF0120286133
S113EA806063FDF71BF9A06A022803D3FDF720FD9C
S113EA902C20F2BD401CA062FDF71AFDE762AF60B6
S113EAA03146226820469047050004D1E169A268F6
S113EAB02046904705461DB1A06A401EA0621AE098
S113EAC00021606B00EB400204EB0210383000F0D0
S113EAD0B9F9606B00EB400204EB0210002198309E
S113EAE000F0B0F9606B00EB400204EB021000216F
S113EAF0F83000F0A7F92846F2BD000038B50168E7
S113EB004D6A006968630024FDF7D8F8A86A40B12B
S113EB10401EA8626A68100003D0E969284690473D
S113EB200446686B00EB400105EB0110383000F03F
S113EB30D7F9686B00EB400105EB0110983000F049
S113EB40CFF9686B00EB400105EB0110F83000F0E1
S113EB50C7F9FDF7BDFC204632BD00002DE9F041A8
S113EB600C4601684F6A0069786300EB40014FF07E
S113EB70FF3607EB01101546B046383000F0FAF9BD
S113EB8078B9FB682A462146384698478046786B10
S113EB9000EB400107EB0110383000F071FA00B1CE
S113EBA0B04623E02DE9F0410C4601684F6A006944
S113EBB0786300EB40014FF0FF3607EB0110154678
S113EBC0B046983000F0D6F978B93B692A46214618
S113EBD0384698478046786B00EB400107EB0110FC
S113EBE0983000F04DFA00B1B04600BF4046BDE891
S113EBF0F08100002DE9F843044688462068466AFF
S113EC002069706300EB40014FF0FF3906EB0110FF
S113EC1015464F46F83000F0ADF968BB0027B8F14F
S113EC2009000ED040F60461401A02D0401E03D001
S113EC300DE0F06A286015E02868F0622868A0609A
S113EC4010E0102028606F604A20A8600AE0D6F81F
S113EC5014C0BCF1000F05D0F36A2A464146304681
S113EC60E0470746706B00EB400106EB0110F830FB
S113EC7000F006FA00B14F463846BDE8F2830000C2
S113EC802DE9F04104462048056805F51C768846C0
S113EC90304600F043FAD5F88C7205F5237500E090
S113ECA03F68AF420ED0B868214600E0401C0A78A5
S113ECB02AB102781AB111F8013B9342F6D00078D8
S113ECC00028EDD1304600F05FFAAF4215D0202085
S113ECD0FFF7FCFD060010D01021FDF709F837609E
S113ECE0FB6818000CD0424621463046984738B19C
S113ECF0FDF782FB3046FFF73FFC0020BDE8F081C2
S113ED003046BDE8F08100BF200AFF1FD0B40A4995
S113ED1009688468D1F898118C420BD3D0E9006754
S113ED20B4FBF1F20023B6185F41C0E9006701FBB0
S113ED3012418160D0BC7047200AFF1F2DE9F047C3
S113ED400D463F49D1F800800446002016469A46F5
S113ED50290027D0310025D00021224613783A2BF0
S113ED6008BF401C00D0CBB15378491C3A2B08BFD4
S113ED70401C00D093B19378491C3A2B08BF401C27
S113ED8000D05BB1D378491C3A2B08BF401C00D09B
S113ED9023B1491C121DB1F5806FDFD3012801D1C5
S113EDA0012902D10C20BDE8F08708F51C794846FA
S113EDB000F0B4F9D8F88C0220B9002108F52370CA
S113EDC0FDF7B6F9D8F88C7208F5237800E03F68AF
S113EDD047450ED0B9684FF48062204600F00CFA23
S113EDE00028F4D1484600F0CFF94FF42060BDE884
S113EDF0F087484600F0C8F92C20FFF767FD0700AC
S113EE0008BF04201AD00F21FCF772FFBC60FD601C
S113EE103E61C7F814A00898B8610998F8610A9887
S113EE2038620B987862484600F078F939464046D3
S113EE30FDF762FB484600F0A7F90020BDE8F08723
S113EE40200AFF1F2DE9F04104461048D0F8008045
S113EE5086B00D0003D100AD00A800F0E3F904B3BF
S113EE6068680B4EB0421CD1D8F8FC7127B900F089
S113EE70EBF9D8F8FC7187B3F868B04218BF1A20D0
S113EE802BD1FCF71BFF386805E000BF200AFF1FE9
S113EE907874756D0068B84206D0A042FAD1FDF7C7
S113EEA017FB4FF4826018E0286829690843A060C2
S113EEB0E6600021E8686061A86820610020A0760F
S113EEC0E062A06204F11C00FDF732F921463846E5
S113EED0FDF712FBFDF7FCFA002006B0BDE8F08157
S113EEE070B5044622480568D5F8FC610EB91820AF
S113EEF070BDF0681D49884201D01A2070BDA06A17
S113EF00E969884203D0204600F034F868BB002049
S113EF10E0602068C8B1FCF7D1FE60682168016038
S113EF2048603089401E30810DE004F11C0000F07F
S113EF30BBF906464FF4826100F0CBF9FCF7BEFE44
S113EF403046FCF79FFFFDF7C3FAA08C0028ECD1F4
S113EF50ED69FCF7B3FEE16A11B1284600F0C9F986
S113EF60FDF7B6FA0BF080FC002070BD7874756D67
S113EF70200AFF1FF8B504463F480068C569008BA6
S113EF8008B10D20F2BD002C3DD0E0683B4EB042EC
S113EF9039D1A06AA84202D140F20940F2BDE86921
S113EFA0C789FCF78BFEA07E80B3A068C0050ED590
S113EFB0A06A016AC9898F4209D2C169C9898F428D
S113EFC03CBF394600F08CF9E06A401CE062686896
S113EFD0296801604860294604F11C00A863207A6E
S113EFE0000704F11C0002D500F09BF901E0FDF7D5
S113EFF083FA40F22320A8600BF044FCE068B0429E
S113F00007D0FDF765FA4FF48260F2BD8020A07648
S113F010A562A06800F48470B0F5807F12D104F179
S113F0201C0000F093F90146286AC089814209D284
S113F030E869C08981423CBF284600F051F9E06A82
S113F040401CE062FDF744FAA068800512D5FCF785
S113F05035FE286A2169C089814209D2E869C089DC
S113F06081423CBF284600F03BF9E06A401CE06264
S113F070FDF72EFA0020F2BD200AFF1F7874756D8B
S113F080F8B5040023480568E86908D0E168224A15
S113F090914201BFA17E8029A16A814202D04FF42E
S113F0A08260F2BDFCF70AFEE66A0020E062207A84
S113F0B010F0030F03D00020A062A07620E0A08C03
S113F0C0E0B104F11C0000F0EFF80746A762FCF77A
S113F0D0D9FEA06880050ED5386A2169C0898142AD
S113F0E009D2F869C08981423CBF384600F0F8F87B
S113F0F0E06A401CE0620BF0B7FB01E0A076A0627E
S113F1001EB13146E86900F0F4F8FDF7E1F900209A
S113F110F2BD00BF200AFF1F7874756D70B50446F8
S113F12017480668308B08B10D2070BD6069154D15
S113F130A8421FD1FCF7C2FDA069012813DAF069C7
S113F14040F22B41816004F1080181634168026847
S113F1500A60516000F13C0104F10800FDF7CCF9AC
S113F1600BF090FB01E0401EA0616069A84203D04F
S113F170FDF7AEF91F2070BDFDF7AAF9002070BDA0
S113F180200AFF1F6D73776C38B505461848194976
S113F19004686869884201D01F2032BDFCF78EFDE7
S113F1A0A86900281ED4298AE1B105F1080000F0FD
S113F1B07BF83C388168CA050DD542680368136042
S113F1C05A6021F48071B4F88421521EA4F8842179
S113F1D041F00301816000218163FCF753FE0BF0D1
S113F1E043FB01E0401CA861FDF772F9002032BD29
S113F1F0200AFF1F6D73776C01E0491C521E72B127
S113F2000B7890F800C09C4505D002D24FF0FF3037
S113F21070470120704710F8013B002BEDD100200E
S113F2207047000010B94FF48260704700210160FC
S113F2308160044941600021C16004210161002012
S113F240704700BF7874756D38B514480468D4F8F5
S113F250FC0108BB1020FFF739FB050001D1042095
S113F26032BD1821FCF744FD00212846FCF760FF5D
S113F2700B48E860FCF722FDD4F8FC0128B1FDF747
S113F28027F92846FFF778F906E0C4F8FC51054849
S113F290C4F83C02FDF71CF9002032BD200AFF1F10
S113F2A07874756DA98D010038B50446FCF706FD28
S113F2B0208918B9FDF70CF9002032BD256869686A
S113F2C02A680A605160401E2081FDF701F9284632
S113F2D032BDC26D002914BF002AC16510467047B3
S113F2E080B5826A42F400428262026D521C026559
S113F2F011E0826A130400D4704780B5036D99420B
S113F30002D2591A016501BD0021016522F40041B0
S113F3108162016AC98900F029F8BDE801400BF057
S113F320A3BA78B4CD6904890268ED890346641CE4
S113F33001E013461268641E03D0D669F689B5420B
S113F340F7D20A46194678BCFFF782B901680089EA
S113F350421C4FF0FF3005E0CB69DB89834238BFA4
S113F36018460968521EF7D170470000F8B50446E4
S113F37014480668E069C7890D462801316A40428D
S113F38040188189A184E061A068022811D16068D5
S113F3902168016048602046FCF774FDF069A042D2
S113F3A007D1A08C7083AF420AD2BDE8F1400BF0C4
S113F3B069BA606D20B92046BDE8F24000F004B897
S113F3C0F1BD00BF200AFF1F7047000010B4FF23E7
S113F3D0002818BF002A18D00C2916DB0021974BEF
S113F3E0CC5C00F8014B491CCC5C00F8014B491C77
S113F3F0CC5C00F8014B491CCC5C00F8014B491C67
S113F4000C29EDDB0C201060002310BC184670475B
S113F4102DE9F8430600894615464FF0FF0818BF4A
S113F420002D35D0089C9CB3B9F1010FA8BF022B65
S113F4302EDB3778032F2BDA00F0BCF91FB1022F33
S113F4401BD00BD324E000F0BEF9002129706870B2
S113F4508846000AA8700320206019E0B9F1030F60
S113F46007DBB078717841EA002000F0AFF94FF083
S113F47000080120287020600AE000F0C1F9022190
S113F480297068704FF00008000AA87003202060FB
S113F4904046BDE8F28370B504461546FF22FF20BE
S113F4A0002C18BF002D17D0049EAEB10129A8BFAF
S113F4B0022B11DB2478022C0EDA14B1012C03D0B8
S113F4C005E000F0AFF901E000F0CBF902462C7042
S113F4D06A7002203060002070BD0246FF2002B92D
S113F4E0704710B5032964DB51789078090241EA2A
S113F4F00040117841EA00040020FCF72DF804F0E4
S113F5000101491E89414F48C943C90F416104F0B3
S113F5100201491E8941C943C90FC16104F00401B4
S113F520491E8941C943C90F816104F00801491E7C
S113F5308941C943C90F016104F01001491E894181
S113F540C943C90FC16004F02001491E8941C94360
S113F550C90F816004F04001491E8941C943C90FA4
S113F560416004F08001491E8941C943C90F01600B
S113F57004F48030401E8041C0433349C00F08600A
S113F58004F40030401E8041C0433049C00F08607D
S113F59004F48020401E8041C0432D49C00F086000
S113F5A004F40020401E8041C0432A49C00F086073
S113F5B0002010BD70B50446FF201546002C18BF6E
S113F5C0002D18D0012916DBFCF7C8F800F00F064F
S113F5D0FCF7CBF800B110200643FCF7CAF800B1E1
S113F5E020200643FCF7CDF800B1402030432070C2
S113F5F001202860002070BDF8B50446FF2016469F
S113F600002C18BF002E18D0069DB5B10129A8BF43
S113F610032B12DB24782746482F0DDA322000F022
S113F6205DF9074830F81700347006F8010F000A36
S113F63006F8010F032028600020F2BD20A400007A
S113F6407C1BFF1F2010FE435C08FE431000FE439A
S113F6501C18FE431820FE432DE9F04104004FF02E
S113F660FF081646404618BF002E18D0069FB7B1B3
S113F6700329A8BF022B12DB2578A178627842EA1D
S113F6800122082D0BDA25B90021002000F01EFA12
S113F6908046357086F80180022038600020BDE87D
S113F6A0F0810246FF2002B9704780B5022910DBC1
S113F6B0117802290DDA527800200021012A02D1A2
S113F6C00120012102E0022A08BF012100F087FA8B
S113F6D0002002BDF8B50446FF26BCB1012915DBA4
S113F6E020784D1E012813D10B2D0FDA012700219C
S113F6F0002000F0F7FCEAB2611C384600F048FD37
S113F70000B900260621002000F0ECFC3046F2BDD2
S113F7100228FBD1152DF9DA0227E8E72DE9F0419B
S113F720FF2590B014469846002818BF002C34D00A
S113F730169E96B30129A8BFB8F1020F2DDB0778F6
S113F740022F08BF0FF25C0006D0012F02D0002068
S113F75030601EE00FF2540000213160C8B1012373
S113F760402200A900F055FD98B99DF8000080B131
S113F770A8F102009DF80010C0B2884209D30A46DD
S113F7800DF10101601CFCF7CDF99DF8000030601B
S113F790002527703068401C3060284610B0BDE852
S113F7A0F08100005B7365723D0000005B70636272
S113F7B03D00000010B5194C206818B90C20FCF766
S113F7C07DFE206010BD164801F047B838B51349D6
S113F7D0096851B10A8843F612239A4205D138C9FF
S113F7E00F4A38C2002221F80C2D0D4C61884018B4
S113F7F0608000F0F3FE2046BDE8324000F0B6BF62
S113F80010B5064C2168002039B1084601F06EF8A5
S113F810206800F0ABFF2068808810BD2C1EFF1FFD
S113F820901DFF1F70B582B001244FF400550020D5
S113F83000F084FA2946002000F02AFC4FF4806688
S113F840042300AA2946002000F01FFB009810F1B1
S113F850010F01D0FF2402E02D1D761EF0D12046B9
S113F86076BDF8B501244FF40055002000F066FA87
S113F8700021002000F0FBFA2946002000F02EFBB6
S113F8800026F1B2002000F032FB761CB6F5805F52
S113F890F7D3002600AF042300AA2946002000F075
S113F8A0F4FA9DF80000F1B2884201BF7878711C27
S113F8B0C9B2884209D1B878B11CC9B2884201BF23
S113F8C0F878F11CC9B2884201D0FF2404E0361D47
S113F8D02D1DB6F5805FDED32046F2BD38B50D4947
S113F8E00C68A8B1E56905F1440101F0A3F9FCF73E
S113F8F0E5F905F1440204F5B27105F1440001F0A3
S113F900CDF9284601F0ECF9BDE83140FCF7E0BD43
S113F91031BD00BF200AFF1F18B412F1010F04BF4C
S113F92014BC01F013BA00210246002301F00F04B5
S113F9301470491C137401F00F045470491C03F132
S113F940100454742033921C1029EFDB012180F839
S113F95020100022022180F82110042180F82210B6
S113F960082180F82310102180F82410202180F829
S113F9702510402180F82610802180F82710FF21CF
S113F98080F8281080F82920552280F82A20AA22FD
S113F99080F82B20002280F82C2080F82D1011BC38
S113F9A07047F0B587B006460D46012404A801F05F
S113F9B0D0F940F628006A4900FB06164FF47A771E
S113F9C002E00520FFF78AFF96F87D012F280ED06C
S113F9D002A801F0BEF900AA02A904A801F0C5F921
S113F9E00098019907FB00108542EAD2FE242046C4
S113F9F007B0F0BDF0B4014640F62803584C03FBB1
S113FA0001418CB091F87D31FF22FF202F2B04BFE0
S113FA1091F84C305E2B56D14C31002304AC0025B8
S113FA2000AE03F00F079F555B1C04F8015B03F065
S113FA300F079F555B1C05F11007203504F8017B67
S113FA40102BEEDB012386F82030022408AB5C7017
S113FA501A7204249C705A730824DC7010241C71DC
S113FA6020245C7140249C718024DC7100245C722D
S113FA7055249C72AA24DC7200241C7300230C46B7
S113FA8014F8015B5E2D1EBF5B1C14F8015B5E2D38
S113FA9003D05B1C2E2BF3DB15E059180120002446
S113FAA0491C00AB11F8015B13F8016BB54202BFAE
S113FAB011F8015B13F8016BB54203D1A41C2E2C81
S113FAC0F0DB00E0FF200CB0F0BC70472DE9F843F8
S113FAD0044688462248002180F87D11914640F66C
S113FAE0280101FB04055E2085F8E200FF270120C0
S113FAF0A87100222E2105F1E300FFF70DFFA8797C
S113FB002E30A87105F20606C0B27080E0B201F092
S113FB1049FA02E00520FFF7E1FE70880028F9D1D8
S113FB200520FFF7DBFE444508D149462046FFF790
S113FB3038FF0746FE280FD020460AE095F87D01DD
S113FB4050B949464046FFF72CFF0746FE2803D02C
S113FB504046FFF74FFF07463846BDE8F2830000F2
S113FB60440BFF1F10B44F480178447882788368AF
S113FB70491CC9B2A1421BD3521CD2B2042AA6BF4B
S113FB800321002204214170C17829B15B1CB3F523
S113FB90966F07D9002104E05B1EB3F5347F01D2D0
S113FBA00121C17040499CB20C6081240C65002184
S113FBB00170836082703C49C86820F08000C8608E
S113FBC010BC704780B5002238494E20FCF7E8FC91
S113FBD0BDE80840012205214E20FEF7ADBE38B530
S113FBE0304C6268002937D0002A55D101280CBF57
S113FBF0002501252846FBF7AFFC45B32C48416F8F
S113FC00490603D5416D41F0040141654FF420726A
S113FC10416D41F001014165002101604160012114
S113FC20E1704FF49661A160816064214161F0212B
S113FC30816120490A600D22026000228A60416DC0
S113FC40490707D5416F41F04001416702E00020B8
S113FC501949086001201EE0F2B1FBF7BEFC01283F
S113FC6015D11348416F490603D5416D41F0040194
S113FC7041650021016040F202210E4A9160416D0C
S113FC80490707D5416F41F04001416702E0012077
S113FC90094908600020606031BD02484068C0B274
S113FCA070470000F805FF1F0880034065FB000053
S113FCB0008003408C8003401000FE4380B5FBF7B6
S113FCC08CFC012801D1002002BD012002BD0000EE
S113FCD013B500EB4001DFF84C0400EBC10460688D
S113FCE030B1012201A901F0D1F9606801F0DDF918
S113FCF013BD10B500EB4001DFF8280400EBC1048C
S113FD0082B06068C8B105218DF80110012200217C
S113FD108DF800100DF1010101F0B8F960680122BD
S113FD2000A901E0012200A901F0D8F99DF8001012
S113FD306068C907F6D401F0B8F913BD7CB5044670
S113FD40022C80F0858004EB4400C000DFF8D4234B
S113FD508518696800297BD18058FEF791FF686097
S113FD60002875D050212046FFF7B2FF01208DF8FE
S113FD700400022200208DF8050001A9686801F042
S113FD8085F9686801F091F990208DF8000000AEC3
S113FD900020707070800422686800A901F076F970
S113FDA06868022200A901F099F9686801F07DF9F8
S113FDB000202872707843281CBF4828492802D0A4
S113FDC04B2804D007E0002141F0020106E00021A5
S113FDD041F0040102E0002141F0010129720128EF
S113FDE018D002281CD0032823D0042824D00528A6
S113FDF025D0412811D043281BD0492810D04A28A7
S113FE0011D04B2812D08C2813D08D2814D08E28D2
S113FE1015D017E04FF4803015E04FF4001012E0D5
S113FE204FF400300FE04FF480000CE04FF400007A
S113FE3009E04FF4802006E04FF4002003E04FF483
S113FE40801000E00020E86004212046FFF740FF16
S113FE5073BD00EB4001B34800EBC100C0687047BC
S113FE6000EB4001AF4800EBC1000069704700EBB4
S113FE704002AC4800EBC2004161704700EB400116
S113FE80A84800EBC100406970477CB5144600EBFC
S113FE904002A44800EBC2061D467068002818BF43
S113FEA0002C1AD0CDB10B228DF800208DF8031050
S113FEB00A0C8DF801200A0A00218DF802208DF821
S113FEC00410052200A901F0E1F870682A462146D1
S113FED001F004F9706801F0E8F873BD00EB40022A
S113FEE0904800EBC200426802B1016170477CB5E2
S113FEF004460D4604EB44008A4901EBC0067068D1
S113FF0040B3706928B13169080504BF204600F088
S113FF10BFF806212046FFF7DBFE02208DF8000023
S113FF2000A930698DF80300020C4A700D71020AB1
S113FF308A700522706801F0A9F8706801F0B5F8BC
S113FF402046FFF7D6FE04212046FFF7C1FE3069A4
S113FF50401C306173BD2DE9F04380460D4608EB2B
S113FF604800704901EBC00683B07068002714464E
S113FF704FF0AD0900281CBF002D002C00F0858037
S113FF80307CC0073BD515F8011B4046FFF7AFFF97
S113FF90641E34E08DF80490012101A815F8012BAA
S113FFA00A54641E4A1C3169491C3161317AC907FB
S113FFB008D515F8011BD2B2641E1154521C3069C5
S113FFC0401C3061D2B2706801A901F05FF870681A
S113FFD001F06BF8706990B1306900050FD14046AB
S113FFE0FFF787FE04208DF80000706830B101220D
S113FFF000A901F04BF8706801F057F80027A4B28B
S214010000022C404636DBFFF774FE706928B1316971
S214010010080504BF404600F03BF8002FBAD1062081
S2140100208DF80000706830B1012200A901F02EF8A9
S214010030706801F03AF8307AC0F3400171B14FF0C0
S214010040AF098DF8049001A831698DF807100A0CE4
S214010050427001270A0A827004219EE7C0F38000DD
S2140100600028EED015F8011B4046FFF740FF641E3E
S214010070F8D10AE0FFF73DFE04214046FFF728FECF
S2140100801CB129784046FFF732FF03B0BDE8F08384
S21401009070B504460D4604EB4400224901EBC00648
S2140100A082B07068E8B106212046FFF711FE2020D5
S2140100B08DF800008DF80350280C8DF801000422FD
S2140100C0280A8DF8020000A9706800F0DFFF70684A
S2140100D000F0EBFF2046FFF70CFE04212046FFF759
S2140100E0F7FD73BD38B50C4600EB40010D4A02EB37
S2140100F0C1056968A1B1082CA8BF07245021FFF7E4
S214010100E7FD01208DF8000002220748205C8DF8EB
S214010110010000A9686800F0B9FF686800F0C5FF33
S21401012031BD00000406FF1F3406FF1F38B5044624
S2140101300D4600A800F0FAFF35B114F8011B00A81F
S21401014000F0F8FF6D1EF8D1BDF8000032BD38B5DD
S21401015004461D46FFF7FFFE012204A92046FFF7CD
S214010160FAFE9DF8102029462046FFF7F4FE0122EC
S21401017005A92046FFF7EFFE01220DF115012046E5
S214010180FFF7E9FE01228DA12046FFF7E4FE31BD0F
S2140101902DE9F043044683B00D461646032700209A
S2140101A0FFF757FEA0F580580020FFF759FE81465D
S2140101B0C14505D30020FFF74CFE401E484506D238
S2140101C00A230FF26C324146002000F080F83146D7
S2140101D02846FFF7ABFF012C02D0022C09D014E011
S2140101E00C2E12DA019000962B4605220FF24C31A6
S2140101F007E0162E09DA0FF24C31019000962B46D5
S21401020005220020FFF7A3FF0027384603B0BDE80C
S214010210F0832DE9FC4F83B081460C46012500F0A2
S2140102209FFF06464FF0000A0020FFF712FEA0F5DA
S21401023080580398801B0190039B00279BB222469F
S2140102400AEB08010020FFF720FEA346019887422B
S21401025038D2324649465846FEF7CEFF48BBB81953
S214010260504400EB08060123224631460020FFF7E2
S2140102700CFE2578AB1C9BB2621C711C0020FFF79C
S21401028004FE2819661C4178807841EA002700A8F8
S21401029000F04CFF35B116F8011B00A800F04AFF2C
S2140102A06D1EF8D1BDF80000B84214BF0225002526
S2140102B00CE004987F1C0BF1010B0028C6D1002727
S2140102C04FF0FF3ABA44BAF5805FB5D3D3E0F8B53C
S2140102D00D46044616461F460021FFF7C8FD29466F
S2140102E02046FFF7D5FE29462046FFF7F7FD39469B
S2140102F03046FFF71BFFADF802008DF800700522AF
S2140103000FF248212046FFF726FE012200A92046CB
S214010310FFF721FE9DF8002031462046FFF71BFE21
S21401032001220DF102012046FFF715FE01220DF113
S21401033003012046FFF70FFE012220A12046FFF70A
S2140103400AFEF1BD2DE9FC4104460D461646374628
S214010350A84600A800F0EAFE37B118F8011B00A86D
S21401036000F0E8FE7F1EF8D1BDF800000FF2E411A0
S214010370ADF804008DF8026004222046FFF7EBFD7D
S21401038001220DF102012046FFF7E5FD9DF802204E
S21401039029462046FFF7DFFD012201A92046FFF787
S2140103A0DAFD01220DF105012046FFF7D4FD0122F9
S2140103B002A12046FFF7CFFDBDE8F3815D000000F6
S2140103C02DE9FD4F82B00C46012500F0C9FE064618
S2140103D00398DDF83890DDF84080801B4FF0000A66
S2140103E0019008E004987F1C0BF1010B80B90027EF
S2140103F04FF0FF3ABA440F9882453CD2039B002740
S2140104009BB222460AEB09014046FFF73EFDA34692
S21401041001988742EED2029932465846FEF7ECFE24
S2140104200028DFD1B819504400EB09060123224603
S21401043031464046FFF729FD2578AB1C9BB2621C6E
S214010440711C4046FFF721FD2819641C417880780D
S21401045041EA002600A800F069FE35B114F8011B38
S21401046000A800F067FE6D1EF8D1BDF80000B0428E
S2140104700CBF00250225284605B0BDE8F08F10B553
S21401048090B00020FFF75AFC284C0FF2C000002362
S214010490402200A9FFF7BDFEA8BB0A220FF2900179
S2140104A00DF10100FEF7A8FE68BB0123402200A95A
S2140104B00FF28800FFF7ADFE68B99DF800000C2822
S2140104C009DA02460DF101012046FBF72BFB9DF8E8
S2140104D00010002008550123402200A90FF26400F5
S2140104E0FFF797FE78B99DF8000016280BDA02464A
S2140104F00DF1010104F10C00FBF714FB9DF800104F
S214010500091900200873207828B908220FF24C0137
S2140105102046FBF707FB207B28B904F1240104F1F0
S2140105200C0000F039FE10B010BD00009C06FF1F45
S2140105304368616C6C656E67657200005B70636230
S2140105403D0000005B7365723D0000005B686472ED
S2140105503D0000005B66773D0000000050434231DD
S2140105603032370010B5DFF850460120208002E017
S2140105700520FFF7B3F920880028F9D160880828FC
S21401058003DA0520FFF7AAF9F8E710BD38B50146EA
S21401059043F612230A884FF07E509A421DD18C886A
S2140105A0DCB1B1F9020000FA84F000F017FE05464E
S2140105B0204600F01DFE0146284600F029FEDFF821
S2140105C0FC1500F0A3FE01D8084632BDDFF8F01591
S2140105D000F0AEFE38BFDFF8EC0532BD80B5002076
S2140105E0FFF7ACFB00210020FFF752FD0021084673
S2140105F0FFF73DFC00210846FFF770FCBDE8084008
S2140106000C22DFF8C4150020FFF7A5BC2DE9F04742
S2140106100020FFF793FBDFF8B4750C233A1D002189
S2140106200020FFF732FCB88843F61221884273D1C6
S214010630F86800F0DDFDDFF8981500F0E9FD0446E6
S214010640381DFFF7A3FF8046204600F083FEDFF843
S2140106508425DFF8843500F0A5FE06468946404627
S21401066000F078FE04460D464FF08B4ADFF86C0525
S214010670414600F069FF00F06DFE02460B4630462B
S214010680494600F0CDFFDFF85825DFF8583501F070
S21401069087F801F0A9F9514600F056FF00F05AFE1E
S2140106A0DFF844354FF0663201F07AF822462B46E1
S2140106B000F078FE01F0E0F938804146DFF82C05BD
S2140106C000F042FF00F046FE02460B463046494621
S2140106D000F0A6FFDFF80825DFF8083501F060F81E
S2140106E001F082F9514600F02FFF00F033FEDFF8EB
S2140106F0F8344FF0663201F053F822462B4600F0EC
S21401070051FE01F0B9F9788080B2FAF7ADFFBDE885
S214010710F0473220FFF7E2B8BDE8F08710B50020B9
S214010720FFF70CFBDFF8A4440C23221D0021002058
S214010730FFF7ABFBA08843F61221884208D0201DA4
S21401074000F0D4F8FFF74AFF201DBDE810400DE089
S21401075010BD10B1012804D07047DFF8700440883E
S21401076002E0DFF868040088FAF77EBF2DE9F0475B
S2140107700446A06800F03CFDDFF8541400F048FD84
S21401078005462046FFF702FF8046284600F0E2FDB8
S214010790DFF84024DFF8403400F004FE06468A46BF
S2140107A0404600F0D7FD04460D46DFF82074DFF81A
S2140107B02C044FF08B49414600F0C6FE00F0CAFDFE
S2140107C002460B463046514600F02AFFDFF8102459
S2140107D0DFF8103400F0E4FF01F006F9494600F0B6
S2140107E0B3FE00F0B7FDDFF800344FF0663200F0DC
S2140107F0D7FF22462B4600F0D5FD01F03DF93880A3
S2140108004146DFF8E80300F09FFE00F0A3FD024634
S2140108100B463046514600F003FFDFF8C423DFF8ED
S214010820C43300F0BDFF01F0DFF8494600F08CFE4E
S21401083000F090FDDFF8B0334FF0663200F0B0FF05
S21401084022462B4600F0AEFD01F016F9788080B204
S214010850FAF70AFFBDE8F04784E62DE9F041DFF834
S21401086058737D880188002443F612224FF07E5883
S21401087091421CD18688D6B1B0F9020000FA86F002
S21401088000F0ACFC8046304600F0B2FC0146404623
S21401089000F0BEFCC94900F039FD804698BF884685
S2140108A005D9C74900F044FD38BFDFF81883012D8C
S2140108B008DB07F20600294630F8022B1419A4B209
S2140108C0491EF9D194FBF5F040F6976148434FF481
S2140108D07A71B0FBF1F080B200F08AFC414600F07C
S2140108E097FC01F0F5F880B2BDE8F0812DE9F047FC
S2140108F0064640F67F70FAF7B7FE3220FEF7EEFFA7
S214010900FFF730FE3046FFF7A8FF00F071FCB9494B
S21401091000F07EFC00F01EFDB74AB84B01F0FAF875
S214010920AC4AAD4B00F03CFF01F05EF800F012FD62
S21401093080468A46A748A8494246534600F032FDFB
S21401094004460D46A14FAE494FF08B494FF080400B
S21401095022462B4601F0DEF8A14AA24B00F020FF0A
S21401096001F042F8494600F0EFFD00F0F3FC9E4B23
S2140109704FF0663200F014FF01F07EF83880224610
S2140109804FF020409F492B4601F0C4F8944A954BFE
S21401099000F006FF01F028F8494600F0D5FD00F00A
S2140109A0D9FC914B4FF0663200F0FAFE01F064F884
S2140109B0788080B2FAF758FE3220FEF78FFFFFF7F5
S2140109C0D1FD3046FFF749FFB080424600208E49F0
S2140109D0534600F0E7FC01F065F8B0600020708037
S2140109E043F612203080BDE8F08738B504460D4640
S2140109F07548FFF732FF00F0FBFB7E4900F008FC6C
S214010A0013E038B504467A48B0F848000D4600F0C1
S214010A10EFFB00F09FFC7D4A7D4B00F0C3FC7D4B55
S214010A20002200F0BDFE00F0DFFF02460223294649
S214010A30204601F0E3F8C0B232BD70B504466C48FA
S214010A40B0F94A000D46002600F0C8FB00F082FC13
S214010A506E4A6F4B00F0A6FC6E4B002200F0A0FE23
S214010A6000F0C2FF314600F063FC03D26A4900F091
S214010A706BFD06E0694900F049FC02D82D21217082
S214010A80012602460223691E301901F0B7F8301814
S214010A90C0B270BD1CB5624C206818B1022843D0A4
S214010AA01AD313BD01F0E6FB012806D05048B0F872
S214010AB0480040F24551884241DB00A800F049F960
S214010AC0009860600198A06001F075FC012808BFDD
S214010AD001F079FC012031E000A800F03AF96268E3
S214010AE0009BA0680199934204D09A1A4FF47A7336
S214010AF003FB0211081A40F6B83188421FD301F0F1
S214010B00B9FB012806D03A48B0F8480040F24551F2
S214010B10884207DB43490120086060680A3060604C
S214010B2002200BE0002009E000A800F012F960683E
S214010B300099884203D23B4900200860206013BD1B
S214010B40374800687047411E8941C9433648C90F76
S214010B5001607047F8B51D4E01F026FC28B900204B
S214010B603061012030490860F1BD301DFFF70EFDF0
S214010B7007461F48B0F8520000F03AFB00F0EAFBC7
S214010B802A4A2B4B00F00EFC04460D46384600F070
S214010B90E1FB02460B462046294600F001FE00F026
S214010BA023FF0E4900F0C4FBD9D23069401C3061E6
S214010BB00628D6DB0020D5E70404FF1FCDCC8C3FEA
S214010BC06766663F6666663F901DFF1F8C1DFF1FAA
S214010BD0002474493BDF4F8D970E32409A99194194
S214010BE0736891ED7C3F014066660A40CDCC5C415E
S214010BF07C1BFF1F00007A44D122DB491A901B4060
S214010C00333323C099992BC080842E4180B740820C
S214010C10E2C7F93F00408F40000080BF0BD7233C5E
S214010C20DC1DFF1F1820FE431C18FE43809FCC9A34
S214010C30B3996E3F30B50C460021A16015494A684C
S214010C40012A06D10968B0FBF1F00021C4E90001D0
S214010C5030BD114B1B68022A09D1D3F89011A1FBB4
S214010C6000014FF47A72002301F020FCEEE7D3F87E
S214010C7090514FF47A72B2FBF5F20A60D3F89051B4
S214010C806A43B2F57A7F02D101224A60DAE702228C
S214010C904A60E2E7041EFF1F200AFF1FF0B4D0E9F6
S214010CA00045D1E90067A4197D41C2E900450B4B17
S214010CB080681B688968D3F898310E18591A8842DB
S214010CC008D3601C45F10001C2E90001F01A9060EA
S214010CD0F0BC70479660F0BC704700BF200AFF1F4B
S214010CE0F8B504461848026802F5BE700146038945
S214010CF0DBB1D2F87C5103F1010C01E029462D68E5
S214010D00BCF1010C11D0D4E91167D5E911239F423A
S214010D100BD301D8964208D3D5E91167D4E911233C
S214010D209F42EBD301D89642E8D3626823681360EA
S214010D305A602246FDF78CFCA06840F48070A060E3
S214010D40BDE8F14009F09EBD200AFF1F002201F018
S214010D5029BC10B584B0044600A801F053FC214616
S214010D6000A801F073FC04B010BD10B40B6849680C
S214010D704468A1423CBF01F57A715B1E0068181AEF
S214010D80091BB1F57A7F08D94FF47A73B1FBF3F3F7
S214010D904FF47A74181804FB13111060516010BCDC
S214010DA0704700002DE9F04704000CD1B24DB34E58
S214010DB0D5F804805FFA88F001F094FC07000AD1A8
S214010DC02B20BDE8F087012C02D1AD4DAD4EEFE7EB
S214010DD04620BDE8F087B5E80F56A6E80F56203D39
S214010DE0203E05215FFA88F0FAF7C6FD3762F06803
S214010DF0B16801EBC0010001B1FBF0F0B0F5005F96
S214010E0028BF4FF0FF305BD2010A3970787000209E
S214010E10B8700C20F8700020B871387CC0F302104E
S214010E2038B1387CC0F302100121401C01FA00F0F1
S214010E30401EF87401207875787C40F0C000787404
S214010E40387C40F0880038747068FAF7D8FD787BF3
S214010E5040F0060078732869FDF742FDF0622869C4
S214010E600020C0460FF29501B06232462869FBF7B2
S214010E7097FB0FF25501706232466869FBF790FBEB
S214010E8070620122A9692869C9B2FDF755FDE969B1
S214010E9068690122C9B2FDF74FFDF8787A4900F07A
S214010EA07700F870F87840F02400F870B87940F0D0
S214010EB00B00B87140F6280000FB04100660002005
S214010EC0BDE8F0876EE70000026B016A521C026300
S214010ED009790A0702D5826C521C8264CA0702D5B8
S214010EE0026C521C02644A0702D5026D521C02654E
S214010EF0890702D5416C491C4164704770B50446A8
S214010F0082B0206B256A401C2063287980060AD5AA
S214010F10E979606805280CBF0120002000F078F808
S214010F20606B401C6063287900063AD56068052826
S214010F300CBF0121002140F62802534B12FB013160
S214010F404FF0FF3091F88027930705D502F0FD009A
S214010F5081F88007FF2012E00A8982B1501E01F253
S214010F6080720881536818785E1C56601A785E2A6B
S214010F7005D191F8802742F0020281F8802700907F
S214010F800098002805D40098E871A06B401CA06367
S214010F9073BDE87800F07F00E870E87840F0040060
S214010FA0E87073BD40F62801374A11FB00218B79A2
S214010FB06BB3DFF8C8C001F206025380542313FB5B
S214010FC000C0006AC37803F0FB03C370002381F8F6
S214010FD07D3191F8803703F0FE0381F880370023D6
S214010FE081F8793153885B1E538001F2807201F2D9
S214010FF0E201516001790906FCD551680978C17191
S2140110005168491C5160C17841F08801C170704730
S21401101038B50C461C4991F826285ABB40F62802DA
S21401102012FB001595F8240848B1FF2C0DD002F0EC
S21401103043F85E2085F84C00012085F87D015E2C82
S21401104003D15E2085F8240831BD95F8240828B11F
S214011050FF2C08BF5E24002085F8240895F87D0142
S214011060401980F84C4095F87D019528BCBF401C7E
S21401107085F87D0131BD000080AF01000C1CFF1F0B
S214011080A0AF0100601CFF1F440BFF1F18B428B15E
S21401109003689B691C0005D12C21C1604FF0FF300D
S2140110A012BC704701B010BC184738B5044600257D
S2140110B014B94FF0FF3032BD2068C369180004D060
S2140110C000220321204698470546A06920B1022246
S2140110D00021204602F06EF8284632BD70B504465F
S2140110E00D46164600204CB1A16909B1022E13DB4C
S2140110F020684369180004D12C20E0604FF0FF30CF
S21401110070BD00291ABF721E691C294620469847E1
S21401111000280AD4A16941B1012E01DA002070BD70
S214011120401CE16929700021A16170BD4FF6FF7175
S214011130018070470288514001804AF2010208216D
S21401114003884FEA530C03F00103012BA6BF82EA82
S2140111500C030380A0F800C0491EF1D170470000BF
S21401116000F10103810704D010F8011B89B1810742
S214011170FAD10268B2F10131914311F0803F04BF08
S21401118050F8042FF6E710F8011B11B110F8011BF7
S214011190FBE7C01A704700005FEA000C830706D021
S2140111A011F8013B00F8013BB3B18307F8D10A6897
S2140111B0B2F1013323EA020313F0803F02BF40F885
S2140111C0042B51F8042FF3E711F8013B00F8013B1B
S2140111D013B111F8013BF9E760467047002840F16A
S2140111E00980F446404200F005F850F000406047A0
S2140111F0002800BF0AD0B0FA80F18840D1F19D01E5
S214011200C905020672F1004241EB1020704700004A
S21401121010B5FF2313EAD0541DBF13EAD1529C42E6
S2140112209A4239E0A41ADA0780EA0103134042EA37
S214011230012142EA0020421A3CBF641E01EB420231
S214011240090AB2FBF1FE01FB1E221202B2FBF1F00B
S21401125001FB10226EF30F201202B2FBF1FE4EEAE2
S21401126000207F3406DDFE2C24DA53EA500050EBD2
S214011270C45010BDD4F1020401FB1E2240F080715F
S214011280192C1DDC21FA04F0C4F12004A1401143FD
S21401129071F10042584110BD9C421ABF03EAD15277
S2140112A09A420FE080EA010E0EF00043400004D09F
S2140112B0490016D143F0FF4010BD490008BFD34393
S2140112C0180010BD9C4205D1D21AF7D001F000419A
S2140112D0484010BD4A0212BF0846484000F0004090
S2140112E010BD4AB90902B1FA81F2914044B1A4187D
S2140112F0C00140F000409EE7C90141F00041524262
S2140113000002B0FA80F4A040141B94E74FF0807CF2
S2140113101CEB400F94BF1CEB410F05E040EA010CAB
S2140113205FEA4C0C01D28142704718BF8842704771
S2140113304FF0807C1CEB400F94BF1CEB410F05E087
S21401134040EA010C5FEA4C0C01D28842704718BF94
S214011350814270475FF0FF0C1CEAD05114BF614513
S21401136006E0C110400721F0E04101F160517047ED
S21401137079B900F0004100020AD0B0FA80FC00FA08
S2140113800CF001F16051A1EB0C5101EBD0214005AD
S214011390704741020CBF40F4E0016FF000010020ED
S2140113A070470000B0B581EA030C0CF0004C40F227
S2140113B0FF7515EA11541DBF15EA1357AC42AF422B
S2140113C039E0E41923EA455343F48013C90241F096
S2140113D0004141EA505EC7021100A7FB0202002845
S2140113E04FF00000EEFB01204FF00001E3FB072168
S2140113F018BF42F00102401800214941E3FB0E01EB
S214011400A4F580640F0302D252004041494154F1D1
S21401141001046CDD470872F1004250F1000051EB07
S2140114200451A1F580115CBF41EA0C01B0BD4CEA44
S21401143005510020B0BD05EA1357AC4214BFAF42B8
S21401144041E050EA410E1CBF52EA430E02E06146FB
S2140114500020B0BD24423C441BD15FEA070EF6D003
S214011460090302BF01460020AEF1140EB1FA81F75E
S214011470AEEB070401FA07FE0C37C7F1200100FAAC
S21401148007F7C8404EEA000E23EA455343F480139B
S214011490A2E733F00043B3FA83F704BFB2FA82FE41
S2140114A077440B3FE41BB7F1200E2FBF02FA0EF371
S2140114B0BB40C7F1200E22FA0EFE38BF43EA0E03E8
S2140114C0BA40641C82E750EA410E14BF52EA430E4A
S2140114D06FF000014FF4001717EB430F8ABF194650
S2140114E017EB410FB5E74CEA05510020B0BDD4F12A
S2140114F00104B4F120070FDAC4F12007520828BF0F
S21401150042F0010210FA07F501FA07F7E1BF2A4394
S214011510E0403843E1400FE0352C98DCC7F1200469
S21401152052EA400220FA07F218BF42F0010231FAED
S21401153007F0A1400A43002172F1004250F1000079
S21401154051EB0C01B0BD0000FF2212EAD05C1DBFBA
S21401155012EAD153944593422BE09C44D30780EA88
S21401156001021A4043EA002043EA0121A1FB0030B0
S214011570410038BF40007CF17F010BDBFE294ADACF
S2140115805B0842EAC15153EA006373F1004C51EB28
S21401159010207047D1F1080CDCF120012FDB5B082D
S2140115A010FA01F10B4373F1004120FA0CF050419F
S2140115B0704794451CBF02EAD153934280EA010268
S2140115C002F000421DD0400019D0490017D05BB987
S2140115D0634514D00902B1FA81F39940BCEB030CC0
S2140115E0C00140F00040C1E70002B0FA80FC10FAEA
S2140115F00CF0B3EB0C0CC90141F00041B6E710004A
S214011600704740000AD0490008D010F1807F94BF8F
S21401161011F1807F02E042F0FF407047D0437047EF
S21401162070B44FF0004591EA030F44BF6B4000F0E1
S2140116307BBA00BF841A71EB030604D26E40001B0E
S214011640B141121973414FF4001C1CEB410F34BF1A
S2140116507CEB430684E00C0DA4EB1356362E7DDCA2
S214011660012E43DC45EAC32343EA525312BFD2029A
S21401167092025B08240545EAC12141EA5051D2EBAA
S214011680C020994125D407D1B0FA80F610FA06F1A8
S21401169064D00020203608E0B1FA81F6B140C6F1E8
S2140116A0200220FA02F21143B0404FEAF474B4EB80
S2140116B0465434F001064FEA74040AD8D6F50016EB
S2140116C0760D04F00044F04061FA06F25040F14015
S2140116D04840C00A40EA415021F0004128BF5FEA75
S2140116E0500550F1000044EBD12137E045EAC32311
S2140116F0DB0A45EAC121C90AB6F120050EDD42EA38
S2140117000242120CC5F1200603FA06F6EB4042EA45
S21401171006056D42984161F100010DE062FA06F599
S214011720F240554063FA06FC82EA0C02F3405A4046
S2140117306D42904161EB030111F4801F05D1641ED7
S214011740620502D06D004041494121F480114308F1
S21401175075F1004350F1000041EB045170BC704735
S2140117601CEB410F15D223F0004352EA43060BD07F
S2140117704FEA4C0CBCEB410F04D80C0D661E342E00
S214011780B7DDEBE7801A994150EA410608BF002110
S214011790E4E708BF1CEB430F28BF6FF00001DDE74D
S2140117A0F0B540F2FF7581EA030C0CF0004C15EA27
S2140117B011541DBF15EA1357AC42AF42E5E0BC41D8
S2140117C0C1F31301C3F31303801A994143F4801341
S2140117D004D2641E4000494180185941C90241EAB9
S2140117E05051B1FBF3F603FB1611A2FB0675D7EBBE
S2140117F0C020A94102D2761E80185941C90241EA89
S2140118005051B1FBF3FE03FB1E11A2FB0E75D7EB85
S214011810C020A94103D2AEF1010E801859418902B8
S21401182041EA9051760546EA8E2EB1FBF3F603FBAC
S2140118301611A2FB0675D7EB8020A94102D2761EAF
S21401184080185941C90241EA50514EEA060EB1FBD1
S214011850F3F603FB1611A2FB0675D7EBC020A941D0
S21401186002D2761E80185941C90241EA5051B1FB95
S214011870F3F703FB1711A2FB0735D3EBC020A941F1
S21401188067F100070CBF004247F0010766F3D52752
S2140118904FEA1E31B80814F5806412DDBD0775F1F4
S2140118A0004250EB0E5051EB045111F5801F5CBF06
S2140118B041EA0C01F0BD4CF07F6141F0E0410020AF
S2140118C0F0BDBD076D0840EA0E5041F48011D4F119
S2140118D00104B4F120060ADAC4F120060200E04051
S2140118E001FA06F3E1401843B24015430EE0342CEA
S2140118F013DCC6F1200445EA40056D0820FA06F21D
S214011900154321FA06F0A1400D43002175F100426E
S21401191050F1000051EB0C01F0BD00205FEA0C0114
S214011920F0BDCFB992185B41B3FA83F704BFB2FAA0
S21401193082F6BF190B3FB7F120062FBF02FA06F356
S214011940BB40C7F1200622FA06F638BF3343BA4039
S2140119501CB1E419641E33E77F4231F00041B1FA4D
S21401196081F404BFB0FA80F6A4190B3CB4F120064A
S2140119702FBF00FA06F1A140C4F1200620FA06F6B0
S21401198038BF3143A0403C1B1AE7AC421ABF05EAF8
S2140119901357AF4212E050EA41061CBF52EA430613
S2140119A0BFE750EA4107304661461CBF41EA055190
S2140119B0F0BD52EA430C08BFC143F0BD00204FF40E
S2140119C0001616EB410F98BF16EB430F08BF16EB38
S2140119D0410F24BFC14305E016EB430F0CBF614620
S2140119E04CEA0551F0BD00004FEAF17CBCF1E04C39
S2140119F02CBFBCF5001F11E05FEA4C0C34BFBCF1F4
S214011A007F5F2EE05FEA9C0C4FEA0C1C4FEA3C0C11
S214011A10C10071F100414CEB50707047C90241EAB8
S214011A205051C00218BF41F0010141F000414FEA98
S214011A306C50C0F10900212810D240EACC7CCCF1D0
S214011A40200C11FA0CF070F10040CCF1200C21FAB8
S214011A500CF00CF0004C40EB0C0070474FEACC70D9
S214011A607047490011F5001F04D84FEACC10FF302B
S214011A70C0057047C8177047F446400D40EAC120BC
S214011A80490006D200F014F8004248BF6FF000404B
S214011A90604700F00DF84FF0004188428CBF0846C1
S214011AA040426047400D40EAC120490080F00D8069
S214011AB040F00040490DA1F58061491C05D4D1F1E3
S214011AC01F0154BFC840C01770474FF00000704751
S214011AD04100090E7F3915D4D1F11F0114D44000FD
S214011AE007D2C00140F00040C84048BF6FF0004038
S214011AF07047C00140F00040C8404CBF4FF0004066
S214011B00404270470020704700424FF0004058BFE7
S214011B10C043704770B44FF0004591EA030C44BFD0
S214011B206B40FFF787BD00BF841A71EB030603D233
S214011B30001BB141121973414FF4001C1CEB410FFD
S214011B4034BF7CEB430443E00C0DA4EB1356352E57
S214011B5050DC45EAC323DB0A45EAC121C912B6F1C6
S214011B6020050DDD63FA05F6EB4086EA0305124211
S214011B7018BF45F00105C01851F100010CD213E061
S214011B8062FA06F5F2405540F3415A40B340F3403D
S214011B905A408018594107D349085FEA30005FEA86
S214011BA0350528BF45F0010501F58011420875F19C
S214011BB0004250F1000041EB045170BC4FF4001C90
S214011BC01CEB410F38BF70470020090D090570470F
S214011BD01CEB410F10D252EA43060BD0BCEB410F6F
S214011BE005D80C0DAB43661E342EB5DD02E0AB43C3
S214011BF08018594170BC704770BC70472DE9F0479A
S214011C00044600270D4692469846002C43D0012DE7
S214011C1041DBDFF8889050464946FFF777FB27708F
S214011C2018D8FFF797FB00221D4BFFF7B9FDFFF70A
S214011C3023FF00F130012170012701F0F1FA0022A3
S214011C40174BFFF7AFFBFFF7CFFE0146504601F0FB
S214011C50FDFA824600266D1E08F1010815E0504681
S214011C60FFF736FF00F1300139557F1CFFF7B6FA52
S214011C700146504601F0EAFA4946FFF765FC8246FE
S214011C8016B92E2038557F1C761C4645B8BFAF4284
S214011C90E5DB002038553846BDE8F08700002041D6
S214011CA000002440F8B50921062001F056FBDFF8B4
S214011CB09C06DFF89C46416ADFF89856DFF898667E
S214011CC041F0006141621F23816941F00061816139
S214011CD05022416A41F4800141620021016040F6D0
S214011CE0A2702060E16048F25F70606044F6FC21FB
S214011CF040F201102061A161A06345F2786145F6CA
S214011D00BB502064206840F0010020602B726420E4
S214011D102870002304206870AA7141F2342068807C
S214011D2068826B725020A87506220620E875642327
S214011D301F202876EA712B740020A980A982687674
S214011D404FF4C0220423EA606B74EA6129463046E8
S214011D5001F074FB304601F031FB2946304601F0B4
S214011D606DFBDFF8F87505F11001384601F066FBEA
S214011D70384601F023FB05F11001384601F05EFB01
S214011D80412030605220386049200FF2D90101F01D
S214011D9068FB0FF2A1114A2001F063FB0FF231013B
S214011DA0582001F05EFB012200214920FCF7C4FD0A
S214011DB0012200214A20FCF7BFFD01220121582003
S214011DC0FCF7BAFD206840F480302060F1BD0000C9
S214011DD070B5DFF88C45E069216A401C491C24284F
S214011DE0A4BF002000212162E061DFF8781501EB35
S214011DF08005E87801280CBF202600266878F9F7C8
S214011E0074FCA978DFF8500501F0030141F0500198
S214011E100162297801F01F01314341F04001016060
S214011E20206A242817DA04EB800000F12405E878FC
S214011E3001280CBF20200020AA78DFF8201502F028
S214011E40030242F050020A622A7802F01F0210438F
S214011E5040F040000860DFF8F804016821F0400116
S214011E60016070BDF8B5DFF80005DFF8EC640478B2
S214011E70306800065DD5DFF8E874DFF8E814F86925
S214011E8001EB8000407800F00700F9F72EFC31697D
S214011E90F869DFF8D82489B222F8101020282EDA43
S214011EA00022182804DBDFF8C8341B785B070CE037
S214011EB0102804DBDFF8B8341B789B0705E00828F8
S214011EC005DBDFF8AC341B78DB0748BF012258235B
S214011ED0DFF8A05413FB025232F83430994219DB72
S214011EE002EBC4025388994207DB93889942B8BF34
S214011EF0022510DBD28891420ADA01250BE022285E
S214011F001CBF2128232806D140F67B62914201DAC4
S214011F10002500E0032500EB40014900DFF85824C6
S214011F20895C01F00C01082903D0E9B2BDE8F44050
S214011F30C4E0F1BD70B50321062001F014FADFF804
S214011F401C040168090640F1B8800569DFF81064D1
S214011F50306A0A2855DADFF8141401EB400102282A
S214011F60A1F8485005D1ADB240F225418D421ADAAA
S214011F7027E0032804D1ADB2B5F5167F13DA20E0C9
S214011F80062809D1ADB240F225418D420BDBDFF8C0
S214011F90EC231E21117014E0072814D1ADB240F6CF
S214011FA0A4318D4201DB002426E040F25A518D42D5
S214011FB0A8BF022420DA40F216318D42A8BF0124C0
S214011FC01ADA032418E0082816D1318819B100213D
S214011FD07180B18031807188082902DA7188491CC4
S214011FE07180B1884A1C06EB4101B280CD80B18870
S214011FF00829A4BF0021B180E1B2BDE870402430B9
S2140120005CE0A0F10E01152957D20E2802D1B06965
S214012010401CB061B069B0F5C07F4ED301F04AFBF9
S214012020002849D0306A0E2804D1BDE8704001204E
S214012030FEF78FBB1B2804D1DFF83003A0F87E50D3
S21401204070BD1D2803D1DFF83803858070BD1E28BA
S21401205003D1DFF82C03C58070BD202802D1C84803
S214012060458170BD222828D10020B061FEF771FBA2
S21401207040F6B633BD4800F27E01B0F87E008A888D
S21401208012FA80F0CA8810FA82F04A8910FA82F0B1
S2140120908010C881B848C98990F8A421994202F0F5
S2140120A0030103DA022908D1082102E0022904D03B
S2140120B00A2180F8A41170BDB06170BD70B50546E7
S2140120C00E460824FEF73CFD05EB4501AA4B03EB43
S2140120D0410106F003020B785E0705D403F0030600
S2140120E0964201D1DE063DD543F004030B7052182B
S2140120F053785B1C5370202D00DA00B110248D78C4
S2140121004E78CB78087955FA86F252FA83F252FA6B
S21401211080F2944226DA0C7822071AD40322A842C7
S2140121203CBF2846012298423CBF18460222B042D4
S21401213038BF002204F00300824201D1E00603D535
S21401214042F00800087004E04879FF281CBF401CD4
S2140121504871087800F0FB0008700020487088700D
S214012160C870087170BD70B5024600200C46202A62
S21401217048DA7E48834E30F81250182A03DB7C4832
S214012180007840070AE0102A03DB794800788007C8
S21401219004E0082A04DB76480078C00748BF7A4E78
S2140121A02846FFF725F83146FFF7CEF90646C5F56E
S2140121B08050FFF713F801463046FFF729F87349B8
S2140121C0FFF7B6F8024603D205220FF2CC1106E05D
S2140121D06F49FFF79BF808D805220FF2C411204675
S2140121E0F9F7A0FC0420042105E00123052120467F
S2140121F0FFF704FD0146491E04D40A5D2E2AFAD1D2
S2140122004B220A5570BD5C48014612220A2301F88A
S214012210063B01F8063B01F8063B01F8063B521E59
S214012220F5D100F2C60103228A77002300F2EA0202
S21401223080F8EA301376022380F8A43103238B71E9
S2140122400B7380F8C63093741E204C4908704FF00B
S214012250FF314348C1610162704700280CBF40F658
S214012260B63140F657414148B0F852208A42804183
S214012270C00F704710B40020002140F66812384B9A
S21401228000E0491C5C8889B2A14205D203EB4104F7
S214012290E4889442F5DA012010BC7047304940F2D8
S2140122A07F10886170472DE9F84F3A4C0022227062
S2140122B0202844DA002519B102291ED004D33EE0B5
S2140122C02146FFF750FF3AE0061D0746B04236DAD0
S2140122D000F103080FF26C092919F8B2FFF743FF62
S2140122E04519474505DA032249462819F9F71AFC24
S2140122F0AD1C7F1CB742EFDB21E0061D0746B0424E
S2140123001DDA00F103080FF23C090FF23C0A07F14F
S214012310010B5A465146281901F0E6F945192919C3
S214012320F8B2FFF720FF4519474505DA032249466B
S2140123302819F9F7F7FBAD1C5F46B742E7DB2046E5
S214012340BDE8F28F2C20000025642D001880044083
S21401235000600340541DFF1F00B0034000B00B4057
S2140123600404FF1FB804FF1F451EFF1F7C1BFF1F31
S214012370471EFF1F4805FF1FDC17FF1F481EFF1FD4
S214012380FA1BFF1F6666964000002041CDCC4C3EEE
S2140123900100C642AC1CFF1F3C304B32000000005F
S2140123A03E39394B000000002A480078C008FFE794
S2140123B000F00100704780B5FDF76FFC401E8041BC
S2140123C0C043C00F02BD00210020FDF708BCF8B5D0
S2140123D0214C60780025000603D5FEF7B1FB00B955
S2140123E001251E4800782946FDF7F9FB01F0FFF9A3
S2140123F008BB1B480078C8B11A4A0021931C254621
S21401240006462F7893F800C0BC451CBF1F700121FB
S2140124106D1C5B1C761EF4D109B9117859B90521DA
S21401242011702146BDE8F44001F0E8B92046BDE848
S214012430F24001F0F9B9F1BD074902780A70407817
S214012440487070470748017809B1491E0170704706
S21401245000000000201EFF1F161EFF1F461EFF1F46
S2140124604C1EFF1F121EFF1F13F0004C03D55B42CC
S214012470524263F100039CEA210C00F0178010B56C
S214012480644603D34942404261F1000100F00EF870
S214012490640004D34942404261F10001244203D55D
S2140124A05B42524263F1000310BD00001B4213D190
S2140124B0094236D12AB18446B0FBF2F002FB10C2C3
S2140124C0704701F001BAFCD30022002370470B00CD
S2140124D00200002100207047904271EB030CF6D3F6
S2140124E070B5B1FA81F4B3FA83F52C1BA340C4F19D
S2140124F0200532FA05F63343A2405FF00046E64077
S21401250002E05B085FEA3202841A71EB030524BF1E
S214012510204629467641F4D302000B003000002104
S21401252070BD012ACFD970B5140C20D0B1FA81F450
S214012530B2FA82F5C4F120046419B4F12006D6D3A8
S214012540B2405FF00044F440002502E052085FEA22
S2140125503303C61A71EB020E24BF3046714664413E
S2140125606D41F3D302000B002000290070BD0C461C
S214012570B1FBF2F102FB11452D0445EA1045B5FB0E
S214012580F2F402FB145580B240EA0545B5FBF2F0C1
S21401259002FB105240EA044070BD000062F30F22B5
S2140125A062F31F42401810F0030308D0C91A1FD364
S2140125B0DB0748BF00F8012D28BF20F8022D1300C5
S2140125C030B414461546103928BF20E93C00FAD825
S2140125D0490728BF20E90C0048BF40F8042D8900B0
S2140125E028BF20F8022D48BF00F8012D30BC7047E7
S2140125F0C91818BF00F8012DCB0728BF00F8012D18
S2140126007047000038B504001DD00F480568F9F77B
S21401261055FB05F5B2700EC80EC4D5F89C110C3CDE
S214012620080003D0D5F8A0018847A060224605F52A
S214012630B8712046FEF732FBF9F74AFF2046BDE89F
S2140126403240FCF763BB31BD200AFF1F2DE9F84677
S214012650064623480568D5F890A1D6E900490F46F5
S2140126602046494652460023FFF720FF012908D39A
S2140126704FF0FF30386040F2E73078600020BDE868
S214012680F2864FF47A72A2FB040102FB09110023C1
S2140126905246FFF70BFF04464FF47A720023FFF70A
S2140126A005FF4FF47A71386001FB10447C604FF4EB
S2140126B0FA61B068A1FB000152460023FFF7F6FE5F
S2140126C0D5F898210023FFF7F1FE401C41F10001E7
S2140126D0400840EAC170001978600120BDE8F28622
S2140126E0200AFF1F052810D8DFE800F003050709B8
S2140126F00B0D07487047074870470748704707485B
S214012700704707487047074870470020704700BF6A
S21401271000A0064000B0064000C0064000D00640BB
S21401272000A00E4000B00E4010B5DFF85C1ADFF8CE
S2140127305C0ADFF85C4A00220A704A708A702270CE
S214012740027062704270A2708270DFF8481A0A70D6
S21401275001F04EF901F058F9607840F00900607018
S21401276000F00BF80421DFF8300A80F8211800F693
S214012770210000214170817010BD70B4DFF8140A89
S214012780DFF80C3ADFF8001A02781C780D78160686
S21401279010D4A5421CBF0C7042F080025C784D78C4
S2140127A0A5421CBF4C7042F080029B788C789C42FC
S2140127B016D012E0A54203D02C430C7042F08002E2
S2140127C04D785C78A54203D02C434C7042F08002D1
S2140127D08C789B789C4203D023438B7042F0800216
S2140127E0027070BC7047F8B5DFF8AC4904F5BE75E9
S2140127F06878A8B394F82118884231D3042908BF11
S21401280000F037F8687894F82118884228D3002019
S214012810A07101F071F8F0B194F87C01C00702D5FF
S21401282000F003FB14E094F82128FF210020931EFA
S214012830012B06DB04F24D0616F8017B79405B1E80
S214012840FAD11219C9B292F84B20914208BF012061
S21401285008B100F059F800206870042084F82108B7
S21401286094F8260800281CBFBDE8F14001F00FB916
S214012870F1BDDFF8240990F87C1190F84D2001F0A5
S214012880F40180F87C1112060CD541F0080180F89D
S2140128907C114A0751BF052141F0030180F87C11E4
S2140128A0062130E000F24D025378082B08D0092BA0
S2140128B013D0102B04D0202B18BF212B10D016E0DC
S2140128C041F0080180F87C114A0751BF042141F00C
S2140128D0030180F87C11052115E09178491D12E06D
S2140128E09278921D80F8212841F0010107E0927844
S2140128F04B0707D5921D80F8212841F0030180F887
S2140129007C117047511DDCE330B5DFF88C4894F834
S2140129104D0083B0400616D594F8220840280DD005
S214012920412808D0462809D0532818BF7E2807D149
S21401293001F0CEF804E001F0E0F901E000F07EFBE2
S214012940002084F8220894F84D0000066BD504F1A7
S2140129504E00FFF771FDDFF838084078C0073FD515
S214012960DFF83008007800063AD5DFF81C0805784D
S2140129704278DFF8181880780D704A708870402009
S214012980A179091981F8E2000021A079401CA07103
S214012990C0B2001980F8E210A079401CA07100F0C6
S2140129A035FBE80627D500A90DF1010000F06FFE02
S2140129B0A1799DF80000091981F8E200A0799DF837
S2140129C00110401CA071C0B2001980F8E210A07975
S2140129D0401CA07194F8E300801C84F8E3000AE030
S2140129E001F054F938B901A904F1E20001F064F8E4
S2140129F028B10198A07100F0C0F903B030BDA179EB
S214012A00091981F8E200A079401CA07194F87C01B4
S214012A10C00703D500F0C7FA00F06EFB002001F0F6
S214012A2023F803B030BD00F041F803B030BD70B5F7
S214012A30DFF86847204601F053F8B0B321785039E3
S214012A40012902D92C3906D070BD01462046BDE8C1
S214012A50704001F0E5B9E678A5780C20232E17D052
S214012A60252E09D0512E0DD0742E17D1DFF8301730
S214012A70601C01F004FE11E0DFF82417601C01F071
S214012A80E5FD0BE0DFF81817601C01F0E1FF05E03B
S214012A9000F099FFDFF8081700F039F932462946A9
S214012AA0BDE87040DFF8FC36F4E070BD10B5DFF825
S214012AB0E84604F24D004178072933D0082900F092
S214012AC0BC80092939D0102914D020297CD021298D
S214012AD000F08780232900F0BC80502943D051297B
S214012AE038D0522948D0572900F0C2807C2900F0FE
S214012AF0CA8047E094F8220840280DD0412808D023
S214012B00462809D0532818BF7E2807D100F0E0FFD9
S214012B1004E001F0F2F801E000F090FA002084F8F9
S214012B20220810BD81780129FBD1C07800F085FD0F
S214012B30FFF723FEBDE81040F6E081780129F0D1C9
S214012B40DFF84C164A78C07842F001024A7000F06D
S214012B50AEFDEFE780780228E3D1042104F14E00B0
S214012B6000F0B9FFE6E780780128DAD1032104F105
S214012B704E0000F0B0FFDDE781780429D1DB8079D3
S214012B8000F095FD94F84D003F210842C9D0A17987
S214012B900919102081F8E200DFF80C16A0790978EF
S214012BA0401CA071C0B2001980F8E210A079401C48
S214012BB0A07194F87C01C00703D500F0F4F900F089
S214012BC09BFABDE81040D5E081780129A9D1C078EB
S214012BD00028A6D094F87C0140F0040084F87C011B
S214012BE0D0E7807801289CD194F87C01DFF8A01505
S214012BF040F0040084F87C01487840F001004870F9
S214012C00DFF8A815DFF8A00500780870C243487001
S214012C108A70CA703F2294F84D1011423FF481AF7A
S214012C20A2791219102182F8E210A179491CA1712A
S214012C30C9B2091981F8E200B8E701F09AF8DFF89D
S214012C4050054078C00748BF00F0E0F9BDE81040E5
S214012C5093E0DFF85405DFF84C450078214600F094
S214012C6056F86078811CC9B2204600F017FAEDE7E5
S214012C70817800293FF455AFC078DFF8341500F0AD
S214012C80010008707EE78078811C04F14E0000F098
S214012C9022FF77E738B515461C467E222270A170C2
S214012CA0062821D8DFE800F00410202004141400C0
S214012CB0062060706F20E0700320207100F083FE14
S214012CC06071A57101201AE02079C01C607017E0C0
S214012CD0062060706F20E0700320207100F073FE04
S214012CE06071A57105200AE0062060706F20E07013
S214012CF00320207100F067FE6071A5710420E07169
S214012D006078811C2046BDE8344000F0D0BE80B516
S214012D100A46242111700D21517090700C21D01C8F
S214012D2002F0FAF8012002BD80B5DFF86C0490F8D5
S214012D304D103F2211421CD082791218102182F8C0
S214012D40E210DFF8642481791278491C8171C9B2D6
S214012D50091881F8E2208179491C817190F87C017B
S214012D60C00703D500F01FF900F0C6F9BDE8024020
S214012D7000E001BD002000F077BE38B5DFF818444A
S214012D8094F87C01C10608D500F0EF0084F87C01B8
S214012D9004F2E2010879C01C487094F8E20084F855
S214012DA0220894F87C01C00723D500F0FCF800F057
S214012DB023F904F2E2014A7872B1942A0CDA00226D
S214012DC007E01319521C93F8E450454083F8E45089
S214012DD0D2B24B789A42F4DB00F08EF9DFF8CC03DE
S214012DE00178027A51400170427A4178514041702F
S214012DF010E0FF20A17939B104F2E2020B4612F885
S214012E00015B68405B1EFAD1091981F8E200A079DE
S214012E10401CA0710020BDE8324000F025BEDFF85E
S214012E20780390F8E310491C05E1F8B5DFF87C63F8
S214012E30FF20307270720025222000F045F9D64C32
S214012E4094F821180020C91E012921DB04F24D0245
S214012E504AF20103377A96F809C047EA0C2792F836
S214012E6000C08CEA07074FF0080C4FEA570E07F030
S214012E700107012FACBF83EA0E077746BCF1010CB0
S214012E80F3D13772401C3F0A521C77728842E1DB4D
S214012E9094F87C21011901F24D00920723D500F028
S214012EA02DF80546012D1CD194F87C01810723D508
S214012EB094F84D1009061FD400071DD404F24D06E0
S214012EC0B078C8B100F098F80021B278914213DAD0
S214012ED00A19491C92F85030434082F85030C9B262
S214012EE0F3E7002508E0327A4078824201BF707A23
S214012EF091F84D10884201252846F2BD2DE9F0478C
S214012F00AA4E377AB7720446757AF5724FF0000802
S214012F10307800F0D9F8707800F0D6F8B07800F084
S214012F20D3F8F07800F0D0F8307A6178884202BFA2
S214012F30707A2178884206D1974900204FF001081F
S214012F4081F823082CE0377275723779384600F01D
S214012F50BBF87579284600F0B7F896F8069048460B
S214012F6000F0B2F896F807A0504600F0ADF8307AB7
S214012F706178884202BF707A2178884210D18648EB
S214012F8090F82318491C80F82318C9B2102907DACB
S214012F903770757086F8029086F803A04FF0010826
S214012FA04046BDE8F08730B480487F4D01782D78E3
S214012FB042788378C4780171427155FA81F11031F3
S214012FC089B28371C471FF29CCBF01250025017028
S214012FD055FA82F189B2FF29CCBF01220022417045
S214012FE052FA83F189B2FF29CCBF012200228170F7
S214012FF01119C17030BC70476C480178427851187D
S2140130008278C07851184018C0B2704762485E494D
S21401301083790A781B1883F8E22082794978521C52
S2140130208271D2B2121882F8E2108179491C81713C
S21401303090F8E310891C80F8E310704770B4544987
S214013040524B4A785C781D7802F0E7024A700020FD
S2140130504D494A780E7802F0E70204F0E7044A7018
S2140130605C70B54218BF0120944218BF0120494A3E
S2140130709B78897814788B420ABF002844F0800038
S21401308004F07F00107070BC704743498A7952186B
S21401309082F8E2008879401C8871704738B50C4682
S2140130A03D4D0146A87940192246E230F8F73AFD2F
S2140130B0A8792018A87131BD3748002180F87D1104
S2140130C0042180F82118704738490A7A4B7A42EA77
S2140130D00322504008224AF201034FEA500C00F046
S2140130E001000128ACBF83EA0C006046521EF4D1F1
S2140130F00872000A48727047F8B52C4CFF202072FF
S21401310060722220FFF7E0FF234DAE79E6B105F2AB
S214013110E20031464AF20102237A677A43EA07233C
S21401312007787B4008274FEA530C03F00103012B75
S214013130ACBF82EA0C0363467F1EF4D12372401CA7
S2140131401B0A6372491EE7D195F87C0180070BD5EF
S2140131502078FFF7B9FF6078FFF7B6FFA078FFF792
S214013160B3FFE078FFF7B0FF607A711981F8E200EB
S214013170A879217A401CA871C0B2401980F8E210E3
S214013180A879401CA871F1BD241EFF1F281EFF1F31
S214013190201EFF1F491EFF1F440BFF1F4C1AFF1F57
S2140131A08F19FF1F8C19FF1FF31DFF1FC41DFF1F63
S2140131B0F21DFF1F80B578B3012A04D02CD3032A51
S2140131C022D014D328E0002926D40161816909B1EF
S2140131D000218161816821F0080181600168CB6965
S2140131E0190002D0002207219847002002BD8369FA
S2140131F00269002B1CBF002A491E002902D54B423A
S2140132009A4209D38918E0E74269002902D54B4260
S2140132109A4201D38918D8E74FF0FF3002BD00006B
S214013220010040F10780F446404200F003F851F0F7
S2140132300041604709D0B0FA80F18840C91CC1F549
S2140132408461090501EBD0214005704790EA010F22
S21401325044BF81F0004101F0E3BE00BF431A4FF0C6
S21401326000423EBF5340C01AC91800BFD3095FEAE7
S214013270D05C13EB400F34BFB3EB410F40E07CEB67
S214013280D1530CD342EA012122D8D1EB402009D3F5
S214013290400A28BF5FEA500140EBCC507047401A05
S2140132A015D04002B0FA80F2521C9040400A4FEA14
S2140132B03C23B3EB026384BF00EB730007E040F4EA
S2140132C000001A16DB07C2F10102D040184370470E
S2140132D0182BFCDC31FA03F202FA03F3591A38BF51
S2140132E042F00102D2EB40203CBF4000ACF1010CA1
S2140132F05FEACC5CC20572F100414CEB502070478E
S21401330013EB400F0FD24B0009D0ACEBD153022B7D
S21401331003DB4902172BDDDD70479143401A43005A
S214013320D5D10020704713EB410FD0D36FF00000CA
S214013330704700001C48012101720021417241744E
S2140133404170418141824180C160416141600020FC
S21401335016490870164908707047134A8154801838
S214013360012101727047104A815470470E4A801835
S2140133700174704780B5F7F7FAFC0B4901F20902B0
S2140133800120491C1378012B06D10B7823B15B1E53
S2140133900B70DBB203B9FEE7401CC0B2491C521CDD
S2140133A00828EFDB01BD0000741DFF1F4A1EFF1F2A
S2140133B04B1EFF1FF7F7DBBCF7F7E3BC30B4016A1F
S2140133C021F040010162416A21F00B014162416A2C
S2140133D041F007014162416A41F0800141620168A2
S2140133E00906FCD5416A490648BF012024D4C16CB0
S2140133F0826C436C046CC56B511859186118826B4A
S214013400691851180904490C41F40041C162C16EA2
S214013410826E436E046EC56D511859186118826D1F
S214013420691851180904490C41F400410163416AC5
S21401343021F080014162002030BC70470A7882602A
S2140134404A78C2604A8882618A88C2618A79026241
S214013450CA794262CA6802650A7A0260497A41609C
S2140134607047F8B50446002600270D46FF2C88BF96
S214013470142605D8F9F787F850F8247040F8245038
S2140134803046F8F7B9FF3846F2BD00002DE9F041A5
S214013490DFF8448298F8000050B1FCF70FFC10B139
S2140134A0FEF789FF20B998F80000401E88F8000052
S2140134B08A4D687828B3E8782989C0EB0012B1EB09
S2140134C0820F06DBFF2804D0854E307800F0EF002F
S2140134D00DE0481C288180B2032812DB0020FEF78D
S2140134E0BCFE01280DD17E4E307840F010003070C1
S2140134F00020FDF72EF9307800F0FD003070002036
S2140135006870784E764C06F2C607B87900F0F70078
S214013510B87100F00300032815D196F8C60000F034
S214013520F70086F8C60000F0030003280BD1387BAD
S21401353000F0F700387300F00300032803D1207869
S21401354000F0DF0002E0207840F0200020704FF00D
S214013550030E96F8EA00E9882A7800F0F70086F864
S214013560EA0010EA0E0F237803F0080C0CD10021B4
S214013570BCF1000F1AD00A2A18DA521CD2B20A2A53
S21401358014D103F0F70010E00022BCF1000F0DD1BA
S2140135902879C0EB001C4FEA8C008842A2BF491C68
S2140135A089B2814202DB43F0080020702A70E9806C
S2140135B02078810717D4800800F00100FEF74DFE41
S2140135C00028A87806D108B1401E06E0207800F051
S2140135D0FB0007E01E2802DA401CA87003E02078F2
S2140135E040F004002070B87F00F0F700B87700F0D4
S2140135F00300217803280CBF01F07F0041F0800012
S214013600207098F800102078002914BF00F0BF0041
S21401361040F04000207096F8A40100F0F70086F80C
S214013620A40100F00300217802280CBF01F0FE007F
S21401363041F001002070BDE8F08138B5274CE070FC
S21401364048B1284890F8EA1001F0F70180F8EA102E
S214013650032001420ED0224D287800F0EF0028709A
S2140136600020FDF776F8287800F0FD00287000208D
S214013670607031BD1A4D287840F002002870FF2096
S21401368060700120FDF765F80020208131BD134AE6
S21401369012894FF4616392FBF3F303704FF4616098
S2140136A000FB13203C2290FBF2F0087070470B4998
S2140136B0087170470948407860B90A4890F8EA10DE
S2140136C001F0F70180F8EA1001F00301481E80417D
S2140136D0C00F704700207047481EFF1FE81DFF1FE0
S2140136E0201EFF1FDC17FF1F0DB400B50A4602ABF4
S2140136F00FF2110101A801F0E1FC019A00211170FD
S2140137005DF810FB0A68531C0B60107070470000D0
S21401371010B4664900228A600122CA60027C012A2E
S21401372004D03BD3032A2FD014D337E0604B0022BA
S2140137301A60027A0AB1022208E0C2682AB1521E51
S214013740C26080220272022200E0032202744FF459
S21401375016622AE0564A012313604468C3681B5D5B
S214013760047A23405C1EA441E40FD460037A5B080C
S2140137700372C468002C02BF102B01235360012280
S214013780027442F6E06210E0494A01231360002306
S2140137905360042202744FF4166206E0444A012381
S2140137A0D36013605360002202740A60007C08B183
S2140137B00320886010BC704780B53E483E4A0168C9
S2140137C041F40001016000203C49086000213748AF
S2140137D0016081600121C16054203949F8F7E0FE9B
S2140137E0BDE80840012202215420FBF7A5B8324863
S2140137F0017C481E8041C043C00F704798B12E4AD5
S21401380010705160401ED06080201072022010742B
S21401381001202749086001212448C1604FF4166140
S21401382001600321816070470278264902F0010297
S214013830531E9B41DB43DB0FCB61027802F0020291
S214013840531E9B41DB43DB0F8B61027802F00402BF
S214013850531E9B41DB43DB0F4B61027802F00802EB
S214013860531E9B41DB43DB0F0B61027802F0100213
S214013870531E9B41DB43DB0FCB60027802F0200234
S214013880531E9B41DB43DB0F8B60027802F0400244
S214013890531E9B41DB43DB0F4B60007800F080003A
S2140138A0421E9241D243D20F0A6070470071034014
S2140138B03010FE433C800440A01DFF1F00700340F3
S2140138C0113701002010FE437047000010B5544C1C
S2140138D00A202072F7F742FFA070F7F746FFE07064
S2140138E0F7F747FF2071E071A178E278617141F046
S2140138F02000A271607010BD4A49DFF824C191F81A
S2140139004D209CF801C0002002F03F03634509D01A
S214013910BF231A4207D14D31497809291CBF5229C4
S214013920572900D101207047F8B5F7F717FF04466D
S214013930F7F71BFF0546F7F71CFF39494E790A7A58
S214013940B44201BF8F79BD42CB79984233D182B35D
S214013950521ED2B26ABB8878B04201BFC878B8425C
S2140139600879984225D046F0200048708E70CF70B6
S2140139700B71002F2C48447814BF44F0200404F047
S214013980DF044470002B447814BF44F0400304F075
S214013990BF034370437843F01003437023484478D1
S2140139A004F08F04234343702148037843F08003D7
S2140139B003700A72F1BD4C718D71C8710A22F8E765
S2140139C01748007970471648017801290CBF102165
S2140139D000214078401E00F00F0040F080000818DB
S2140139E0C0B270470E49C978102001B12020704737
S2140139F00B4A0D48D2784178002A14BF41F02001C5
S214013A0001F0DF0141707047054A07481279417895
S214013A10002A14BF41F0400101F0BF014170704718
S214013A20F21DFF1F440BFF1F201EFF1F241EFF1F3A
S214013A30491EFF1F10B540F628012E4A11FB00242F
S214013A4096234FF4806204F5C27104F10C0002F073
S214013A500DF804F2845104F12C00BDE810409623C1
S214013A604FF4FA7202F002B838B50446214D01202F
S214013A7085F82608FFF720FB40F6280111FB0451C4
S214013A80052081F81F08BDE8314002F04BB910B59A
S214013A90184C94F81F0848B1401E84F81F08C0B29D
S214013AA020B9FDF77FFA002084F8260810BD8AB2F7
S214013AB00146114802F0AFB810B50C4601460E4853
S214013AC002F07EF8002848BF00202060C0B210BD7A
S214013AD0094802F0CFB88AB20146084802F09BB8FE
S214013AE080B50146054802F040F8002848BF00208E
S214013AF0C0B202BD440BFF1F500BFF1F700BFF1F10
S214013B0030B4C148C149C24AC24B0824002500F856
S214013B10015B032501F8015B02F8015B03F8015B19
S214013B20002500F8015B032501F8015B02F8015B43
S214013B3003F8015B002500F8015B032501F8015B32
S214013B4002F8015B03F8015B002500F8015B032521
S214013B5001F8015B02F8015B03F8015B641ED5D135
S214013B6030BC70472DE9F047FFF73CFF8046002543
S214013B70A84EA54FA84CDFF8A49220784FF0000A73
S214013B8001071BD510F0030006D0012806D0032834
S214013B900CBF0620032002E0052000E00220317859
S214013BA001F0F80108433070F7F7C6F8207800F006
S214013BB0F7002070F7F7C4F84FF0010A454514DA0C
S214013BC0307800F00701A8B200F018F8BAF1000F3B
S214013BD00BD03878002802BF307800F007000328A1
S214013BE003D099F80000800038706D1C7F1C761C8D
S214013BF004F20604202DC0DBBDE8F08770B505464B
S214013C00824E0C46A95D0A060BD501F00701022972
S214013C1003D0032939D1022C03D0062C18BF052C5A
S214013C2033D1C0B27849425C805D00F007000228BB
S214013C300ED0032804D0052812D006280DD070BD5A
S214013C401ABB062C18BF052C12D0022C1DD10FE072
S214013C50062C0DD0052C07D10AE0052C02D107E071
S214013C60062C05D0022C03D0032C08BF002A0CD149
S214013C70F7F762F8A85D00F0F800204340F08000F6
S214013C80A855BDE87040F7F75BB870BDF8B50026DB
S214013C90FFF7A8FE0446FFF7A5FE5C4D00212A4665
S214013CA000E0491CC9B2814225DA12F8013B1B0625
S214013CB0F7D5574E2021304602F04AF84120FFF74B
S214013CC0E4F90020FFF7E1F90027012C12DB287840
S214013CD001060AD507F01F0141EA4010C0B2FFF7FE
S214013CE0D4F928783070FFF79AF87F1C761C6D1C83
S214013CF0A742ECDB01263046F2BD10B5FFF772FE97
S214013D0001280CDB4249414A13780C789C4204BFD7
S214013D1003F07F031370521C491C401EF4D110BDE2
S214013D202DE9F041FFF75EFE80460025B8F1010F50
S214013D301DDB354E354F374C307890B1401E307014
S214013D40C0B270B9387801060BD4217801F00702A9
S214013D5000F00700824204D001F00701E8B2FFF745
S214013D604DFF6D1C641C7F1C761C4545E4DBBDE8DD
S214013D70F0812DE9FC4100A80021002206C0FFF7D2
S214013D8031FE0646700806EB90708405240E44202A
S214013D90FFF77BF90020FFF778F90020012E25DBDD
S214013DA01A4900AA0B7803F00703022B09D0032B4C
S214013DB009D0052B03D0062B06D1002504E00125EA
S214013DC002E0022500E00325471000EB9777BF10BD
S214013DD000F00308BB5C4FEA480805FA08FE4EEA05
S214013DE00303BB54401C491CB042DBDB012C08DB3F
S214013DF000AD15F8010BFFF748F9FFF710F8641E40
S214013E00F7D1BDE8F3810000341DFF1FF41CFF1F2E
S214013E10141DFF1FD41CFF1FDC17FF1F441EFF1FAE
S214013E2038B50546D9B12878DFF8BC47512805D101
S214013E3000206070A070207000F06DFB287850287C
S214013E400BD1A878DFF8A41708702078062804D2CA
S214013E500FF2E07151F820008047F020207131BD4B
S214013E6010B5DFF88407DFF888470021417001703C
S214013E70817001710122D1A1A01CFFF735FC81B22E
S214013E80204600F09AFB02F091F800281CBFBDE81E
S214013E90104002F02EB810BD80B5DFF85807007844
S214013EA0002802BFDFF8440700783A282CD000210A
S214013EB0052002F0DDF8012802D002280BD001BD52
S214013EC0DFF824078178491C8170C9B2062924D3FA
S214013ED00021817021E0DFF820070188002904BF56
S214013EE0BDE80140FFF7BCBFDFF8FC060022017009
S214013EF042700178062913D281700FF2387050F89B
S214013F002100BDE802400047DFF8DC06817809B9E8
S214013F10062181708178491E8170BDE80140FAE270
S214013F2001BD000070B5DFF8C0466078072800F2D2
S214013F30E380DFE800F03E043E425E92D5DB0021DE
S214013F400A2002F095F8012802D0022804D070BD9C
S214013F5000F0FFF80320C7E0DFF89C06DFF89C5668
S214013F6000882978C2B291421CBF287002F018F866
S214013F702978072000F024F900281CBFBDE870400E
S214013F8000F0F2B81B2002F013F9064628780FF26B
S214013F907C620B2102F018F9DFF8545602463146CE
S214013FA0A81CFFF7A1FB81B2284600F006FB022001
S214013FB09AE000F0D9F8012096E000210F2002F0E7
S214013FC057F8012802D0022804D070BD00F0B1F8DD
S214013FD0042089E0DFF82006DFF8241600880A7836
S214013FE0C3B29A421CBF087001F0DAFFBDE8704008
S214013FF0AFE00021012002F03BF8012802D00228A0
S2140140001CD070BD00206071182002F0D1F8064661
S214014010DFF8F0050078C0074CBF19201A2002F01F
S214014020C7F80346DFF8C85501223146A81CFFF73A
S2140140305BFB81B2284600F0C0FA54E0DFF8B80511
S214014040DFF8C41500880A78C3B29A421CBF08700C
S21401405001F0A6FFBDE870406BE0DFF89005007840
S21401406030283AD03A2802D03B2829D070BD607952
S2140140700125032808DADFF88C150A7805FA00F01E
S2140140805040087001F08CFFDFF87005017894F954
S214014090050005FA00F0C0B200F092F808B16079A8
S2140140A018E01C2002F084F8DFF844550146A81CED
S2140140B0FFF71AFB81B2284600F07FFA062013E0CC
S2140140C0FFF790FC102808D06079401C6071C0B2E0
S2140140D0032802DABDE8704056E0BDE870400CE007
S2140140E0607900F051F80520607070BDDFF8FC04BF
S2140140F000783B2800D154E170BD38B5DFF8FC04E8
S214014100DFF8E4440178072000F05AF808B10020EF
S214014110FDE11D2002F04CF80146DFF8D454A81C3E
S214014120FFF7E2FA81B2284600F047FA07206070EE
S21401413031BD70B5DFF8D0442078022808D21620A9
S21401414002F036F8054620780FF2D8420221A4E0A4
S21401415070BD10B5172002F02BF8DFF8A414DFF8B5
S21401416090440A780146F5E170B5DFF8904420786E
S2140141700B2808D2132002F01BF8054620780FF210
S2140141808C420B2189E070BD70B506463446032C7F
S21401419013DA182002F00CF80546DFF868040078F8
S2140141A00121B140084214BF19201A2002F000F87C
S2140141B00346DFF83C64621C75E070BD25630000B1
S2140141C070B504460D460126FFF70CFC102808BF03
S2140141D004F00104DFF82C040078204205D0072DF6
S2140141E01CBF082D092D00D10026304670BD30B504
S2140141F087B01E2001F0DCFF0446062105A8FCF767
S214014200F4FB062103A8FCF718FC062101A8FCF71D
S214014210F8FB03A8009001ABDFF8D45305AA2146AA
S214014220A81CFFF761FA81B2284600F0C6F907B06C
S21401423030BD10B5DFF8B043607810B1012806D064
S21401424010BDFFF7D4FF6078401C607010BDDFF82A
S2140142509C0300783A2802D03B2803D010BDBDE865
S2140142601040C4E7002060702070BDE8104052E1A5
S21401427070B50446202001F09BFF0546601E002114
S214014280C0B2FEF710F8DFF86863034622462946F7
S214014290B01CFFF729FA01460AE001F095FFDFF8A6
S2140142A05063227803462946B01CFFF71DFA81B2F7
S2140142B03046BDE8704080E138B50446212001F063
S2140142C077FF0546601E0221C0B2FDF7ECFFC84C21
S2140142D002462946A01CFFF707FA014620462EE1B2
S2140142E070B5FFF77FFBC04C617819B1022943D046
S2140142F00FD370BD1F2001F05BFFBD4D0146A81C0A
S214014300FFF7F2F981B2284600F057F90020E07075
S21401431029E0B64909783A2902BFB6490978002941
S21401432003D1E17809B1084623E0002101F0A0FE9F
S214014330012834D0022833D1AF480088B8B901200B
S214014340E070212001F034FF064602210020FDF72F
S214014350AAFF0246A64D3146A81CFFF7C5F901463D
S214014360284600F02AF96078401C607070BDE07045
S214014370E078BDE870407BE79C4909783A2902D08D
S2140143803B2902D070BDE07806E0E178091DE170B6
S214014390C9B2884203D30846BDE870408CE700E006
S2140143A070BD002060702070BDE87040B3E02DE95C
S2140143B0F8438D4C607830B1022849D013D30328D6
S2140143C068D0BDE8F1838A4D9121A81C00F0E4FD78
S2140143D00646C6F191017019C9B2801C00F09CFD19
S2140143E056FA80F04AE0222001F0E2FE064623203B
S2140143F001F0DEFE8046FCF7B3FEC7B23046FCF79E
S214014400AFFE5FFA80F97A4D4A463146A81CF7F7A7
S21401441089FBC9F1910109EB0500C9B2801C00F0C6
S21401442087FD4844C6B2C6F19100874207DA701983
S2140144303A464146801CF7F775FBBE19F6B2C6F13F
S21401444091017019C9B2801C00F082FD801914E038
S214014450242001F0ADFE0646FCF782FEC7B2644D8D
S2140144603A463146A81CF7F75DFBC7F1910178196A
S214014470C9B2801C00F0A6FDC019C0B25321297034
S2140144806870811C2846FFF712FB6078401C60703C
S214014490BDE8F183002060702070BDE8F1433AE08A
S2140144A038B5514C607818B102282DD002D331BDF1
S2140144B0252013E04D4800783A2821D0002142F209
S2140144C00F7001F0D5FD01281ED002281ED14A48E2
S2140144D00088012818D101F055FD262001F068FE5C
S2140144E0434D0146A81CFCF757FEA81CFCF738FEF6
S2140144F00146284600F061F86078401C607031BDC6
S21401450000203C49087000E0002000E031BD6070EA
S2140145102070BDE8314038B5072001F049FE044659
S21401452031480FF204128078062101F04DFE304D1D
S21401453002462146A81CFFF7D7F881B22846BDE8F7
S21401454034403AE010B52A4C012202E010B5284C5E
S214014550024623A1A01CFFF7C7F881B22046BDE89A
S21401456010402AE018B401460B291DDA0222204821
S21401457049B1831C5C2403F8014B921C382403F8D0
S214014580014B491EF6D1D2B25C211154511CC9B25D
S21401459032220A54491CC9B25322891E0270417044
S2140145A0891C14BCFFF783BA11BC704710B5104CB8
S2140145B00CA1A01CFFF798F8CFE7532202704170B8
S2140145C0891CFFF774BA0848017931B1491E017197
S2140145D0C9B2002908BFFFF743BC704700000000BE
S2140145E0256300005C3800000C1EFF1FBD1DFF1F69
S2140145F0E41AFF1FBF1DFF1FC21DFF1F451EFF1F21
S214014600441EFF1F471EFF1F461EFF1F080009000E
S2140146100A000B000C000D000E000F001000110028
S214014620120000001400150001000200030004003F
S21401463005000600993E0100253F010033420100B6
S214014640E1420100AF430100A1440100C378012209
S21401465093B1007974280FD10870042048702A4855
S2140146600078887029480078C87029480078087151
S21401467028480078487100E0062210467047F8B5D1
S21401468004460026E578032D36DB27790B20C04645
S214014690874207DA1C4801788F4204D0077001F080
S2140146A07FFC00E004266079102807DA17490A78AB
S2140146B0904204D0087001F073FC00E00426A7794C
S2140146C00220C046874207DA114801788F4204D09B
S2140146D0077001F065FC00E00426042D0DDBE0798F
S2140146E000F007070B4801788F4203D0077001F0EE
S2140146F057FC02E0042600E0062601F057FC08B14C
S21401470001F0F7FB3046F2BD451EFF1F441EFF1F9A
S214014710461EFF1F471EFF1FDFF8D807002180F83F
S2140147207A11017080F8751180F8741100F5D47053
S21401473001F062BD70B5DFF8BC472078002582B075
S214014740102800F24B81DFE810F011004901190032
S21401475049011B005B0080004901490149014901EB
S214014760A90049014901BE00FF00170100F05FFBE7
S21401477010B900F0A0FB2FE10E202EE103202CE162
S21401478094F87A014FF440563146022808BF4FF498
S2140147907E21FA23621C0020FBF777FB102204F12E
S2140147A0110104F5B070F7F7BDF90C2204F15901B7
S2140147B004F5CE70F7F7B6F994F87A01022808BF27
S2140147C04FF47E2606F12100C4F80001C4F87051AA
S2140147D094F8270094F8281000EB012094F829108B
S2140147E000EB014094F82A1000EB01602138C4F870
S2140147F05C010520207004F5827001F010FDEDE0EB
S214014800D4F800114023621C0020FBF73EFBD4F8CD
S2140148100001D4F85C114030C4F8000104F582723E
S214014820D4F87001091A412907D34030C4F8700141
S2140148304021601C01F0F7FCD0E00818C4F87001B4
S214014840601C01F0F0FC0620C7E004F5B07104F529
S214014850827001F038FD08B90720BEE094F87A01AD
S21401486084F875510C2204F5CE71012809D1022075
S21401487084F8780104F5C270F7F764F984F87B517F
S21401488008E0022084F8790104F5C870F7F75AF9B0
S21401489084F87C5100F0D6F808209EE094F87A015E
S2140148A0012805D1032084F8780184F87B5107E0BC
S2140148B0022084F87A0184F87C51032084F8790177
S2140148C000F0C0F8FEE7112500F0B1FA94F87A017D
S2140148D0012817D194F87901052808BF132594F803
S2140148E07811032926D1042184F87811022184F84D
S2140148F07A1102281CBF032804281BD1012084F842
S214014900790117E0022815D194F87801052808BF27
S214014910132594F8791103290CD1042184F879110F
S214014920012184F87A1102281CBF0328042801D12A
S21401493084F8781194F87D0110B1032084F87D0184
S21401494000F080F8257015E000F071FA8DF800503F
S21401495000A800F045F818B184F87D5100F072F80F
S21401496094F9740110F1060F16BF10F1020F122010
S21401497001202070022531E000F059FA94F87A01FE
S21401498001280DD194F87801012804BF94F8790123
S214014990022821D1052084F8790104F5C8700DE0BC
S2140149A0022801BF94F87801022894F879010128B9
S2140149B012D1052084F8780104F5C27000210A4658
S2140149C00B460EC094F87D01012812BF0328022071
S2140149D084F87D010B2000E001202070284676BD7A
S2140149E0DFF8102510B402F5BC7300219C78012C69
S2140149F012D192F87841032C21D1042182F8781142
S214014A00022201219A700170587802281CBF0328DF
S214014A10042814D1597012E0022C04BF5C78032CD0
S214014A200DD10421597001219970017092F8780115
S214014A3002281CBF0328042801D182F8781110BC73
S214014A400846704770B5DFF8AC4414E20000000079
S214014A502DE9F0470C4651212170002581787D29EA
S214014A6008BF801CC678C02E80F29081021D117886
S214014A70891F112900F28A81DFE811F012004B002C
S214014A809300880188018801B200C1009800CD001A
S214014A90E90036014C0162016C0175010701310123
S214014AA0DFF8507497F87A010022012809D187F8B7
S214014AB078210C2107F5C270F7F7E2FC87F87B51E5
S214014AC008E087F879210C2107F5C870F7F7D8FCBC
S214014AD087F87C51FFF7B6FF01210020FBF7C7F9E5
S214014AE097F87A014FF440542146022808BF4FF444
S214014AF07E210020FBF7CCFA02203870A7F8FC5084
S214014B0097F87A01022808BF4FF47E24C7F80041BF
S214014B103CE1DFF8E0733878032838D1B7F8FC00B9
S214014B2000F10109501C00F10208427801781202D6
S214014B3052FA81FA1FFA8AFABAF1010F0AD197F8E6
S214014B407A014FF44051022808BF4FF47E2100201D
S214014B50FBF7C4F91FFA89F0824509D0512020706D
S214014B60032060700D20A070FD20E07025710CE11F
S214014B70F21EA7F8FCA092B241460020FBF7EBF923
S214014B80D7F80001F11E0818C7F80001FEE0512011
S214014B902070032060700D20A070FC20E07025714D
S214014BA0F3E00420DFF84C130870EFE0DFF84473FD
S214014BB097F87A0101280DD197F8780102280DD0CF
S214014BC051202070032060700D20A070F920E07045
S214014BD02571DAE097F879010228F1D10B2034E04B
S214014BE0C44F97F87A014FF44051022808BF4FF49A
S214014BF07E2116237A1C0020FBF747F9C6E0BD4844
S214014C00007851212170032161700D21A1700321CB
S214014C10E1702071B9E0B74F97F87A01012809D100
S214014C2097F87801012804BF97F87901022840F027
S214014C30AD8009E0022801BF97F87901012897F8AD
S214014C407801022840F0A280102038709EE05120A2
S214014C5020701B2060701020A0700C22A54F07F555
S214014C60C271E01CF6F75EFF0C2207F5C87104F16D
S214014C700F00F6F757FF97F87A01012818BF0020B2
S214014C80E07601250120207780E00020994F97F8F3
S214014C9078210146032A08BF012105D097F879211A
S214014CA0032A04BF012001215122227009226270C9
S214014CB01622A270E070217197F87D01607197F855
S214014CC07A01A07197F87801E07197F8790120725E
S214014CD097F87B01607297F87C01A07255E0214637
S214014CE000F057F8054651E051202070B1211120FF
S214014CF0A070201D00F066F9E070051DEDB2C5F14B
S214014D00B4012819C9B2401C00F068F928554019A9
S214014D10401E39E051202070B1211220A070201DC4
S214014D2000F0FAF8E070051DEDB2C5F1B4012819DE
S214014D30C9B2401C00F01EF928554019401E23E058
S214014D406D4805682846FCF70BFA06465120207088
S214014D50132010E0694D2846FCF702FA064651205A
S214014D602070142007E0664D2846FCF7F9F9064640
S214014D70512020701520A070F6B232462946201D1B
S214014D80F6F7D0FEE670B01C607001252846BDE837
S214014D90F08710B58279C379017A4079A6280CD1BB
S214014DA000F089F84FF440510020FBF771F94FF4F9
S214014DB07E210020FBF76CF937E00020ABB9002A12
S214014DC002BF4C4B93F87841032C03D1012083F8A2
S214014DD0780122E0012A01BF464B03F5BC725378E5
S214014DE0032B1AD10120507017E0012B15D1002A90
S214014DF002BF404B93F87841012C03D1032083F87E
S214014E00780109E0012A01BF3A4B03F5BC725378D9
S214014E10012B02D1032050700120052902DA3948FE
S214014E20417100E008B1FFF70DFE002010BD30B55E
S214014E3083B04FF48050019000244FF4005000904E
S214014E40029401232B4D0FF2C800FA22691CFBF7CE
S214014E50B7FA68B901242422A91C05F5BC70F6F737
S214014E6061FE95F87A0101281CBF022885F87A416F
S214014E70204603B030BD04F5D475284601F0BFF9CD
S214014E800020FAF7FBFF064605230FF27C024FF4DB
S214014E9000510020FBF71BFA242204F5BC71002008
S214014EA0FBF750FAF1B20020FAF7E1FF2846BDE819
S214014EB0704001F0B2B9F8B50E4D05F5BC7401208D
S214014EC0A0700C26002085F878010246002731469E
S214014ED005F5C270F7F7D4FA67703A46314605F51C
S214014EE0C870F7F7CDFAA760E770A780FFF7AAFDAD
S214014EF00120F2BD0016FF1FCC06FF1F9C06FF1FF8
S214014F00A806FF1F7817FF1F46575F55470000008A
S214014F105B66773D00000000F8B50446144E0D466A
S214014F203046FCF71DF90746BD42B8BF2F4642E0A2
S214014F30F8B504460E4E0D4606F18000FCF710F952
S214014F400746BD42B8BF2F463A4606F1800134E017
S214014F50F8B50446064E0D4606F58070FCF700F9D6
S214014F600746BD42B8BF2F463A4606F5807124E093
S214014F7020A4000070B504460D46FFF7D9FF202196
S214014F800155461CA91BF0B2C9B20019FFF7E0FF94
S214014F908019C0B270BD0000F8B50446004801E0B3
S214014FA00C09FF1F06680D463046FCF7D9F8074680
S214014FB0BD42B8BF2F463A4631462046F6F7B2FD07
S214014FC0F8B2F2BD10B50C240C29B8BF0C46224627
S214014FD04FF48461F6F7A6FD204610BDBCB50D461C
S214014FE004464FF494610C2D15DB08270B22F6F7C7
S214014FF099FD2020E072142DBCBFA5F10C07FFB26D
S2140150003A464FF4A46104F10C00F6F78BFD07F164
S2140150100C05EDB202E02A46F6F784FD2846B6BD39
S214015020421A3CBF801A89184FF0004CC0F3C75291
S214015030FF2A24D0C1F3C75313B3D21AD2F11903EE
S21401504027DD4CEA01214CFA03F321EA0303D140A0
S214015050C20D4CEA0020401834BF20EA0C004CEA8E
S2140150605000D20553EA006373EB0C0C52EB102090
S214015070420012F1807F38BF7047C00DC0057047EF
S214015080490212BF9A4200EB5120F8E7D2F117030A
S214015090D9D57047F8B504460D461646002701E0F7
S2140150A07F1C761C307820B12146A8473178814292
S2140150B0F6D0307800B17F1E3846F2BD2DE9F14FAB
S2140150C096B000208B4614469A460D90814604E021
S2140150D01699D8470D9009F1010914F8010B2528F6
S2140150E00AD00028F4D10D9810F1010F02D14FF02B
S2140150F0FF30BFE34846BDE32078252803D1169943
S21401510014F8010BE5E720208DF8080000260C9620
S2140151108DF8096006960A96059600230B96374683
S21401512002E001200C90641C2078B0B120280DD03C
S21401513023280FD02B2807D02D28F2D0302808BFDF
S2140151408DF80800EFD008E00123ECE701208DF888
S2140151500900E8E701200690E5E7049720782A2869
S2140151600DD15AF8040B0490641C0CE0049800EB73
S2140151708001480014F8011B40183038049020784C
S21401518030380A28F2D3019720782E2815D114F842
S214015190010F2A280DD15AF8040B0190641C0CE06B
S2140151A0019800EB8001480014F8011B40183038C4
S2140151B00190207830380A28F2D30EA8079014F808
S2140151C001EBBEF1000F08D116992520D84710F142
S2140151D0010F8CD009F101004CE36D22BEF1680F7E
S2140151E018BFBEF16C0F05D0BEF14C0F18BFBEF153
S2140151F06D0F02D1724614F801EB00210D46704680
S214015200BC46039543282AD0442818BF49283BD0DA
S2140152104E2800F04D814F2800F0D880502800F02D
S2140152200781532828D055282FD0582800F0088108
S214015230632814D0642818BF692825D06E2800F08A
S21401524037816F2800F0C280702800F0F380732841
S21401525012D0752819D0782800F0F6802EE15AF879
S214015260040B8DF838009DF8380008B9012003902A
S2140152708DF83910019102E05AF8040B07902020AE
S2140152808DF80800069123E10121BEF1750F12BFCA
S214015290BEF1550F01200B9001980128A4BF0120F3
S2140152A00A9091B34C2A17D10AF1070020F0070A99
S2140152B0FAE80201CDE90801002908BF002802D159
S2140152C00127B3B91CE00029FBDA2D26404261EB29
S2140152D04101CDE9080134E0682A06BF0AF1040A53
S2140152E03AF9048C5AF8048BB8F1000F03D1012760
S2140152F033B12B2625E0FBD52D26C8F1000820E08A
S2140153009DF80900E8B120261BE0682A04D10AF1BD
S214015310040A3AF8048C10E06C2A0CD04C2A0AD104
S2140153200AF1070020F0070AFAE80201CDE90801B0
S21401533039B9002803E05AF8048BB8F1000F08BF0A
S21401534001274C2A17D0B8F1000F06D5DFF818054B
S21401535080446D1CB8F1000FF8D400230A220EA970
S214015360404600F08AFA9DF8380028188DF8380073
S21401537000200690ACE0DDE9080100290CDADDE941
S2140153800823DFF8E804DFF8E81410185941CDE9DE
S21401539008016D1C0029F2DBDDE90801CDF800C02B
S2140153A014230DF1390200F0D2FA9DF839002818BD
S2140153B08DF83900C0B23A2804DB0A388DF8390076
S2140153C03120D3E70DF139000790D1E701200B908A
S2140153D001980128A4BF01200A904C2A13D10AF192
S2140153E0070020F0070AFAE80201CDE908010029C2
S2140153F004BF002801270095DDE9080116230EAA3F
S21401540000F0A5FA11E0682A06BF0AF1040A3AF983
S214015410048C5AF8048BB8F1000F08BF012700234B
S2140154200B220EA9404600F028FA032005904FE013
S2140154304FF0010C63465AF8040B08220EA934E01B
S2140154404FF0010CCDF814C0012101980B910128F1
S214015450A8BF0A910598411CC9B205914C2A14D1DE
S2140154600AF1070020F0070AFAE80201CDE908016F
S214015470002904BF00280127DDE90801CDF800C096
S21401548010230EAA00F063FA22E0682A06BF0AF18A
S214015490040A3AF8048C5AF8048BB8F1000F08BFD6
S2140154A00127634608220EA9404600F0E6F90FE000
S2140154B05AF8040B0790C0F800900EE61699D847E4
S2140154C010F1010F7FF486AE11E60398401C03909D
S2140154D003980799405C0028F7D10498002844BF38
S2140154E0002004900198002844BF002001900198F4
S2140154F004990025084321D00A980028019847D12D
S21401550040B10399884205DA07980EA9884238D037
S21401551001980390049808B10399451A06B16D1EC7
S214015520069887F00101C0B2084204D005986D1EA6
S2140155300328B8BF6D1E002D48BF00250B999DF8A6
S214015540090081F0010108421CBF2B2E2D2E0AD026
S2140155500020009020201699D847202804BF01205B
S2140155600090009881440C98002840F002810A9827
S214015570002876D00295002000900298002823D5B6
S2140155802BE003980199401A079940180790BFE746
S2140155908842C3DA0398019988420498A8BF039900
S2140155A0451A069880F001003843C0B2002804BFAF
S2140155B005980328B2D1039801998842AEDA6D1C8A
S2140155C0ACE70098401C009000980299884204DAE3
S2140155D016992020D8472028F3D0009881442B2EF6
S2140155E018BF2D2E0AD10020009030461699D847B4
S2140155F0864204BF0120009000988144069887F0F7
S2140156000101C0B208421BD00598012802D0022829
S21401561002D008E092A200E092A216985946FFF73F
S21401562039FD81440CE001980399401A012807DAF4
S214015630169900273020D847302808BF0127B944DB
S21401564001980399471A0026002F01D5E4E0761C3D
S214015650BE4280F2E18016993020D8473028F6D035
S214015660DAE09DF80800019030283DD12B2E18BFB6
S2140156702D2E0AD10020009030461699D847864232
S21401568004BF0120009000988144069887F001012C
S214015690C0B2084218D00598012802D0022802D0CC
S2140156A008E06FA200E06FA216985946FFF7F2FCD9
S2140156B0814409E0012D07DA169900273020D847E2
S2140156C0302808BF0127B94400270095002D01D5D1
S2140156D04DE07F1C0098874249DA019E16993046B4
S2140156E0D8478642F5D042E0039500200290039801
S2140156F0002803D50EE00298401C029002980399F8
S214015700884207DA0198169900900198D8470099BF
S2140157108142F0D0029881442B2E18BF2D2E0AD13B
S2140157200020009030461699D847864204BF0120D3
S214015730009000988144069887F00101C0B20842A3
S2140157406BD00598012802D0022802D008E044A2B6
S21401575000E044A216985946FFF79CFC81445CE0A1
S214015760169900273020D847302808BF0127B944AA
S21401577053E02B2E18BF2D2E0AD100200090304664
S2140157801699D847864204BF0120009000988144AC
S214015790069887F00101C0B208420BD0059801288F
S2140157A002D002280FD010E02DA216985946FFF716
S2140157B071FC81440A9880B301980399471A002620
S2140157C0002F22D528E027A2EFE70A9860B10198BA
S2140157D00399401A0128EFDA16993020D847302865
S2140157E0EAD109F10109E7E79DF80800302803D15D
S2140157F0012D12DA169901E016993020D847302883
S2140158000BD109F1010908E0761CBE4204DA1699AB
S2140158103020D8473028F7D0B144079E002701E052
S2140158207F1C761C307820B11699D8473178814292
S214015830F6D0307800B17F1E0C98B94400283FF4AA
S2140158404CAC0027002D01D507E07F1CAF4204DADF
S21401585016992020D8472028F7D0B9443DE4000007
S2140158603078000030580000003665C400009C58AF
S2140158704C491FF217B0BDE8F08FF0B484B0002495
S2140158808DF800400B2A1BD100AB00F00704303422
S2140158905C70C0100DF10204052500F007063036D5
S2140158A004F8016BC01000F007063036C01004F88B
S2140158B0016B6D1EF1D1D87A00F03300D87232E058
S2140158C00A2A19D10DF1010305240A2590FBF5F5E5
S2140158D005EB8507A0EB4700303003F8010B0A20E3
S2140158E095FBF0F000EB8007A5EB4705303503F894
S2140158F0015B641EE9D116E00124012A13DB0DF1D8
S21401590001050FF254160FF23C1700F00F0C002B96
S21401591014BF1CF807C01CF806C00011641C05F86B
S21401592001CBA242F1DA00A8101800E0521E10F8CE
S2140159300139302BFAD02AB9012200A8105C01F8EF
S214015940010B521E002AF8D504B0F0BC70472DE9B1
S214015950F04388B004461E4600200D4691468DF859
S2140159600000162E1CD10DF101000B2104F00702D8
S214015970303200F8012BE40844EA457404F00702CB
S214015980ED10E40844EA45743032ED1000F8012BBE
S214015990491EEBD100A8817D01F0310181753DE002
S2140159A0142E20D10DF101080A27204629460A2285
S2140159B00023FCF759FD00EB8003A4EB43023032D1
S2140159C008F8012B04460A220023FCF74DFD00EBE4
S2140159D08003A4EB4302303208F8012B04460D463F
S2140159E07F1EE2D11AE00121012E17DB0F980FF27C
S2140159F068030FF250070DF1010204F00F0C0028A6
S214015A0014BF1CF807C01CF803C0240944EA057437
S214015A102D11491C02F801CB8E42EEDA00A830188F
S214015A2000E0761E10F801193029FAD02EB90126A9
S214015A3000A8305C09F8010B761E002EF8D508B0D8
S214015A40BDE8F083303132333435363738394142A8
S214015A504344454600000000303132333435363792
S214015A603839616263646566000000000382016084
S214015A708160C1605118491E416070478168C068E5
S214015A80814202D14FF0FF30704700207047826894
S214015A90C3689A4207D3D0F804C00068ACEB000094
S214015AA0D21A801A01E0981A401E884201DB0020B3
S214015AB070476FF001007047C26883684FF0FF318E
S214015AC0934206D01178531C42689A4238BF036845
S214015AD0C3600846704770B48368C268934205D3B2
S214015AE045680668AD1B9A1AAA1A01E0D21A521E18
S214015AF0012A0ADB1970002241685C1CA14238BFEA
S214015B000468846070BC104670476FF00102F9E7C4
S214015B10C268891842688A4204D20368D21A521CA3
S214015B2052425118C16070478168C2688C469142E2
S214015B3028BFACEB020005D241680068081A401C79
S214015B40801A604480B270478168C2688C46914270
S214015B5006D341680068081AA0EB0C00101802E092
S214015B60A2EB0C00401E80B27047F8B504460D4605
S214015B7000F0ACF80646012E1ADBE068811C60686E
S214015B80884204D22268821A521C52425118401A84
S214015B90471CB74202DB3246284606E03A4628460C
S214015BA0F5F7C0FF2168F21B7819F5F7BBFF02E095
S214015BB016F1030F02D1204600F05CF83046F2BD24
S214015BC0F8B504460D4600F081F80646012E1ADBAC
S214015BD0E068811C6068884204D22268821A521CDE
S214015BE052425118401A471CB74202DB3246284639
S214015BF006E03A462846F5F795FF2168F21B781924
S214015C00F5F790FF05E016F1030F04BF204600F0FC
S214015C1031F83046F2BD2DE9FC410E461746B91C57
S214015C20044689B2FFF733FF5FEA000821D107B3C4
S214015C303946204600F061F86168091A4D1CBD42DC
S214015C4002DB3A46314606E02A463146F5F76AFF58
S214015C5020687A1BA919F5F765FFA06861683818EE
S214015C60801C814204D22268891A491C49420818BC
S214015C70A06053E0C26883684FF0FF31934209D0B9
S214015C80436811789A4212BF537803681B7801EB78
S214015C90032189B2038A8B42B8BF6FF0020112DB7F
S214015CA000290DD48A184368921C934206D2D0F874
S214015CB000C0A3EB0C035B1C5B429A18C26003E0B6
S214015CC011F1030F00D1826008467047C2688368ED
S214015CD04FF0FF31934209D0436811789A4212BFC0
S214015CE052780268127801EB022189B2008A884252
S214015CF0B8BF6FF00201084670478368D0F804C049
S214015D0019700A0A634504D081684A708068801C4D
S214015D10704701680A700068401C70474046BDE83D
S214015D20F681000000BF08490A200870704706483F
S214015D30017831B1491E0170C9B211B90348017029
S214015D404170704700000000FB1DFF1F161EFF1F5D
S214015D500022F6F799BB00002DE9F84F0A9C804611
S214015D608A4693461F46002505EB4500BB4901EBD5
S214015D70C0063046FBF7F4F9C0B2824545D152461B
S214015D803146404600F0C2FA00283ED1BBF1070F6B
S214015D903BD8DFE80BF004040D0D1A1A2D2DB0794F
S214015DA0012818BF002830D1F1683878087029E03A
S214015DB0B079032818BF022827D1797838780902E4
S214015DC051FA80F0F16808801CE0B079052818BF08
S214015DD004281AD179783878090251FA80F0B9780E
S214015DE000EB0140F97800EB0160F168086009E01A
S214015DF0B079072818BF062807D1F0682246394629
S214015E00F5F790FE0120F07104256D1C042DABD32F
S214015E10BDE8F18F70B5924C924E0425607820BB98
S214015E202078072821D8DFE800F004040A0A1010B9
S214015E301616D4F80610D4F80E00087012E0D4F83E
S214015E400610D4F80E0008800CE0D4F80610D4F83A
S214015E500E00086006E0A27AD4F80E10D4F8060008
S214015E60F5F760FE01206070307018346D1ED5D1D4
S214015E7070BD00B579480021C171002200F207010A
S214015E8080F8372000F237004A700A764A76427068
S214015E900276427687B04FF48051002000F064FB12
S214015EA007210FF2C41000F064FBC8B90AE09DF8A0
S214015EB00400029B9DF805209DF80610009003A89B
S214015EC0FFF74AFF01A8009002AB0DF105020DF1A4
S214015ED0060103A800F071FB0028E8D00128F1D1E3
S214015EE0FFF798FF5F48007808B100F002F807B0A6
S214015EF000BD38B54FF48051002000F035FB072176
S214015F000FF2641000F060FB544C2046FBF728F9B2
S214015F1004F10C0501462879E368A2790090C9B21C
S214015F20204600F087FB04F11800FBF719F9297FDA
S214015F30AB69AA7C0091C1B204F1180000F07AFBAB
S214015F4004F13000FBF70CF904F13C052979E36B09
S214015F5094F836200091C1B204F1300000F06AFBDB
S214015F6004F14800FBF7FCF8297FAB69AA7C009195
S214015F70C1B204F1480000F05DFB3A48002101700F
S214015F80417031BD80B54FF48051002000F0ECFA2D
S214015F904FF480510020FAF77BF8BDE8014068E72E
S214015FA03048012101707821417070472D480078F2
S214015FB0704770B52B4C607882B000284DD0401EDB
S214015FC06070C0B2002848D12078002845D04FF430
S214015FD08051002000F0C8FA07210FF28C0000F073
S214015FE0F3FA1E4D2846FBF7BBF805F10C060146F1
S214015FF03079EB68AA790090C9B2284600F01AFBFE
S21401600005F11800FBF7ACF8317FB369B27C00915B
S214016010C1B205F1180000F00DFB05F13000FBF7E9
S2140160209FF805F13C063179EB6B95F83620009127
S214016030C1B205F1300000F0FDFA05F14800FBF7AA
S2140160408FF8317FB369B27C0091C1B205F1480087
S21401605000F0F0FA00202070607073BD3C06FF1F50
S2140160604206FF1F401EFF1F4F7074696F6E73005C
S21401607010B54E4A002410729172507A232816D019
S2140160803A2804D03B2804D050280DD012E02A2903
S21401609003D100F04AF8044611E0D07A78B1401EE8
S2140160A0D072FEF783FA0AE03A20507205E03C20EF
S2140160B0507202E030380A2801D200F002F8204679
S2140160C010BD38B5394C627AE17A257A104695B911
S2140160D00A2912DA21B921706170A170E17021716B
S2140160E04B08CD071D5D52BF62F3030505F00F0592
S2140160F045EA021507E00529ECDB0846FEF732FA09
S2140161000020E07231BD1D55491CE172A17A09B12A
S214016110084606E03C2A08BF232002D03A2A08BFD8
S2140161205020BDE83240FEF711BA38B51F4DE87A67
S214016130002408B901240FE0297A19B9EC722873F2
S214016140022409E0062804DA002100F007F80446D4
S21401615002E0FEF707FAEC72204632BDF8B5134CA2
S2140161600022E2812073024600250123002688B121
S214016170521ED2B201EB6200D707005D4CBF000988
S21401618000F00F0003FB006603EB830043009BB2A5
S214016190002AEDD1207AB04227BFE6810225E07AB7
S2140161A0FEF7E0F90020E0722846F2BDB41DFF1F9D
S2140161B038B504460F4D2720C046844202D255F812
S2140161C0240032BD286832BD2DE9F041094F3E68F2
S2140161D004460D4690462720C046AC4207D238F802
S2140161E014402720C046844238BF57F82460304602
S2140161F0BDE8F081B4AE01000021F8F723BE38B542
S214016200044640F2064501E000F04EFA204600F052
S21401621061FAA842F8D0002032BDF8F731BF00215C
S2140162204165F4F7FDB92DE9F8430D46814614465C
S2140162304FF00008402D14D34E464022314604F15B
S2140162401000F5F76FFC214604F11000F4F710FD7D
S214016250606D403D4030403608F140086065402D95
S214016260EBD275B3606D2818606504F11006C7009F
S2140162702A4608EB09013046F5F754FC0022C5F121
S2140162804001A819FCF78AF98020A855382D08D3B3
S21401629021463046F4F7ECFC002240213046FCF75C
S2140162A07DF906F1380086F83870390A4170390CE4
S2140162B08170390EC17030462146BDE8F443F4F7CB
S2140162C0D7BCBDE8F18330B40122002310F8014B9E
S2140162D011F8015BAC4201D0002214E010F8014B2A
S2140162E011F8015BAC4202BF10F8014B11F8015BDB
S2140162F0AC4202BF10F8014B11F8015BAC42EBD186
S2140163001B1D102BE2DB30BC10467047030000203B
S21401631013F0030F09D0521E22BF13F8010B11F818
S21401632001CBB0EB0C00F3D07047121F22BF53F81D
S214016330040B51F804CB6045F7D0121D0AD200BAFF
S2140163409CFA8CFCB0EB0C0038BF6FF0000088BFE5
S21401635001207047521E22BF13F8010B11F801CB22
S214016360B0EB0C00F6D0521C08BF10467047000078
S21401637038B504460D4600A8FAF7D8FE35B114F82C
S214016380011B00A8FAF7D6FE6D1EF8D1BDF8000075
S21401639032BD2DE9FE4F82B080460126FAF7E0FEB7
S2140163A0A34C676C81460025206C4FF0000A402301
S2140163B02246E919F9F769FDA346C9F1400082456D
S2140163C04CD24A4641465846F8F716FF00283AD1BD
S2140163D00AEB0900401900EB0708206C012322464E
S2140163E04146F9F752FD2678206CB31C9BB2621C1D
S2140163F008F10101F9F749FD3019354641788078F1
S21401640041EA0029671C00A8FAF790FE35B117F893
S214016410011B00A8FAF78EFE6D1EF8D1BDF800002C
S21401642048450ED1029960780870A01C039908604F
S214016430701E0499087006EB0800001DA064002673
S21401644010E002260EE00E980AF1010A0BF1010B8C
S2140164500028B2D14FF0000A4FF0FF355544B5F58C
S2140164607C6FA1D3304605B0BDE8F08F2DE9F34F20
S2140164706F4F81B0BC6C90469A4601264FF00009DA
S21401648004E06D1C401C362D0ED3A944786C09EB34
S214016490040100F57C60814262D2386C00254023FD
S2140164A03A46F9F7F2FC384601785B29E9D14FF014
S2140164B0000B00210246491C0A290CDA53783D2BB1
S2140164C01EBF491C93783D2B1EBF491C12F8033F83
S2140164D03D2BF0D18B465FFA8BF10029D1D04E1EB1
S2140164E0E819411C01983246F5F71CFB0298067024
S2140164F07019801C48440619386C01233A46314607
S214016500F9F7C3FC3C78386CA31C9BB27A1C711C4F
S214016510F9F7BBFCE01925464178807841EA002965
S21401652007F1010B00A8FAF701FE35B11BF8011BB4
S21401653000A8FAF7FFFD6D1EF8D1BDF8000048452A
S2140165400DD1787888F80000B81CCAF80000601EE3
S2140165500C990870A019001DB864002600E00226F8
S214016560304603B0BDE8F08F314A10645164F9F744
S214016570E5BB70B584B00446002000900D4601AB23
S21401658002AA0DF105010FF21810FFF702FF06002F
S21401659002BF01269DF80500072802BF9DF80400EA
S2140165A0E9B2884206D102982A462146FFF7AEFE96
S2140165B000B90026304604B070BD10B582B0049C08
S2140165C00094FFF753FF16BDF8B5194C676C0546E6
S2140165D00E46206C0021F9F74AFC206C3946F9F783
S2140165E057FD206C3946F9F779FC05220FF2B00108
S2140165F02046F5F7A7FA701C607132460720A07195
S2140166002946E01DF5F78EFA711C89B2A01DFFF729
S214016610AFFEF11D0A190855000A5070881C5D214D
S2140166200155421C206C2146BDE8F84035E00000CB
S214016630601CFF1F2DE9F0410C46014D02E000BF32
S214016640601CFF1F5B2129701646014698462246AC
S214016650681CF5F767FA601C3D214155401C069CF5
S214016660611C4155471C78197E5522464146401CFF
S214016670F5F758FA611C89B27819FFF779FE611CA3
S214016680C9194A194855000A5070881C5D214155A0
S214016690421C286C2946BDE8F04192B2F9F75BBC72
S2140166A05B7365633D00000010B509480068C46966
S2140166B0F5F704FB60682168016048602046F5F73D
S2140166C0E1FB04F0DFF8BDE81040F5F701BF00BFBD
S2140166D0200AFF1F38B504001C48056803D0E0688F
S2140166E01B49884202D04FF4826032BDF5F7E6FAC4
S2140166F004F11A0004F09CF958B1F5F7E9FEA06A16
S214016700E969884202D140F2094032BD40F20640B2
S21401671032BDE869A062F5F7DBFEA068800513D5F7
S214016720ED69F5F7CBFA286A2169C089814209D259
S214016730E869C08981423CBF2846F8F7D1FDE06A86
S214016740401CE062F5F7C4FE002032BD200AFF1FA0
S2140167507874756D10B5A94CF4F78BFF2070FCF7B3
S21401676029FEF9F753FFF9F78AFEFFF782FBFDF7DB
S214016770D3FFFBF748FDFDF7C3F9FDF7A7F8FBF7D5
S214016780D3FFF9F71FFAFCF7D5FDFCF713FEFDF76B
S21401679013F8FBF787FAF9F7C1FFFCF70BFE4FF486
S2140167A0C870F9F79BF80120FAF7CDF9FBF776FDEB
S2140167B06420F9F793F80020FDF73CF90020FAF77A
S2140167C081FBFDF7BFFE192060800921FA20A08019
S2140167D04FF47A70E0800720FCF7BFFD8848894CAB
S2140167E0016841F0040101600020207004206070FF
S2140167F00020A070E070207101206071A071F4206B
S214016800E07101202072F42060720520A072002041
S214016810E07251200FF28111FCF723FE01220221C2
S2140168205120F8F789F8607940F00200607100F0B5
S214016830F9F8FCF7BFFDF8F707FDFA21012000F093
S21401684071FAFA23012200210FF2F90000F0DAFAB8
S2140168506D490020086000F0E9FA0446022100F0C4
S214016860EDFA0521204600F01BFB00220221002044
S21401687000F060FB040006D0022100F0DFFA0521DB
S214016880204600F00DFB00220321002000F052FB01
S214016890040006D0022100F0D1FA0521204600F0BE
S2140168A0FFFA06210120FCF758FD584C08E020703D
S2140168B002210120FCF75AFDFDF73CFFFFF7F4FE2D
S2140168C006210120FCF74FFD01210120FCF74EFDBA
S2140168D0FDF776F80028EAD00220E8E710B5062191
S2140168E00220FCF73AFD4A4C06210220FCF73BFD4C
S2140168F001210220FCF73AFD2068401C2060FAF7CF
S214016900C9F8FBF764FD0120F8F7E8FFECE710B5DE
S21401691006210320FCF721FD3E4C06210320FCF74F
S21401692022FD01210320FCF721FDFDF71BF9FCF7F1
S2140169307EF800F001FB2068401C2060FFF7B4FEE3
S214016940EBE7000018B43448416803780422DC07FA
S21401695006D543F00402027001222B4B1A6016E0A2
S214016960C3F3400404B10122491C91420FDB00210C
S214016970254AC3F380032BB901231360027842F042
S214016980040203E01160027802F0FB02027041602B
S21401699011BCFCF7EFBC000010B503210720FCF783
S2140169A0E2FCFBF720FF154C608838B1401E608082
S2140169B080B218B919206080FCF7B6FF174AA18883
S2140169C01378002905D0491E89B211B943F008038E
S2140169D0FA21A180E18831B1491E89B219B94FF473
S2140169E07A7143F01003A0681370401CA060E18028
S2140169F00B48017861708078607010BDD01DFF1F54
S214016A0034800440002006405C08FE434C1EFF1FF5
S214016A10181EFF1F1C1EFF1FFC1DFF1F0004FF1F6B
S214016A2005200640044890F8020100F00300022801
S214016A3008BF00F003B87047DC17FF1F2DE9F041CF
S214016A40BAB00024FCF7B8FC002211465120F7F733
S214016A5073FF2046F9F772F900F0E6FA019005ADEA
S214016A6003206872FF260120A872059018AF03E084
S214016A700598002800F0B48000203864B046687A93
S214016A80032862D1A87A012817D002281BD00A2829
S214016A9022D00F2829D010282CD0112830D0122827
S214016AA037D013283ED0142841D0152844D0FA28D0
S214016AB004BF4FF00008012447E028AA402129A876
S214016AC0F8F784FC40E028A800904023E97A29AA38
S214016AD008A8F8F79DFC37E028A800904023E97A3B
S214016AE029AA08A8F8F7D7FC2EE0E97A08A8F8F74B
S214016AF0F4FC29E028AA402129A8F8F75BFD23E049
S214016B0028A800904023E97A29AA08A8F8F774FD76
S214016B101AE028A800904023E97A29AA08A8F8F7DD
S214016B209BFD11E0E97A08A8F8F7BBFD0CE0E97ACD
S214016B3008A8F8F7CFFD07E028A800904023E97AD7
S214016B4029AA08A8F8F7EAFD80460020A8645E2076
S214016B508DF860000120A864032078700220A864E4
S214016B6001A8A97A00F0C8F8386C411CC9B201A87E
S214016B7000F0C2F8414601A800F0BEF8002017E078
S214016B8001AA81183F2B91F8A01010DA9A1882F802
S214016B905C10AA6C521CAA645E2908D1022A06DB84
S214016BA001A9511881F85C60A96C491CA964401CB4
S214016BB0C0B23A6CAB6C9042E2DB0122591E0DF179
S214016BC0610000F06EF8014601A800F095F8AA6C85
S214016BD0019818A900F088FA00200590686002E084
S214016BE001A800F012F8019808B100F0ADFA0120F2
S214016BF0F8F774FE002C3FF43BAF6420F8F76EFE06
S214016C00F4F72DFD3AB0BDE8F08170B5044682B0C8
S214016C1004F1180605E0E06820F00100E0600020BD
S214016C2060610122206800A900F075FA012837D1B9
S214016C309DF80050002D33D4E0685E2D03D140F05E
S214016C400100E06019E0C10710D520F00100FF2D1A
S214016C50E06006D0002060615E21204600F03DF82D
S214016C6007E060690028DCD05E2103E06069002847
S214016C70D7D02946204600F030F860690428A2BF24
S214016C80E17E4D1DA842CCDB0022A91E701C00F03F
S214016C9008F8A91911F8011C8142BCD10120206114
S214016CA073BD30B4FF23002401290BDA12E0012A58
S214016CB008D1012C06DB0578FF2D04BF10F8015C16
S214016CC05E2D03D010F8015B6B4000E0401C641C95
S214016CD08C42ECDB30BCD8B270474269402A04DAF9
S214016CE0121811764169491C04E0C16821F00101BE
S214016CF0C160002141617047826D3F2A10DA121887
S214016D0082F85C10826D521C82655E2908D1022AC7
S214016D1006DB1218FF2182F85C10816D491C816523
S214016D20704700002DE9F04104462A48056888B0FE
S214016D30288B0E4608B10D205AE005F5EA78404644
S214016D40F8F7ECF9D5F8000200284DD16420F7F7E2
S214016D50BDFD070004D14046F8F716FA042047E0C7
S214016D601D21F4F7C5FF00213846F5F7E1F90021AA
S214016D7007F10C00F5F7DCF900200090002E16480C
S214016D80019006BF4FF4487002900296002C06BF91
S214016D9001200390039400AA0FF25C0004900021E6
S214016DA0002005900790C5F8007200F0C3F8B8639C
S214016DB0A0B9C5F80002786300F002FA040008BF23
S214016DC004244046F8F7E0F93846F7F7D5FB2046A5
S214016DD00EE000BF200AFF1F65790100004801E0B0
S214016DE0F58D0100C5F838024046F8F7CDF90020C8
S214016DF008B0BDE8F081000054696D6572205461E9
S214016E00736B000070B584B004460D4616461846EE
S214016E1001A9F9F70FFF0020009001AB3246294681
S214016E20204600F0D9F904B070BD000002480068A1
S214016E30C069C068704700BF200AFF1F70B50D46C5
S214016E40164909680124012D1CBF022D27200CD1EB
S214016E5010F1010F04D1D1F8F442C1F8F4521AE04E
S214016E6000F04CFA060005D12A20F5F7C5FA4FF0D6
S214016E70FF3070BD96F82800400748BF0224F4F79B
S214016E801DFFB06A022D0CBF40F0040020F0040084
S214016E90B062F5F71DFB204670BD0000200AFF1FFB
S214016EA010B5044688B0084604A9F9F7C3FE01AA3E
S214016EB004A9204600F04AFA009028B1F5F79CFA9A
S214016EC04FF0FF3008B010BD00A901A800F0B4FAD9
S214016ED008B010BD30B50C461146154A126800259B
S214016EE083B0002C48BF152007D458B1FF2803DC17
S214016EF0D2F8A421904205D01320F5F77DFA0020A0
S214016F0003B030BD0093204600231A4600F096FADF
S214016F10040009D0E568F4F7D1FE2046F4F7B2FF85
S214016F20F5F7D6FA03F0A0FC284603B030BD000002
S214016F30200AFF1F0023CDE710B5154C2078010766
S214016F4004D500F0F7002070FCF7EAFE2078C106B1
S214016F501DD500F0EF002070FEF7E9FEFBF772FA90
S214016F60F3F7EAFEFCF792FAFBF707FCF3F7E8FE05
S214016F70FDF729FBFFF71DF86078401E6070C0B270
S214016F8028B90A206070BDE81040F9F7E3BD10BDCE
S214016F900004FF1F10B1022802D1012082490863B4
S214016FA070472DE9F041804CD2F800800D46216BE8
S214016FB0012937D1242808BF012002D0232803D174
S214016FC000206063BDE8F081042820D1606B0128B1
S214016FD028D104F17800FEF7B7FD07466868B84285
S214016FE038BF87B20026012F08DB2868315C04F120
S214016FF07800FEF770FD761CBE42F6DB04F138021F
S2140170004046BDE8F0414023032100F070BC032850
S21401701004BF606B012805D12188201DFEF778FD8D
S21401702000202080BDE8F08130B55F4D686A0024FD
S21401703091B010F1010F4FD14FF48060F5F77EFA51
S214017040A86200284DD04FF48060F5F777FAA96A58
S214017050E86200283BD04FF480631A4605F17800B9
S214017060FEF704FD4FF48063E96A1A46281DFEF711
S214017070FDFC4FF44370F7F729FC022100910E90B6
S2140170800A940B940120494906918DF804000321C6
S21401709007910220464908918DF8050005F1240163
S2140170A00991032043490C918DF8060005F124014E
S2140170B00D9141490F91F4F701FE00A800F03AFB4B
S2140170C068622C80F5F704FA686A50B905E008464C
S2140170D0F7F752FAAC6204E018B9686A374951F812
S2140170E02040204611B030BDF8B52F4F0C4615464E
S2140170F00026381DFEF728FDA8420ADB012D07DB16
S2140171002E4614F8011B381DFEF7E5FC761EF8D155
S2140171102E463046F2BDF8B5234E0C46154606F10E
S2140171207800FEF701FD0746BD42B8BFAFB2012F9A
S21401713008DB3D4606F17800FEF7BEFC04F8010BBD
S2140171406D1EF7D13846F2BD70B5174C606A10F166
S214017150010F28D038BB1948006820B3206B0128DE
S21401716004BF606B01281ED1201DFEF787FC10F1BD
S214017170010F18D02088B0B9201DC068C04605464A
S214017180A068401B461C201DFEF7CEFCB6B2864208
S21401719088BF064626802388606A2A46BDE8704076
S2140171A0022100F05DBB70BDD006FF1FA407FF1FC4
S2140171B0956F0100A36F01006807FF1F301EFF1FB8
S2140171C004480068018B002919BF406BC068C0697C
S2140171D0C06D7047200AFF1F2DE9F04F80461B48FF
S2140171E083B00468D4F800628A461546994646B9C3
S2140171F04FF448710120FFF795FDD4F80062002E88
S2140172005DD0706BDFF848B0584518BF1A2056D1CC
S2140172105FEA080017D0012D18BF022D13D1DFF841
S21401722034C0D9E90023DCE900018B4214D301D82C
S214017230824211D3DCE90023D9E900018B420BD34A
S21401724001D8824208D30C2039E000BF200AFF1F74
S214017250726D6974D8AF01003C20F7F737FB070061
S21401726048D01E213046F4F743FDB9E80E0007F179
S2140172700800A9F10C090EC0012D00A802D100F0EA
S21401728051FB01E0FBF7BEF9C7F82080C7F824A040
S214017290FD8607F114020C98386300A91120B88600
S2140172A04846F9F7FBFCE069B862F16BE069884291
S2140172B009D006F11800F7F731FF20B11F20F5F7C6
S2140172C09BF8002016E0C7F82CB0304600F062FCB0
S2140172D0B863012D39460CBF304606F10C0000F0AC
S2140172E039FCE069F16B88421CBF06F11800F7F71C
S2140172F04BFFB86B03B0BDE8F08F000070B504001B
S2140173001148056801D1E86970BDE86D844202D173
S21401731005F1500070BDF4F7D1FCD5F81C01A0F1C1
S2140173206C06B5F8240102E0F16EA1F16C0638B1E5
S214017330F168401EA142F7D1F5F7CAF8304670BD94
S214017340F5F7C6F8002070BD200AFF1F70B50C4681
S21401735011490E68154610F1010F08D106F53E7069
S2140173600EC80EC5F4F7AAFC06F53E700DE0FFF751
S214017370C5FF060001D12A2070BD06F1A0000EC887
S2140173800EC5F4F79BFC06F1A0000ECC0EC0F5F777
S2140173909FF8002070BD00BF200AFF1F2DE9F041B5
S2140173A005462448D0F8008084B00020CDE90200CC
S2140173B00C46D5E90001CDE9000108F5C877164667
S2140173C0B96800AA00A800F006FCA96800AB042270
S2140173D000A800F04DFC00AA42F2107100A800F0CF
S2140173E0FAFBD8F8901100AA00A800F05AFCB96878
S2140173F000AA00A800F055FC2EB100AB042205211E
S21401740000A800F035FC00AA0A2100A800F049FCFB
S214017410DDE90201002908BF002805D10198401EB8
S2140174208041C043C00F00E001202060009804B0F6
S214017430BDE8F081200AFF1F0122AFE72DE9FC47D6
S2140174400C4619490F681546984668B1A146D7F803
S214017450B441002600E020342168002918BF81428B
S214017460F9D1080003D103E0D4F8189001262CB90D
S2140174701020F4F7C1FF0020BDE8F68707F5A47ACF
S2140174805046F7F74BFECDF8048000953346F86971
S214017490C1684A462046F4F731FC04465046F7F7E1
S2140174A073FE2046BDE8F687200AFF1FC06800224B
S2140174B000E0521C0378D2B29A4204D2436813F811
S2140174C032308B42F5D11046704770B584B00C4609
S2140174D001792046FFF7EAFF00EB80118800616C16
S2140174E041188B78CA785B1C8B70616C4018817868
S2140174F0914212D0CB0801EB13731B09A1EB0311C8
S21401750000EB0110001D6AC800AA6AC29DF80410AB
S214017510606833462A4600F0BBFCE36A180006D0D2
S214017520226B04B0BDE8704000210320184704B068
S21401753070BDF0B5054687B00C4629792046FFF7A1
S214017540B5FF00EB80118800616C41188B78CA7812
S2140175505B1C8B70616C41188B78934212D0DA08F1
S21401756003EB12721209A3EB021201EB0211091DC1
S214017570CCC902A8CCC09DF80C1060683B463246C8
S21401758000F086FCE06B40B12869009000A96869AC
S2140175900190226CE36B0320984707B0F0BD00B55D
S2140175A083B00269009240690190CB6B180003D04A
S2140175B00A6C00A90420984703B000BD2DE9F84FD6
S2140175C004468B461646022C33D1F068DFF83C831E
S2140175D0DFF83C93DFF83CA3009000270AE0B06890
S2140175E000F085FD287840F01001B068002200F018
S2140175F023FE7F1C00980078FFB287422CD20098A9
S214017600406800EBC705B0680122294600F058FD26
S2140176106878022805D00328E4D129783346424603
S214017620DDE7A8782978002833460CBF52464A463B
S214017630D5E78CB900220BE0736C00EB801103EBED
S2140176408103401C9A70C0B2736C03EB8101CA704F
S214017650F16809788842EFDBF36A180006D0326BCE
S2140176605946204601B0BDE8F04F1847BDE8F18FF6
S21401767070B505461C462B78CD2003F06006202EFB
S2140176804DD16B780020022B1FD0032B0AD0042B80
S21401769010D0202B29D0212B1FD0222B2DD0232BED
S2140176A033D03AE013460A4629462046BDE87040E4
S2140176B000F0A2BE2069106000200B6818700868F0
S2140176C0401C086000200B68187013460A462946BD
S2140176D02046BDE8704000F0ADBE13460A46294676
S2140176E02046BDE8704000F02CBE13460A462946E7
S2140176F02046BDE8704000F034BE13460A462946CF
S2140177002046BDE8704000F03DBE13460A462946B5
S2140177102046BDE8704000F065BE106070BD03F005
S2140177206003402B05D1666B330002D0A36B28465D
S214017730B04770BD2DE9F04782B0040008BFFF20B6
S21401774000F08C804820F7F7C1F85FEA000808BF10
S214017750812000F08380DFF8C091D9F8000028B1BD
S2140177604046F6F709FF8D20BDE8F68748214046DA
S214017770F4F75CF908F12807A06BF86108F1080135
S214017780A569207D88F828002878421CD2B20020FE
S21401779000F005FC5FEA000A55D1E06B5F4A002164
S2140177A0016008F104060090434670685C4900F0E9
S2140177B01AFBC8F8040004F13001404600F0A8FDA9
S2140177C05FEA000A3FD1B56017E06A68FB6912F804
S2140177D0302000EB80118900CA546A68FB6902EB0D
S2140177E0C002CB1852785A700022FB69CB18401C95
S2140177F09A70C0B2FB69C918CA7029788842E4DB5E
S214017800206A7860606AB860A06AF860E06A3861E9
S214017810206B7861606BB8612068F0602079307405
S214017820002070746079B074A079F074A0687061FB
S214017830E068B0612069F0610020C8F80000C9F86E
S2140178400080BDE8F687D9F80000F6F795FE00201F
S214017850C9F800004046F6F78FFE5046BDE8F687A9
S2140178602DE9F04100270C4615469846022803D21A
S214017870294951F8206016B9FF20BDE8F08121465C
S2140178803046FFF713FE00EB80118800716C431839
S214017890D9789A78A1EB020C5FFA8CFCBCF1100F38
S2140178A021D001F00F0C03EB0C13491C1C72736CF6
S2140178B0C31803EB0C1CCCF80C50CCF81080D6F88F
S2140178C008E0CCF804E0D970716C4018C078801AD2
S2140178D0C0B2012808D1706843462A46214600F006
S2140178E0D7FA074600E0C1273846BDE8F08118B44C
S2140178F0022803D2084C54F8200010B912BCFF200D
S2140179007047806801B010BC00F0C2BDCB740100A6
S214017910337501009F750100301EFF1F717601004F
S214017920BD75010038B5040013D00A480568F4F7A0
S214017930C5F905F5B2700EC80EC4D5F89C110C3CFD
S214017940080003D0D5F8A0018847A060F4F7C0FD71
S21401795002E031BD200AFF1F2046BDE83240F7F79E
S214017960D5B900002DE9F0417848046886B0D4F80E
S21401797000520DB902F089FFE069E863002128464C
S214017980F4F7D6FB002105F10C00F4F7D1FB00213A
S21401799005F14000F4F7E4FA012105F11800F4F7C7
S2140179A0DFFA6B4868630FF21910C4F804030095F8
S2140179B005F10C00019018E005F11800F7F7E4FB5B
S2140179C020B11F20F4F718FD02F05FFF641C08F1D8
S2140179D00408022C0CD305F14000F7F79FFB20B1F9
S2140179E01F20F4F709FD02F050FF00240DF10008F6
S2140179F0D8F8006005F11800F7F790FB50B11F208A
S214017A00F4F7FAFC02F041FF04E00020F862384681
S214017A10F6F7B2FD30890028CED03768002C02A8D0
S214017A2002D1FFF77FFF01E0FAF7ECFDDDE9022363
S214017A30D7E905018B42BFD301D88242BCD378680F
S214017A403968016048603089401E30812F66F86AC7
S214017A500028DAD0796AB86B3B6A02AA9847B88ED2
S214017A600328D2DBF86A0028CFD007F1140207F109
S214017A70080107F11400F9F711F9D6F800E04FF004
S214017A80000C02E0F446DEF800E0B64511D0D7E976
S214017A900523DEE905018B420BD301D8824208D3C8
S214017AA0DEE90523D7E905018B42EBD301D88242F3
S214017AB0E8D33A4661463046F6F7CAFDAAE7000023
S214017AC0F0B52248046883B0D4F80052002D1EBFDA
S214017AD0E86B8068022836D000A8FFF723FF2889C4
S214017AE090B12868DDE90067D0E90523BB4226D3BB
S214017AF001D8B24223D3DDE90023D0E90567BB42B2
S214017B001DD828BFB2421AD2A88AE0B100AA04F54D
S214017B10B87100A8F9F7C2F8E868DDE90067D0E9AE
S214017B200523BB420BD301D8B24208D3DDE90023BB
S214017B30D0E90567BB4206D301D8B24203D305F1AB
S214017B404000F7F721FB03B0F0BD0000200AFF1F3D
S214017B50726D6974FCB40268002301E01346126872
S214017B60824211D0D1E90545D2E90567BD420BD362
S214017B7001D8B44208D3D2E90545D1E90567BD422B
S214017B80ECD301D8B442E9D302B0F0BC0A46194698
S214017B90F6F75EBD30B4C16D09B90121C165C16D8D
S214017BA003E0956B8D420BD1491C002300E00BB915
S214017BB0044601E000F10C0422682489641C00E0FC
S214017BC01268641EEDD15B1C022BF0D34A1CC26501
S214017BD0084630BC70472DE9F04385B00026CDE954
S214017BE000660346002479B1D3E90089B9F1000F94
S214017BF008BFB8F1000F0AD1D3E90289B9F1000F25
S214017C0008BFB8F1000F02D1CDE9026629E00129CB
S214017C1003D133CB33C2002027E098460DF1000C88
S214017C204FF0030E0C4658F8046BA6FB0401DCF873
S214017C3000608619CCF800605CF8046B8642B64199
S214017C4001EBD670CCF80000BEF1010EEBD1D8687E
S214017C50A0FB0467039830180390B042804107EBFD
S214017C60D07400A8CAC8CAC2204605B0BDE8F083D1
S214017C7030B450F8044B0C198C4243F8044B89413C
S214017C80C90F012408E050F8045B491943F8041BA6
S214017C90A9428941C90F641C9442F4D330BC0846FA
S214017CA070472DE9F04E86B0924611B94FF0FF307D
S214017CB03AE0012934D0D0E90023002B08BF002A7E
S214017CC005D1D0E90223002B08BF002A28D00022C4
S214017CD0CDE90222CDE9002200F1080BC26802AE0E
S214017CE003270C4613465BF804090022151843EBDC
S214017CF00209494622460023FAF7D8FBA4FB0023D3
S214017D00736819447160AA1A3168084446F8040970
S214017D107F1EE7D100A872C8AAE87200104603E0E9
S214017D201EC8AAE81E00002006B0BDE8F08E0000BE
S214017D3070477047017921B900680022102100F0D0
S214017D407BBA704701690A784978006841EA0222DD
S214017D50052100F071BA30B583B004460D0037D066
S214017D6000208DF802008DF80000012240200190CD
S214017D7000A900208DF80100206800F0A1F99DF807
S214017D80000040F010012068002200F055FA0120A2
S214017D908DF802000122206800A900F091F99DF8F3
S214017DA0000040F090012068002200F045FAEB68E0
S214017DB0180003D0AA6800210020984720680222F4
S214017DC0012100F039FA20680122062100F034FA78
S214017DD003B030BD31B1CB681A0003D08A6801699F
S214017DE00520184770472DE9F043044683B00D4639
S214017DF0904699461020F6F769FD060008BF8120D7
S214017E0043D0524F386820B13046F6F7B5FBC12053
S214017E103BE07460F560C6F808904B460A980190FE
S214017E204246002000902946204600F063FB306061
S214017E30FF2828D03346464A1021204600F057F93D
S214017E403346444A1221204600F051F93346424A4D
S214017E501421204600F04BF93346404A13212046B0
S214017E6000F045F933463E4A1721204600F03FF917
S214017E7033463C4A1621204600F039F903220121F7
S214017E80204600F0D9F93E60002003B0BDE8F0833B
S214017E902DE9F0410C462D4982B051F82060154677
S214017EA09846002716B9FF20BDE8F681706800AA3B
S214017EB0012100F085F970680DF10202062100F03B
S214017EC07FF9BDF80000802816D1BDF802008007B2
S214017ED012D5306800F024FD01280DD1F3F7EEFE2F
S214017EE0706800F006FAADF8007000227068012193
S214017EF000F0A2F9F4F7ECFABDF80000802806D0ED
S214017F00706843462A46214600F01AFD0746384661
S214017F10BDE8F68118B4022803D20C4C54F82000B0
S214017F2000B921E0006801B010BC00F0DFBC18B455
S214017F30022803D2054C54F8200000B914E000686A
S214017F4001B010BC00F0DFBC00000000341EFF1FB3
S214017F50577D0100457D0100317D0100337D010023
S214017F60357D0100D57D010012BCFF207047000061
S214017F7038B504460D46F3F7A1FE606900280FBF29
S214017F806561A069806C0560A5610020A96C086028
S214017F90206A401C2062BDE83140F4F799BA2DE909
S214017FA0F84F80468A46144600F00AFD424940468C
S214017FB000F014FDB8F1020FA8BF8B2076DA4FF45B
S214017FC06070F6F783FC060008BF87206ED04FF47A
S214017FD06071F3F72BFD042000F01EFD10EB8810F6
S214017FE0706008BF892061D0404600F041FD10B1A5
S214017FF0C420BDE8F28F404600F05AFD306040468E
S21401800000F062FD86F83700371DFF20388586F8B8
S21401801039404FF41860F6F759FC040008BFA92050
S21401802044D0FC604FF4C070F6F750FC38625FEA4B
S214018030000929D0002038617861F8614D464FF07B
S214018040200BC4F848901D4868602E60F3F736FE92
S214018050706900280FBF7461B069806C0460B461F8
S2140180600020A16C0860306A401C3062F4F730FAD8
S2140180704C340C3509F10C09BBF1010BE1D14C2054
S214018080F6F724FCB86010B98120BDE8F28F4C21C8
S214018090F3F7CCFC70684268100009D031464046C0
S2140180A09047002814BF8D20CAF80060BDE8F28F03
S2140180B0FF20BDE8F28F0000040BFF1F717F010057
S2140180C018B4C4680B782370C4688B786370C4686E
S2140180D04B682382C36849789970C1684A614168D0
S2140180E04A69110002D018BCC168104741E0F8B5D2
S2140180F004000D4616461F4601D1FF20F2BDF3F7D8
S214018100DDFD083401E000F10C04206830B101788F
S214018110A942F8D1F4F7DCF98420F2BD1020F6F775
S214018120D5FB18B9F4F7D4F98120F2BD0570466085
S21401813087600021C1602060F4F7CAF90020F2BD13
S21401814070B50D4604462E68F3F7B8FDB26800E038
S214018150D26852B11078A042FAD191685268284686
S2140181609047F4F7B5F9002070BDF4F7B1F9832014
S21401817070BD12BCFF20704720B14268D26A13005E
S21401818018BF1047FF20704770B582B004000D4637
S214018190164612D00094F3F791FD00984068C06926
S2140181A058B1009B5B68DB693246294620469847F2
S2140181B00446F4F78DF9204676BDFF2076BD000013
S2140181C070B582B005000E46144618BF002C2DD09F
S2140181D00095F3F773FD701E052818D8DFE800F048
S2140181E003060D11140A0098808D2080F4F770F9AB
S2140181F0002076BD0098C08DF7E7009890F83C0007
S214018200F3E70098408FF0E70098008EEDE7F00660
S2140182100ED500984068006A40B1009B5B681B6AF7
S214018220224606F00F0128469847DFE7FF2076BD75
S214018230F4F74EF9822076BD2DE9F0410F4682B063
S21401824006461546002407F00F0816B9FF20BDE8BC
S214018250F6810096F3F732FD781E052825D8DFE86B
S21401826000F00305130D100A00988585F4F730F920
S2140182702046BDE8F6810098C585F7E70098458752
S214018280F4E700980586F1E7009880F83C500098DE
S2140182904068C06A38B10098009A5268D26AE9B25A
S2140182A090470446E2E7FF24E0E7F8060FD5B8F169
S2140182B0100F0CDA00984068406A0028F3D0009B43
S2140182C05B685B6A2A46394630469847E9E7F4F721
S2140182D0FFF88220BDE8F68182B048B10090009B8D
S2140182E05B68DB6B23B1009B5B68DB6B02B01847F6
S2140182F00BE082B048B1009000994968896B21B1C2
S21401830000994968896B02B00847FF2002B07047A0
S21401831070B504460D462020F6F7D8FA060001D1BE
S214018320812070BD2021F3F781FB0A223146554892
S21401833000F0D0FB2868F060686830616662002053
S21401834070BD18B4446A14B912BCFF2070478988FE
S21401835021771346227F406801B010BC2121FFF728
S214018360D9BD02B500211960416A09B9FF2002BDD5
S214018370009A92880A7700AB0A7F40682021FFF7AF
S214018380D6FD02BD10B5446A0CB9FF2010BD00220F
S2140183901A60498821766277E16809B3217E4A0826
S2140183A002F001029201627742EAC112627701F09D
S2140183B00101616100F05CF8207EE36822698007B4
S2140183C047BF00212220002121209847207EE36814
S2140183D02269C00747BF0021242000212320984797
S2140183E0002010BD406A08B9FF20704700221A60BD
S2140183F0498841830020704770B5456A0DB9FF2052
S21401840070BD06691E6000248E882E774988012972
S21401841003D113462A7F232104E0022907D11346FC
S2140184202A7F24214068FFF775FD044600E01C60A2
S214018430204670BD70B5456A0DB9FF2070BD06694E
S2140184401E6000248E882E774988012903D11346A1
S2140184502A7F252104E0022907D113462A7F2621F7
S2140184604068FFF764FD044600E01C60204670BDCE
S214018470426A2AB1117F11710A23517F117203E0FA
S21401848070470000280AFF1F017D0068FFF7E8B962
S214018490F8B504000D4616461F4626D0F3F70EFC27
S2140184A0206A18B9F4F714F80320F2BD60690100D8
S2140184B004D0806C0068606100B9A061206A401E2B
S2140184C020620D70002048708F604E60C8600620E4
S2140184D0C8706068C268100007D0204690470446FE
S2140184E0F3F7F6FF1CB90020F2BDFF20F2BD942081
S2140184F0F2BD00002DE9F8430446884691461F4622
S2140185004C20F6F7E3F9050012D0DFF82C6430684A
S21401851028B12846F6F730F8FF20BDE8F283089820
S214018520A864002028615420F6F7D0F9286110B914
S2140185308120BDE8F2836C60C5F81490AF61C5F880
S2140185401C802F622422099805F1240100F0C2FA4A
S2140185502B460FF2150200212046FFF7C8FD3560B5
S2140185600020BDE8F283000070B584B00646002006
S214018570ADF8080003900C463068CD2502AA01210B
S214018580FFF71EFEB068012853D13069082204F1B6
S214018590080100F09FFAA089A081602260896081AD
S2140185A0E089E081217A114220D1607ADFF88C637C
S2140185B006EB8001D1F89C10002956D0BDF80810B2
S2140185C0032952DA00EB400206EB820050F8210044
S2140185D001284AD1657A06EB850501ABD5F89C5092
S2140185E003AA04F108012046A8473DE00190B0B176
S2140185F0207A000613D40198083055283ED2216906
S214018600082204F1080000F065FA2069019B00F1D8
S214018610080230680021FFF73BFF04B070BD6669B1
S214018620300022D0A36901AA03A904F10800B047CB
S2140186301AE0BDF80800042804D1204600F0C9F865
S21401864004B070BD207A000618D4F068B0B9E0898D
S214018650A0B1606948B1706908300190A3692069CA
S214018660656901AA03A9A847054601A8009003ABBE
S21401867004F108022946204600F002F804B070BD55
S21401868038B5044615461846CD2906D16068BDE8BA
S214018690384001229021FFF7CFBD0499EA880B6884
S2140186A09A4238BF0A6002680B68A06C0021FFF787
S2140186B0EFFB2878000608D5606801B0BDE83040B9
S2140186C0002200231146FFF7E3BE31BD7CB51546F7
S2140186D004461E460A78FF2003231A4209D1606821
S2140186E022460621FFF76CFD217801F00301218067
S2140186F017E002F00303012B07D18988606A236B18
S2140187002246C9B2984701210CE002F00302022A70
S21401871009D1888840F0100160682246C9B2FFF787
S2140187204FFD022131602C6076BDF8B5044600206D
S2140187300E461860CD257078C0F3400730780321C7
S21401874008421BD1B078084233D0606800AA0621DF
S214018750FFF736FD718801208840BDF80010002F14
S21401876014BF084321EA0000ADF800000621BDF859
S21401877000206068FFF760FD05461AE000F0030080
S214018780022816D1B0888DF802003A469DF80200FC
S21401879040F010016068FFF74FFD0546002F14BF3B
S2140187A007200820E369190003D0226A0DF10201AF
S2140187B098472846F2BD38B50446002018600D4695
S2140187C0606804220121FFF737FD68886080002079
S2140187D032BD10B5044661886068C9B2FFF7CCFCAB
S2140187E0606801220121FFF727FD62886068032186
S2140187F0FFF722FD002010BD38B5044601201860A1
S2140188001546606822460421FFF7DAFC2C6000203A
S21401881032BD38B504460020186004254888ADF8F6
S21401882000000146606AA26B9047D8B1BDF800000F
S214018830002200B9012260680121FFF7FDFCBDF8A6
S214018840002060680421FFF7F7FCE369054618007D
S21401885008D0226A00A901209847226AE36900210C
S21401886002209847284632BD38B5044601201860D4
S21401887015468988606A236B2246C9B298472C60E0
S21401888032BD10B5044600201860087800F00300D9
S214018890012801D0042010BD4A888988606A636B6C
S2140188A0D2B2C9B29847002010BD38B5044602209E
S2140188B018601546606822460521FFF781FC2C608A
S2140188C032BDF0B583B04F8806463D0AFF24FF202F
S2140188D0032D04BF88883C46019300920346E2B20A
S2140188E0706AB46A2946A04703B0F0BD10B50228E5
S2140188F003D2114C54F820400CB9FF2010BD606A19
S214018900646CA04710BD10B5022803D20A4C54F877
S21401891020400CB9FF2010BD606A246CA04710BD32
S214018920022803D2044951F8201009B9FF207047E4
S214018930486AC96B08470000381EFF1F340AFF1F2C
S214018940F8B504000D4616461F4635D00094F3F7D9
S214018950B5F90098006A18B9F3F7BAFD0320F2BD1D
S214018960009841690098406950B10098009A526990
S214018970926C126842610098406908B9009A906149
S2140189800098026A521E02620D70012048708F60C4
S2140189904E600020C8600620C87000984068806855
S2140189A050B1009A52689268204690470446F3F701
S2140189B08FFD1CB90020F2BDFF20F2BD9320F2BD51
S2140189C004480068818A4FF6FE721140818202488F
S2140189D000F034B9200AFF1F55A3010070B5044604
S2140189E00D46042000F018F806000DD14020F5F7DA
S2140189F06DFF060001D1882070BD0421F3F716F83B
S214018A003146042000F017F806EB84102946402270
S214018A10F3F798F8002070BD80B5082804D30C2021
S214018A20F3F7EAFC002002BD1049096801EB80005B
S214018A30D0F8A40202BD70B504460C4806680D467F
S214018A40082C04D30C20F3F7D7FC002070BDF3F7F5
S214018A5035F906EB8400D0F8A442002C14BF002D93
S214018A60C0F8A452F3F734FD204670BD200AFF1F5C
S214018A7080B5F2F7B4FFD0B91048016841F0004163
S214018A8001600F48017B41F080010173017B0906FB
S214018A90FCD400210170012210210172017B41F0FA
S214018AA04001017359200421F5F746FF002002BD5D
S214018AB008B100207047034870470000007004406A
S214018AC0002107400020074008B1002070475920C8
S214018AD07047000030B403461C460846042AC0F01E
S214018AE0A080DD0706D514F8011B00F8011B2346FC
S214018AF00146521E980704D533F8020B21F8020BE3
S214018B00921E900941D053F8044B41F8044B401E85
S214018B1053F8044B41F8044B53F8044B41F8044B0B
S214018B2053F8044B41F8044B53F8044B41F8044BFB
S214018B3053F8044B41F8044B53F8044B41F8044BEB
S214018B4053F8044B41F8044B53F8044B41F8044BDB
S214018B5053F8044B41F8044B53F8044B41F8044BCB
S214018B6053F8044B41F8044B53F8044B41F8044BBB
S214018B7053F8044B41F8044B53F8044B41F8044BAB
S214018B8053F8044B41F8044BBDD1900800F00F0098
S214018B90401E0E2845D8DFE800F0403C3834302C23
S214018BA02824201C1814100C080053F8040B41F854
S214018BB0040B53F8040B41F8040B53F8040B41F86B
S214018BC0040B53F8040B41F8040B53F8040B41F85B
S214018BD0040B53F8040B41F8040B53F8040B41F84B
S214018BE0040B53F8040B41F8040B53F8040B41F83B
S214018BF0040B53F8040B41F8040B53F8040B41F82B
S214018C00040B53F8040B41F8040B53F8040B41F81A
S214018C10040B53F8040B41F8040B53F8040B41F80A
S214018C20040B900744BF33F8020B21F8020BD00760
S214018C3044BF1878087030BC7047000002490A68C3
S214018C40916A906208467047200AFF1FF0B4049CA0
S214018C500598032920D14D4D33B92968216029791A
S214018C6001600020F0BC7047AD68B5F800C0002672
S214018C7001211746634503D1042F02DA114600E0AD
S214018C80012606EB460205EB8202536853F82730AD
S214018C9023609268895CE3E7082907DA3B4D05EB18
S214018CA08101CA6A22600AB1C968D9E7CD20F0BC41
S214018CB07047022904DA3648085C107000207047B5
S214018CC0CD207047022903DA31480A540020704744
S214018CD0CD2070472F480278914201D1012070477C
S214018CE040788142FAD000207047002070472A4819
S214018CF07047CD20212904D0232906D0242908D065
S214018D007047022A0ADA254806E0022A06DA2448CB
S214018D1002E0022A02DA2348186000207047CD20BC
S214018D20202904D025291BD0262923D07047022AC2
S214018D302ADA19681948097A01701968497A41705E
S214018D401968897A81701968C97AC1701968097BAE
S214018D5001711968497B41711968897B817112E03B
S214018D60022A11DA19680D480978017219684978DA
S214018D70417208E0022A07DA196808480978817200
S214018D8019684978C1720020704700007C08FF1FEF
S214018D90421EFF1FFC08FF1FA407FF1F0009FF1F3D
S214018DA00809FF1F0A09FF1F70B504460F4805682A
S214018DB0D5F8FC61C6B1F0680D49884214D1F2F7C6
S214018DC07DFF03E0E9698162F6F75AF93068B0423F
S214018DD006D0817E11B1816AA142F3D00068F6E720
S214018DE0BDE87040F3F774BB70BD00BF200AFF1FDB
S214018DF07874756DF8B504461C480068D0F80052C2
S214018E009DB305F11800F6F789F928680FE00168A7
S214018E10826A0E46A24209D1426811604A602989D7
S214018E20491E29810021C162F5F7A6FB3046A842FA
S214018E30EDD105F10C0738680FE00168826A0E462D
S214018E40A24209D1426811604A603989491E3981B6
S214018E500021C162F5F790FB3046B842EDD105F12D
S214018E601800BDE8F240F6F78FB9F1BD200AFF1FE2
S214018E7038B504460B480068C569F2F71FFFA868B5
S214018E800B280AD00B20A860AC6341212846F6F7D0
S214018E9020FA6868296801604860BDE83140F3F748
S214018EA017BB00BF200AFF1F0A480068D0F8C4128B
S214018EB0491CC0F8C412F9D100F531714A68521C38
S214018EC04A60F3D18A68521C8A60EFD1CA68521C84
S214018ED0CA60EBE7200AFF1F80B507480068C06933
S214018EE0D0F88400010018BF8047BDE8024000208A
S214018EF000F0D2B800000000200AFF1F2DE9F0475D
S214018F0064490C6800281FBF010CD4F8A42192B252
S214018F10914207D1FEF7F2F905001CBF04F150009B
S214018F20854202D11220BDE8F08704F5A4784046B8
S214018F30F6F7F4F8F2F7C2FEA868092805D1F3F7A8
S214018F40C7FA4046F6F720F9A1E0022807D1E06902
S214018F50854220D068682968016048601BE0C10529
S214018F600FD56868296801604860B4F88401401E1E
S214018F70A4F88401A86820F4807040F00300A8607B
S214018F8009E0800507D56868296801604860A86B14
S214018F900189491E0181A868400507D5286CE96B3F
S214018FA001604860A86B0189491E01810920A860FB
S214018FB0F3F78EFA04F50C771026396808001CBF03
S214018FC0284688473F1D761EF7D195F82800AF89B9
S214018FD0E66980061AD40021284600F05FF881462B
S214018FE011E04946284600F059F88246AE4204D0C0
S214018FF004F150014846F3F73FFAA9451CBF48461D
S214019000F5F7BAFAD146B9F1000FEAD14FF00040B0
S214019010E86004F59271B4F82401012803D1012215
S2140190204A60002205E04A68974203D24F602A6FE1
S2140190306C3A8A60296FEA6E0A605160401EA4F895
S21401904024014046F6F7A0F8B54216D1F2F736FEEF
S21401905068682968016048602846C046C04695F899
S2140190602800800607D404F150012846F3F704FAD5
S2140190702846F5F781FA01F0F5FB2846C046C046BA
S21401908095F8280080065CBF2846F5F775FA00209B
S214019090BDE8F087200AFF1F00212FE7F8B5044638
S2140190A01748056819B9D5F81463F76804E0A1F103
S2140190B00C00016846680F18F2F700FE706901E0BF
S2140190C03968CF1931698F4210D2E268398992B274
S2140190D09142F5D100E0806808B1B842FBD3B842AE
S2140190E0EED0F3F7F5F907F10C00F2BD3668D5F8C6
S2140190F01403F7688642E1D1F3F7EAF90020F2BDDE
S214019100200AFF1F38B504460094F2F7D7FD0098F1
S21401911045690098406950B1009800994969896C81
S214019120096841610098406908B90099886100980A
S214019130016A491E0162F3F7CBF9002028706870B6
S214019140A860A8700120686194F85910DFF8CC0D6A
S214019150400A400201F0010140EAC1014968696024
S214019160A16C00290FBFA564E16C896C0D60E564F4
S2140191700021AA6C116094F8581081F0010184F85E
S2140191805810002184F8571094F8591001F0010185
S21401919040EAC100B4F852108905890941F08801F6
S2140191A0016031BDF8B506000F4614461D461FBFC7
S2140191B0306800900098002801D1FF20F2BDF2F738
S2140191C07DFDDFF8580D400A400207F00F0140EA26
S2140191D04110342111FB076101F25702937803F025
S2140191E0010340EAC3035B680B67937803F001034E
S2140191F040EAC3035C60927891F8571002F00102CE
S21401920040EAC200AA0501F00101920D890141EA76
S214019210024141F088010160F3F75AF9009890F88D
S214019220941001F0DF0180F894100020F2BD18B40C
S21401923000281FBF04680094009C002C08BFFF2074
S21401924035D0342414FB0100B0F852409C4298BF3C
S2140192502346029C236001F00F01DFF8FC4D640AEF
S214019260640200F2520044EA4111847904F00104D8
S21401927041EAC40444F0100462608279007902F085
S214019280010241EAC2019A0500F00100920D800137
S21401929041F0100140EA024040F088000860009862
S2140192A090F8941001F0DF0180F89410002012BCB1
S2140192B07047F8B400281FBF016800910099002983
S2140192C008BFFF2054D0009AFF2182F888104FF083
S2140192D0FF34009A92F8943043F0020382F89430F7
S2140192E00022009B83F8982000F15803DFF82C5CDD
S2140192F06D0A6D0202F00F0645EA4615002645F096
S21401930008072E603E6045F0100745F018053E60E0
S2140193102E605E701E705E609C6112B9012580F839
S21401932058500025009E06EB8206521C343386F800
S214019330C050102ADADBDFF8243D1D60009A92F84F
S214019340943003F0FD0382F8943080F83C500222FA
S2140193508285009880F88C109F20009981F88400FF
S214019360009890F8941001F0DF0180F89410002026
S214019370F2BC704770B50446342010FB014582B03C
S214019380A86C009001F00F06DFF8CC0C400A4002F2
S214019390483540EA46106E7C06F0010640EAC606ED
S2140193A076681E60D30803F00103920802F00102FA
S2140193B040EA031343EAC20213681A0CC3F3830399
S2140193C0002908BF0D2B14D10122204600F0ACFF66
S2140193D0012084F85600012104F256004170C1783C
S2140193E081F00101C170817881F001018170002056
S2140193F076BDE97B81F00101E973697C81F00101A9
S2140194006974AB6A13F1010F07D081F0010140EADC
S214019410C10043604FF0FF30A86200980028E6D0F4
S2140194200098C068009989688842E0D29005DED02D
S2140194300099204600F0CAFC022076BD2DE9F04FC7
S2140194408BB00446002004902068039003980028FF
S21401945000F0E9800398DFF8002C90F8905003990B
S214019460082081F88000520A280901904FEA422814
S214019470E808019A00F00101A80848EA421200F043
S214019480010042EA011242EAC0000068C0F3094A3C
S214019490C0F383000D280CBF0126002601984FF06B
S2140194A0340909FB004000F14007002960D0016C37
S2140194B000910099CA685244CA600099C9680A9125
S2140194C000994968099100998968009AD268B1EBB8
S2140194D0020B02D0798A8A4510D2009A0021D170F7
S2140194E0016C009121B1896C0968016401B9796048
S2140194F0009818B120460099FEF73AFD0199C9B2C5
S21401950019FB014048EA4111026C02924030027E8A
S21401951002F0010241EAC20141F0100149680491DA
S214019520017E81F001010176817D81F00101817565
S214019530029850B10298C06802998968884204D09E
S2140195400299204600F0E4FB6DE0788A824502BF6E
S214019550BBF1000F0198002844D1DFF8001B012061
S21401956008600022002311462046FFF7E9F95AE079
S214019570DFF8E80A0168012904BF00210160B86824
S21401958000900098C1685144C1600098C0680A9074
S214019590009840680990009880680099C968411A47
S2140195A000988068002818BF002902D0788A824572
S2140195B010D200990020C870B868009020B1806C65
S2140195C00068B86000B9F860009818B120460099A4
S2140195D0FEF7CEFC019904AB2A46C9B22046FFF736
S2140195E0C9FE00BB0198002802BFDFF8700A0068B8
S2140195F050EA0A0004BF2046FFF784FD01988DF863
S21401960018000594E808079600F00100089005A9DF
S2140196100198C0B2FEF794FD039890F8941001F0FB
S214019620DF0180F894100BB0BDE8F08F2DE9F04F04
S21401963089B004001FBF206800900098002800F041
S2140196407681009890F88000009991F8841001EADC
S2140196500005A8072BD500208DF822002068009071
S214019660009820B3009890F89000009A022182F8A2
S2140196708010009991F88810009A92F88C20029434
S21401968011408DF822100109C0F3C0008DF80C10AE
S214019690059000210DF122000491069007911620F5
S2140196A002A9FEF74DFD0099FF2081F88800E80722
S2140196B040F187800026206800900098002800F07E
S2140196C080800099012081F88000B046009890F8CB
S2140196D090004FEA101BB1464FF6FF7A4FF0FF3766
S2140196E00194019878B3019800680090009850B3EF
S2140196F000223146204600F017FE00994144002022
S21401970081F8C00001984844C06D40B101984844B2
S214019710C06DF4F731FF019949440020C86506F091
S2140197200F01DFF83409400A400240EA4110476061
S21401973040F00800476001984844A0F852A0002075
S2140197400199494488660194019820B301980068FC
S21401975000900098F8B101223146204600F0E4FD61
S21401976000994144002081F8C00006F00F01DFF89F
S214019770E808400A400240EA411040F0100140F07B
S21401978018004F60476001984844A0F852A0002096
S21401979001994944C866761C09F1340908F10408A0
S2140197A0102E9DDB2046FFF784FD002004900590D7
S2140197B00690079002948DF80CB002A91020FEF7CF
S2140197C0BFFC280744BF2046FFF738FEE8062AD527
S2140197D020680090009830B30099202081F880001E
S2140197E01020009981F8800004F1340201212046FE
S2140197F0FEF7E6FC802201212046FEF71DFDFF2034
S2140198008DF80C00029400200490059006900790B5
S21401981002A91420FEF794FC009890F8841041F0F9
S214019820200180F88410A80620D5206800900098B2
S214019830E0B10099202081F880000121A28E204607
S214019840FEF7FAFCFF208DF80C000294002004902D
S21401985005900690079002A91320FEF771FC009868
S21401986090F8841001F0DF0180F88410680728D58D
S21401987020680090009820B30099042081F88000A9
S214019880009890F8A40000022086009991F8A01094
S214019890084320862020009981F8800002A90098BC
S2140198A090F89000029400098DF80C0000200490B6
S2140198B0059004F130000690002007901220FEF774
S2140198C03FFC680607D520680090009818B10099FB
S2140198D0402081F88000280629D50020ADF8200018
S2140198E020680090009810B30099802081F88000CD
S2140198F0FF2500200490069007900294059508AA7B
S21401990010212046FEF75CFCBDF82000012806BFAA
S21401991000208DF80C008DF80C5002A91720FEF7D8
S2140199200FFC9DF80C0010B92046FFF7EBFB09B0C1
S214019930BDE8F08F1CB50191019921B10199096823
S2140199400091009909B9FF2016BD019981F83600EA
S214019950019A0198DFF8C81990F83700F2F720FE4F
S21401996008B98A2016BDDFF8F0464FF4007120468C
S214019970F2F75CF80198FFF79CFC0099200A81F841
S2140199809C00200C009981F8B000200E009981F807
S214019990B400FF20009981F880009F20009981F88B
S2140199A084000120009981F89400009890F8001135
S2140199B001F07F0180F800118420009908770020CB
S2140199C016BD2DE9F04184B00D46009000260099A1
S2140199D021B1009909680291029909B9FF204EE167
S2140199E0A9780429BABF6A78022A952080F24781AD
S2140199F02978009C4FF0340818FB014404EB8203DD
S214019A009B6E012B08BF00F03DF968782978009A13
S214019A1018FB012101EB8000012181660099CE61CE
S214019A20E868002804BF6878002825D100980190CE
S214019A30F2F744F9019847690198406950B10198D5
S214019A4001994969896C096841610198406908B9B9
S214019A50019988610198016A491E0162F2F738FD91
S214019A602878387068787870A868B860E868F86010
S214019A70A878B87068697861A878012818BF0126A7
S214019A802C8A412CA8BF40242978009A18FB012172
S214019A9081F850002878009918FB0010697880F842
S214019AA051102878009918FB0010A0F85240287829
S214019AB0009918FB00100521A0F86010287800997D
S214019AC018FB0010002141660298297800EB8100FE
S214019AD090F8C010314380F8C010029869780029C8
S214019AE014BF042108212A7800EB820090F8C020D8
S214019AF0114380F8C010687800282878009918FB70
S214019B00001040F08C80002180F857106000009E05
S214019B10F4F7DCFE297818FB0161C8652A780098FD
S214019B2018FB02F10818C06D08B98120A7E0009B58
S214019B30DFF82405CB18400A93F85930400202F0AA
S214019B400F0240EA421203F0010342EAC302009BFD
S214019B50C918C96D5160E968002904BF69780029F0
S214019B6027D12978009B01F00F0218FB013140EA4A
S214019B70421291F8591001F0010142EAC101496807
S214019B8079602978009A18FB01F18A18926C002AEC
S214019B90009A02D189188F6403E08918C96C896C10
S214019BA00F602978009A18FB0121CF640021BA6C56
S214019BB01160A1052A78009E02F00F0318FB0262CD
S214019BC040EA431392F8592002F00102890943EA58
S214019BD0C20241F088031360009B2E7818FB06F240
S214019BE0D31806F00F0693F8593040EA461683F06C
S214019BF0010346EAC303009E9219D26DA2185A6069
S214019C002A7802F00F0340EA4310009B18FB023249
S214019C1092F8592082F0010240EAC2002BE00021AE
S214019C2080F85610A0052A78009C02F00F038109DF
S214019C3018FB0242DFF8200492F85820400A40023E
S214019C4040EA431302F0010243EAC20242F0100264
S214019C5041F0080313602A7802F00F0340EA43102C
S214019C60009B18FB023292F8582082F0010240EA6B
S214019C70C20040F0100041F048010160002004B02D
S214019C80BDE8F0817CB50D4600901446009921B1DF
S214019C90009909680191019909B9FF2076BD294605
S214019CA000F042FB019901EB8501002081F8C0001C
S214019CB0342010FB05F664B900983018C06D40B129
S214019CC000983018C06DF4F757FC00997118002001
S214019CD0C86505F00F01E048400A400240EA41101D
S214019CE004F0010140EA01104FF0FF31416040F0FD
S214019CF0080041604FF6FF7000997118A1F85200F4
S214019D0000210098301800EB84008166002076BDA3
S214019D1030B50C4683B0A168E268891A02910190B9
S214019D20019800B9E7E1E568C5B92178019A3420C0
S214019D3010FB01F18A18126C002A019A02D18918C7
S214019D400C6403E08918496C896C0C602178019ACF
S214019D5010FB012044640020A16C08600298626830
S214019D602178002802A800900EBF0023029BAA18A3
S214019D700198FFF75CFA050025D00020E07034203A
S214019D802178019A10FB01210C6C2178019A10FBB5
S214019D9001F18A18126C8AB1019A019BCB188918B5
S214019DA01B6C9B6C1B680B64217810FB01F00199FE
S214019DB04118096C11B9019A801841641CB12146F9
S214019DC00198FEF7D5F8284603B030BD30B583B00C
S214019DD00C4601900199002914BF002CFF2055D094
S214019DE0A168E268891A02913425E168B9B9217837
S214019DF0019A15FB01F18A18926C002A019A02D188
S214019E0089188C6403E08918C96C896C0C60217808
S214019E10019A15FB0121CC640021A26C1160217806
S214019E20019A029B15FB01F18A18B2F852209A4258
S214019E3004D2019A8918B1F85210029102A9009130
S214019E40E2686168029B52182178FFF7ABF9E8B126
S214019E502178019A15FB01218C6C2178019A15FB5A
S214019E6001F18A18926C8AB1019A019BCB18891864
S214019E709B6C9B6C1B688B642178019A15FB01F126
S214019E808A18926C12B9019BC918CA6403B030BD16
S214019E90F8B50D4600901446009900291EBF00999A
S214019EA00E68002E01D1FF20F2BD3421009A11FB6D
S214019EB005F7BA18012151662246294600F034FA00
S214019EC06548400A400205F00F0140EA411000993A
S214019ED0002C09D0791891F8581001F0010140EAD8
S214019EE0C10040F0100006E0791891F8591001F011
S214019EF0010140EAC10000997918B1F852108905AC
S214019F00890941F08C01016096F8940000F0DF00A9
S214019F1086F894000020F2BD000000000014FF1F28
S214019F20F0B583B00C460090009800281DBF00983D
S214019F300568002DFF2000F08C803420009910FB6E
S214019F4004F7791800204866002A05EB840090F88B
S214019F50C01001F0FD0180F8C01090F8C0101DD0AF
S214019F6041F0050180F8C01004F00F0200983A494C
S214019F703818490A90F85800490241EA421100F09F
S214019F80010041EAC0000099791840F01000B1F8CC
S214019F9052108905890941F0080152E041F0090192
S214019FA080F8C01000980190F1F788FE0198466984
S214019FB00198406950B1019801994969896C09680D
S214019FC041610198406908B9019988610198016A5F
S214019FD0491E0162F2F77CFA347000207070B0609E
S214019FE00098381890F85000B07001207061009801
S214019FF03818806C0028009802D13818866403E06F
S21401A0003818C06C806C066004F00F02009838188F
S21401A010C6640020B16C08600F4900983818490AD8
S21401A02090F85900490241EA421100F0010041EA64
S21401A030C00000997918B1F852108905890941F0D4
S21401A0408801016095F8940000F0DF0085F894001F
S21401A050002003B0F0BD00000014FF1F3C1EFF1FD0
S21401A06030B583B00C4600901546009800B942E022
S21401A0703420009910FB04F0002D16D04118096C0D
S21401A080019100994118096C29B30099009A821828
S21401A0904118126C926C12680A6400994118096C96
S21401A0A0C9B9009A8018416415E04118896C01917C
S21401A0B000994118896C71B10099009A821841186B
S21401A0C0926C926C12688A6400994118896C11B975
S21401A0D0009A8018C164019840B100200199C870A7
S21401A0E0019818B101990098FDF742FF01980028E0
S21401A0F0BED103B030BDFF2003B030BD82B00090AA
S21401A100009A22B1009A12680192019A02B995E06A
S21401A11039B1019A82F89810009A82F83C10012110
S21401A12081858EE000B583B00090009921B1009939
S21401A13009680191019911B9FF2003B000BD019A88
S21401A140002182F89410FF220121FEF775F800988D
S21401A1508068F4F711FA00980069F4F70DFA009890
S21401A160406AF4F709FA0098C068F4F705FA00980F
S21401A170F4F702FA002003B000BD83B00190019805
S21401A180002814BF002AFF2032D06648DDF804C03C
S21401A190400A400201F00F0340EA4310342313FB48
S21401A1A001C191F8591001F0010140EAC10040686F
S21401A1B000900098007810700098407850700098D1
S21401A1C0807890700098C078D070009800791071EF
S21401A1D00098407950710098807990710098C07904
S21401A1E0D0715088508090889080D088D080002090
S21401A1F003B0704782B00190019820B101980068C1
S21401A2000090009800B919E00099202081F880009C
S21401A210009890F8941001F0DF0180F894100098EF
S21401A22090F8941041F0040180F89410009890F88A
S21401A230941001F0FB0180F8941002E0FF2002B0B8
S21401A2407047002002B0704781B00090009810B9A6
S21401A250FF2001B07047009B342010FB0130B0F89E
S21401A2606000108001B00020704770B582B00C46C7
S21401A2700090FF23009D04F00F010DB9FF2076BD6D
S21401A2803425009E15FB01F5AE19012AA6F86020BB
S21401A29003D1E209FEF720F80CE0002A01BF009A7C
S21401A2A0AA18526E012A06D1009AAA1892F85120CD
S21401A2B0FDF76AFF0346184676BD82B00523019076
S21401A2C0019820B1019800680090009800B9B5E7A0
S21401A2D0102922DA009800EB8100002390F8C000D4
S21401A2E010F00C0F08BF052317D0800748BF0123C5
S21401A2F013D40C48400A400201F00F0140EA411015
S21401A30002F0010140EA01100178090604D440F088
S21401A31008000078000600D50323184602B07047EF
S21401A3202D9601000014FF1F70B504460D46164613
S21401A330F1F7C4FC60680369180008D03246294664
S21401A340204698470446F2F7C3F8204670BDFF2022
S21401A35070BD00002DE9F04304467348006883B0E1
S21401A360C5690FF2C81000F045F9EA680FF2DC1073
S21401A3702B46214600F03EF9EFF303800190EFF300
S21401A3800986EFF3088772467946009733460FF23F
S21401A390EC1000F02FF90FF22028404600F02AF9C1
S21401A3A0F0680FF2282901903146B0680090736872
S21401A3B03268484600F01EF9F069019006F1100176
S21401A3C0B069009073693269484600F013F9F06A83
S21401A3D0019006F12001B06A0090736A326A48461D
S21401A3E000F008F9F06B019006F13001B06B0090B7
S21401A3F0736B326B484600F0FDF8F06C019006F185
S21401A4004001B06C0090736C326C484600F0F2F874
S21401A410F06D019006F15001B06D0090736D326DD4
S21401A420484600F0E7F8F06E019006F16001B06E64
S21401A4300090736E326E484600F0DCF8F06F0190C3
S21401A44006F17001B06F0090736F326F484600F0EE
S21401A450D1F8404600F0CEF8F86801903946B86861
S21401A46000907B683A68484600F0C4F8F8690190A5
S21401A47007F11001B86900907B693A69484600F017
S21401A480B9F8F86A019007F12001B86A00907B6A72
S21401A4903A6A484600F0AEF8F86B019007F13001D1
S21401A4A0B86B00907B6B3A6B484600F0A3F8F86CEB
S21401A4B0019007F14001B86C00907B6C3A6C4846FD
S21401A4C000F098F8F86D019007F15001B86D009012
S21401A4D07B6D3A6D484600F08DF8F86E019007F1F5
S21401A4E06001B86E00907B6E3A6E484600F082F8C6
S21401A4F0F86F019007F17001B86F00907B6F3A6FAB
S21401A500484600F077F8F1F7E3FFA8680B2806D075
S21401A5100B20A860AC63686829680160486003B0D6
S21401A520BDE8F043F1F7CABB200AFF1F0A0D2A2A2D
S21401A5302A20554E48414E444C454420494E5445E8
S21401A5405252555054202A2A2A0A0D005665637421
S21401A5506F7220233A203078253032782054617388
S21401A5606B2049643A2030782530782054645F7037
S21401A570747220307825780A0D00000050433A2086
S21401A580307825303878204C523A203078253038CB
S21401A59078205053503A20307825303878204D5363
S21401A5A0503A20307825303878205053523A2030AF
S21401A5B078253038780A0D000A0D0A0D4D656D6F45
S21401A5C072792064756D703A0A0D00003078253076
S21401A5D03878203A20307825303878203078253081
S21401A5E0387820307825303878203078253038781B
S21401A5F00A0D00000EB430B5044603AD012000F08C
S21401A6000BF82B4622460349FAF758FD30BC5DF895
S21401A61010FB00BF5DA601000F49096880B205283E
S21401A62018D8DFE800F00E111403060AD1F89802D4
S21401A630704701F526704068704701F526708068FE
S21401A6407047C869406F7047C869806F7047C869AE
S21401A650C06F704700207047200AFF1F10B50446E0
S21401A66082B008000DD00368996911B92C21C16028
S21401A67007E08DF8004001229B6900A99847012850
S21401A68002D04FF0FF3016BD204616BD816807E0A8
S21401A69002681168536889185B18C3600832026043
S21401A6A0C2689142F4D04A1C82600878704738B577
S21401A6B004460D46A068E168884212D120686168A8
S21401A6C0884208BF00F0C5F82068227C016802B104
S21401A6D04944A16042685218E26008302060914205
S21401A6E0ECD0A068401CA06000F8015D31BD2DE9EA
S21401A6F0F0418AB000F1080105910168059A490800
S21401A70002EBC101069100210791089101684908F1
S21401A71000EBC10108310091017901F001018DF8CA
S21401A720101040680099400801EBC000019000201D
S21401A7300290039085E005A8FFF7A8FF044614F0F1
S21401A740030603D105A8FFF7A1FFC61C25090F2D97
S21401A7501BD105A8FFF79AFF00F10F0515E0059834
S21401A760016808180599079049680818089005981F
S21401A77008300590079808998842F0D0401C079049
S21401A78010F8011D00A8FFF792FF761EF2D1002DEA
S21401A79052D005A8FFF77AFF0646A00800F003008E
S21401A7A0032804BF05A8FFF771FFDDF800800299B2
S21401A7B0039F06EB002008E0A8F10808801A58F865
S21401A7C0041C58F8082C8F18394658F8082C8A1A91
S21401A7D08242F1D340424418AE1C2DD0BC4206D171
S21401A7E058F8044B58F8040B0719BC42F8D00298E5
S21401A7F0039914F8015B884217D1009801998842A1
S21401A80008BF00F026F8009800689DF81010029026
S21401A81009B148440290009902984968009A0918BB
S21401A8200832039100928842E7D00298401C0290B9
S21401A830761E00F8015DD1D10298039988427FF413
S21401A8407AAF0198009981427FF475AF0AB0BDE8EE
S21401A850F0810120F1F75EBC00000000000000005E
S21401A86001DF704701DFFEE77D48006872B6018BA5
S21401A87031B9416AC269D369994201D062B603DF30
S21401A88062B6704703DF7047FEE702DF704772B6B5
S21401A8901EF0040F0CBFEFF30881EFF309818969FD
S21401A8A011F8021C032905D100B500F01CF85DF86B
S21401A8B004EB16E0012902D16948006830E002295C
S21401A8C00FD167480068C1698A6842F001028A6050
S21401A8D000B54A680B6813605A6000F004F85DF82A
S21401A8E004EB62B6704707B55E48416811F0805FB9
S21401A8F007D1EFF31182A2F1100280F822205A4903
S21401A900416007BD72B6EFF3098C58498A78EFF3B8
S21401A91011832CE9FC4F52480068C369C3F814C080
S21401A92072B6416A0A688A420CD189680900F9D16F
S21401A93081F311884D49FF228A7062B630BF72B624
S21401A940016AEFE74162C261938C4383D2F814C077
S21401A950BCE8FC4F83F311888CF3098841484449CD
S21401A960416062B6704772B600B53D4B1B68198BE5
S21401A97001F101011983002001B4EFF31182EFF315
S21401A9800581586B07B4EFF30880586308461A6BC5
S21401A99002B92FE090422DD8DA6A811A2ADB9A6B27
S21401A9A04FEAD1014FEA8101515801B922E00A6804
S21401A9B022B1824203D009690942F8D11AE0C86877
S21401A9C04A6862B608B4904708BC72B607BC5863BA
S21401A9D001BC198B491E1983DA69906A10F4805FED
S21401A9E006D129B9596A0968914218BFFFF77BFF5A
S21401A9F062B600BD9A6AE4E772B6F1B4184B1B68FA
S21401AA00D3F834C00CF1100C5CF804EB194820F0B4
S21401AA100100CCF818009CE8FF005DF804CBACF10F
S21401AA20040C2CE9FF00F0BC8CF3088862B6704772
S21401AA3002B5017811F0800F03BF41F0800101706B
S21401AA404040802002BDEFF309807047EFF3088095
S21401AA50704780F308887047EFF303807047000063
S21401AA60200AFF1F00ED00E00000001020ED00E0CE
S21401AA7000000008C9A901007461736B5F32000011
S21401AA807461736B5F3100006D61696E5F74617331
S21401AA906B000000030000000F690100E8030000DE
S21401AAA00900000078AA0100000000000000000074
S21401AAB00000000002000000DD680100E80300005D
S21401AAC00900000080AA010000000000000000004C
S21401AAD0000000000100000055670100E8030000C7
S21401AAE00900000088AA0100010000000000000023
S21401AAF00000000000000000000000000000000050
S21401AB00000000000000000000000000000000003F
S21401AB1000000000737069303A00000073706932FB
S21401AB203A000000545331303230202D20537461E6
S21401AB306E64617264204447500000005C312A2A2A
S21401AB40205441424C45204552524F52202A2A0059
S21401AB5054533130323020416E616C6F6775652019
S21401AB6044475000312D536574757020444750207A
S21401AB704F7074696F6E7300322D44475020566FC4
S21401AB806C7461676520262043757272656E740069
S21401AB90332D4D65617375726520454F4C205265A6
S21401ABA0736973746F727300342D56657273696FAF
S21401ABB06E000000352D466163746F72792044651E
S21401ABC06661756C747300005C3125735C37302DDB
S21401ABD0457869742C204D656E753A20000000009A
S21401ABE031304B204F686D00344B37204F686D0075
S21401ABF0324B32204F686D00364B38204F686D005F
S21401AC00354B36204F686D00334B37204F686D004B
S21401AC10334B33204F686D00324B30204F686D0048
S21401AC20314B35204F686D00314B30204F686D0039
S21401AC30324B322F364B38204F686D005C31454F12
S21401AC404C205265736973746F723A2025752D25F1
S21401AC50735C37436F64653A200000005374616E7D
S21401AC606461726420536972656E00004443205625
S21401AC706F6C7473000000005C31536972656E205E
S21401AC804D6F64653A2025752D25735C374D6F64CD
S21401AC90653A20005C31496E7075742052657365A3
S21401ACA0742054696D65723A2025755C3754696D58
S21401ACB0652028536563293A200000005C31496EFF
S21401ACC070757420457870616E6465722025753ADA
S21401ACD02025735C372A2D4368672C20302D457854
S21401ACE069743A2000000000545330303231202875
S21401ACF05638290054533130323120285631302904
S21401AD00000000005C315C3243616E27742075736D
S21401AD106520454F4C2028257329207769746820C3
S21401AD205453303032315C37526573656C656374E9
S21401AD3020454F4C210000005C315C3243616E2798
S21401AD40742075736520545330303231207769741E
S21401AD50682073656C656374656420454F4C5C3789
S21401AD6054533130323120706C65617365210000B7
S21401AD705C315C325761726E696E673A204261647B
S21401AD8020454F4C2F457870616E64657220636F65
S21401AD906D62696E6174696F6E5C37506C65617364
S21401ADA065206669782100005C314447503A2025C9
S21401ADB073562C2025734120204261747465727984
S21401ADC03A202573415C374E455854206F72204512
S21401ADD04E544552000000005C314D65617375723A
S21401ADE06520454F4C205265736973746F72735CAE
S21401ADF037496E707574204E6F2028302D416C6C6B
S21401AE00293A20005C3125752D25735C37496E7013
S21401AE107574204E6F2028302D416C6C293A200025
S21401AE205C3125735C374E455854206F7220454E71
S21401AE30544552005C314275696C64204461746506
S21401AE403A20000020617420000000005C31426F4F
S21401AE506F746C6F61646572205665723A200000EB
S21401AE605C31526573746F726520466163746F72EC
S21401AE70792044656661756C74733F5C37312D5972
S21401AE8065732C20454E5445522D4E6F3A200000D6
S21401AE905C31416C6C204F7074696F6E7320526523
S21401AEA073746F7265645C37507265737320454EB8
S21401AEB0544552003CAB010050AB010064AB0100AD
S21401AEC078AB010090AB0100A8AB0100B4AB010068
S21401AED0C8AB0100E0AB0100E8AB0100F0AB01003C
S21401AEE0F8AB010000AC010008AC010010AC010099
S21401AEF018AC010020AC010028AC010030AC010008
S21401AF003CAC01005CAC01006CAC010078AC01000B
S21401AF1094AC0100BCAC0100E8AC0100F4AC01004B
S21401AF2004AD010038AD010070AD0100A8AD01000F
S21401AF30D8AD010004AE010020AE010034AE010020
S21401AF4044AE01004CAE010060AE010090AE0100BF
S21401AF507E5C312843292032303134205554432039
S21401AF604669726520262053656375726974792077
S21401AF704175737472616C696120502F4C5C3700A7
S21401AF804000000003000000006CDC02C01200005C
S21401AF90430000004400000003000000040000001D
S21401AFA04000000005000000006CDC0200C2010049
S21401AFB047000000480000000300000004000000F5
S21401AFC0467265657363616C652F4672656573636A
S21401AFD0616C65204D515800000000000000000023
S21401AFE0000000000000000000000100000000005A
S21401AFF0002D3101006CDC020000000000010000A1
S21401B0000001000008000000100000000900000018
S21401B010110000000100000000000020F0FF0020E9
S21401B0200004000094AA01000200000002000000D3
S21401B03010000000000000000000000000000000FA
S21401B04000000000570BFFFF0C130000440BFF1F0E
S21401B050000000009BF6FFFF020000000200000057
S21401B06048000000250000000000FF1F000400004B
S21401B0707FF6FFFF02000000020000005100000002
S21401B0805C0400000004FF1F4407000063F6FFFF96
S21401B090020000000200000091040000030000000E
S21401B0A00000002004000000F00900F0FE002081EE
S21401B0B0AC000067A90104E101838FA818F2060518
S21401B0C024F1FF11F5FF21F9FF31F96FB0F0010C02
S21401B0D0000A000152FF01110B13010104100304C1
S21401B0E0000100050D120604120704120E10120FBD
S21401B0F008121204F3351A0001921208D2121461D2
S21401B100071004010F0100010E04120D04120C04B5
S21401B110120B04120A04120904120804121704126C
S21401B1201304121504121104121604121204121436
S21401B13004121004122704122304122504122104F7
S21401B14012260412220412240412200412470412A6
S21401B15043041245041241041246041242041244E6
S21401B16004334001841208FC120904120C046056D0
S21401B17025049909F00B7B0EB202B7065E09580D3D
S21401B1808D0122047806E30B62032108B40AF40D4C
S21401B19003036207040AA50D4A02D6057408E80CE3
S21401B1A01C0270050408B00C7001DB031E06B30B0D
S21401B1B023011B031C05240BCF004002DB036A0A94
S21401B1C094029402D907440D5054308F0125047C13
S21401B1D006E50BF8005002F403790A10025305E461
S21401B1E007A00CC901AF0425073E0C49017B039F4C
S21401B1F0056D0B2C0130033905340B001029D108DD
S21401B20084087A017A014A05CF0B00044CC4011464
S21401B210AB015C5108F2061C1870090004080C10FA
S21401B22014181C69746D1C6002441EFF1F207001F7
S21401B230656F6C189245187001736D641892461804
S21401B240700169657418524718F315070001F00D6F
S21401B25014556E617661696C61626C650024AB01A0
S21401B2603459D0F15C03217110034D8C0100EF04B9
S21401B27012B30412C50412D50412EB0410031F8D79
S21401B2800100F3083401010301A7100302020100C3
S21401B2904008400103020008110418028C07FF1F32
S21401B2A0BF220213100660152014020001022F109F
S21401B2B00300090243002F1401C03209D122011FE5
S21401B2C0101A0524001001052401010104240206B8
S21401B2D005240600010705810310000A0904412D13
S21401B2E0F003100207058202592001070503071023
S21401B2F0220004030904180349006E007400650067
S21401B30072006C006F006700690078002E002C0345
S21401B310430068006114126C1C126E18212210057D
S21401B3202000560031003008325310326922230AB9
S21401B3300314123204300700002203420041004485
S21401B3402210075400520049004E00470E210820E3
S21401B35003440045005878280108FF1F8712E408B7
S21401B36025242DE403F60A434416AC0443C0072CF7
S21401B370E104500304182C0A225412080412200473
S21401B380124C04125804251B12D008D3C8083C29B5
S21401B3902F22C20532080F2F50AF14041C484567F0
S21401B3A089ABCDEFFEDCBA987654321078A46AD712
S21401B3B056B7C7E8DB702024EECEBDC1AF0F7CF5D3
S21401B3C02AC68747134630A8019546FDD898806956
S21401B3D0AFF7448BB15BFFFFBED75C892211906B40
S21401B3E0937198FD8E4379A6FA036CBF4962251EB8
S21401B3F0F640B340C0515A5E26AAC7B6E95D102F83
S21401B400D65314440281E6A1D8C8FBD3E7E6CDE1C2
S21401B41021D60737C3870DD5F4ED145A4505E9E360
S21401B420A9F8A3EFFCD9026F678A4C2A8D4239FA34
S21401B430FF81F6718722619D6D0C38E5FD44EABEF9
S21401B440A4A9CFDE4B604BBBF670BCBFBEC67E9BCD
S21401B45028FA27A1EA8530EFD4051D880439D0D40F
S21401B460D9E599DBE6F87CA21F6556ACC4442229CF
S21401B470F497FF2A43A72394AB39A093FCC3595BE7
S21401B4806592CC0C8F7DF4EFFFD15D84854F7EA84D
S21401B4906FE0E62CFE144301A3A111084E827E53F1
S21401B4A0F735F23ABDBBD2D72A91D386EB2C0323CC
S21401B4B0A12006760237960143FD037603F10718AD
S21401B4C0A11CF2060128F10760D20124F1030C4009
S21401B4D004CD8601002B8712610812B70843C38882
S21401B4E00C12F90C12130C12690412830452AB18D5
S21401B4F0100735990100119D0100CD041361A0309C
S21401B5001110100B859C0100219F010049A201002A
S21401B5106B0412BB0412FD1C100325A101007B0461
S21401B52012F5040002919E010012000100000000C5
S21401B5300000000000000000000000000000000005
S21401B54000000000000000000000000000000000F5
S21401B55000000000000000000000000000000000E5
S21401B56000000000000000000000000000000000D5
S20501B8000041
S903ACCD83
